:1000000000800020BD01000071C5000029C500006E
:1000100029C5000029C5000029C5000029C5000028
:1000200029C5000029C5000029C5000071C50000D0
:1000300071C5000029C50000F1BB0000F5BC00003F
:1000400071C5000071C5000071C5000071C50000D8
:1000500071C5000071C5000071C5000071C50000C8
:1000600071C5000071C5000071C5000071C50000B8
:1000700071C5000071C5000071C5000071C50000A8
:1000800071C5000071C5000071C5000071C5000098
:1000900071C5000071C5000071C5000071C5000088
:1000A0002DA1000039A1000071C5000071C500003C
:1000B00071C5000071C5000071C5000071C5000068
:1000C00071C5000071C5000071C5000071C5000058
:1000D00071C5000071C5000071C5000071C5000048
:1000E00071C5000071C5000071C5000071C5000038
:1000F00071C50000DDE5000071C5000009E70000E2
:1001000071C5000049CF000071C5000071C5000035
:1001100071C5000071C5000071C5000071C5000007
:1001200071C5000071C5000071C5000071C50000F7
:1001300071C5000071C5000071C5000071C50000E7
:1001400071C5000071C5000071C5000071C50000D7
:10015000E1BD0000F5BD000009BE00001DBE0000AD
:1001600071C5000065D2000071C5000071C50000B6
:1001700071C5000071C5000071C5000071C50000A7
:1001800071C5000071C5000071C5000071C5000097
:1001900071C5000071C5000071C5000071C5000087
:1001A00071C5000071C5000071C5000071C5000077
:1001B00071C5000071C5000071C50000564B4CF2BE
:1001C000205210B51A804DF628121A8000BF00BFC9
:1001D0000CF0D2F9514B4FF010621A60504A9A60FD
:1001E000504ADA60504A136813F4807304D14F49BF
:1001F0000B604FF4A85313604D4B1A78110703D5C9
:100200001A7842F008021A704A4B4B492A221A7097
:100210004A4A4B4B8B4204D252F8040F43F8040B6A
:10022000F8E7484B484900228B4202D243F8042B9E
:10023000FAE74649464A002352F8230041F82300D2
:1002400001336F2BF8D1434B434A802103F8011B44
:100250009342FBD1414B3D4A1A60414B8A221A70AE
:10026000A3F5805324225A70A0221A709A7992071B
:10027000FCD59A79D406FCD43A4A937903F00C035E
:10028000082B384BF9D103221A7140225A719A79FE
:100290009006FCD5334A9179324B4906FBD5324A58
:1002A000324911600221516020221A709A7902F0BD
:1002B0000C020C2AFAD12E4B2E4A1A602E4B2F4AD2
:1002C0001A6000225A60072243F8042C2C4AC3F813
:1002D0000C2D62B60CF000FD144B1B68DA0705D537
:1002E00028480CF0CDFA284B284A1A60284B1B7876
:1002F0005B0609D5244C254B22689A4204D121483B
:100300000CF0BEFA002323600FF0B6FC0CF03AF9B3
:100310000CF068F8FEE700BF0E2005403080044076
:10032000823F04000100002B10D0034014D0034092
:1003300002D0074000E00740349BFF1F94340100C7
:100340004088FF1F349BFF1F24A3FF1F0082FF1F55
:100350000000000000E400E05FE400E008ED00E0E1
:100360000050064000400640448004400000030165
:1003700004800440C010050014E000E0FF76010096
:1003800000002020BF32185F1CE00340A5C3945A30
:1003900000F00740FFFFFFFFFFFFFFFFFFFFFFFF32
:1003A000FFFFFFFFFFFFFFFFFFFFFFFFFFFFFFFF5D
:1003B000FFFFFFFFFFFFFFFFFFFFFFFFFFFFFFFF4D
:1003C000FFFFFFFFFFFFFFFFFFFFFFFFFFFFFFFF3D
:1003D000FFFFFFFFFFFFFFFFFFFFFFFFFFFFFFFF2D
:1003E000FFFFFFFFFFFFFFFFFFFFFFFFFFFFFFFF1D
:1003F000FFFFFFFFFFFFFFFFFFFFFFFFFFFFFFFF0D
:10040000FFFFFFFFFFFFFFFFFFFFFFFFDEF9FFFF23
:1004100010B5054C237833B9044B13B10448AFF33E
:1004200000800123237010BD349BFF1F00000000DB
:1004300098340100084B10B51BB108490848AFF3C8
:1004400000800848036803B910BD074B002BFBD0A0
:10045000BDE81040184700BF00000000389BFF1F98
:1004600098340100349BFF1F0000000038B504469B
:10047000104621700A491D460FF0E0F901464FF081
:100480007E500FF08FFA07490FF0D8F9E5606060F1
:10049000256165610CF0B0FBE061204638BD00BF0E
:1004A000DB0FC9400024744938B50446104621705A
:1004B00009491D460FF0C2F901464FF07E500FF07A
:1004C00071FA06490FF0BAF9E5606060256165616F
:1004D0000CF092FBE06138BDDB0FC9400024744989
:1004E00038B503780446032B20D8DFE803F01A1848
:1004F0001002C16840690FF097F80D490546606821
:100500000FF050FA014628460FF04CFA38BD084962
:1005100040680FF047FAE1680FF090F938BDC06805
:1005200038BDC16840690FF07FF838BD002038BD84
:100530000024744970B504460E460CF05DFB054678
:10054000E069281A0FF026F9E3682361E561666126
:10055000A061014660680FF025FA0146A0601048CE
:100560000FF020FA0EF0F6FC0EF096F90FF008F8F6
:10057000054601464FF07E500FF056F861690FF0C6
:100580005DF92169064628460FF058F901463046C4
:100590000FF04CF8E0602046BDE87040FFF7A0BFC8
:1005A000000080BF08B50E200BF0F6FD114B1B8834
:1005B000012B19D0104B1B88984213DB40F6FF71BA
:1005C0008842D4BFC3EB0001C3EB0101C1EB013191
:1005D000C3F57F630F33282091FBF3F1BDE808409A
:1005E0000CF060B90021F3E70146BDE80840142093
:1005F0000CF058B9609DFF1F109CFF1F10B50446FA
:100600000BF0CCFB204610BD70B44C88A04220D922
:1006100001230133DBB21CB2660031F8144084427E
:100620001D46F6D3A04211D005F10045013D965B71
:1006300031F8151032F81530401AF21A00FB02F0AA
:10064000641A90FBF4F4E01870BC7047905B70BCC7
:10065000704702260125E5E700280CDA064A4342E6
:1006600082FB0320DA17C2EB600000EB4000A3EB33
:100670008000C0F10C007047ABAAAA2A2DE9F04710
:100680000C200BF055FD0C200CF00AFA9C491420AC
:100690000CF016FA9B499C4809F04EFA02210320FF
:1006A0000CF0A4FA022104200CF0A0FA022105208B
:1006B0000CF09CFA022106200CF098FA01210A2085
:1006C0000CF094FA012109200CF090FA01210D2080
:1006D0000CF08CFA012128200CF088FA012114205A
:1006E0000CF084FA02210B200CF080FA01210C207E
:1006F0000CF07CFA0C2000210CF064FA04200CF0C1
:1007000067FA70B305200CF063FA044680B3002446
:1007100020467E4D287006F04FFC2B78EBB9204622
:1007200008F05CF87A4B7B491B887B4C09887B4A34
:100730002170A3F5AF7140F23A7303FB01F382FB22
:100740000312DB17764D7748A3EB621332335A213D
:100750002B6009F09BFD90B9FEE7BDE8F04709F07A
:10076000FBB806200CF034FA0028CBD10124D0E7E6
:1007700003200CF02DFAB0FA80F04009C9E76A4A6C
:100780006A481268DFF8F8A100230121FFF78CFE08
:100790000B200CF01DFA011E0CBF012300238AF868
:1007A000003002D111200CF021FADFF89081604E68
:1007B000604F614D0023C8F8003033603B604FF05C
:1007C000040914E00BF0E8FC33681844306009F0C9
:1007D000010080F0010005F013F92B88002B14BFF5
:1007E0004B20DC200CF02AFAB9F1010919D00F20B6
:1007F0000CF016FC3B6803440E203B600BF0CCFC75
:10080000D8F800309AF800200344C8F800301520CA
:10081000002AD7D111200CF003FC33681844306053
:10082000D5E73B68D8F8002044493068DFF854E148
:100830002D88002BB8BF0333002AB8BF03329210B3
:100840000A603F493F4A0988128800284FEAA303FB
:10085000B8BF03303B6080103B4F30605E1A1944D4
:100860003E60CEF80010394F394E3A49C2EB000EC7
:100870000244C7F800E032600B605DB94FF4FA70D3
:1008800005F0CEF805F0B8F806F09EFE4FF4AF6024
:100890000CF0D4F9304B012504201D600CF098F9C0
:1008A00010B92E4B20701D702D4B1B881C2B1CD09B
:1008B0002C4C04F1C80523200BF06EFC44F8040F07
:1008C00001200CF0BBF9A542F5D1274A274B10783F
:1008D000187007F08DFE05F08BF845F6BF522449DD
:1008E0002448BDE8F0470BF00FBA234B18880028C6
:1008F000DED0224BC0B2197807F0C2FDD8E700BFA6
:10090000001B374640420F003C90FF1F949BFF1F87
:10091000B49DFF1F949DFF1FE49BFF1FB5814E1BDD
:100920009489FF1F049CFF1F2489FF1F289DFF1F20
:10093000509BFF1F809DFF1F569DFF1F689BFF1F41
:10094000A689FF1F2C89FF1F849DFF1FDC9DFF1FB1
:10095000E89BFF1FD09DFF1F8C9DFF1F829BFF1FE9
:10096000929DFF1F1C9CFF1F149DFF1FFA9CFF1FE1
:10097000A5050000A89DFF1FEC9BFF1FB09BFF1F5C
:10098000709DFF1FFC9CFF1FF0B40E8886420DD2A5
:1009900003F10043013B31F81350854202D9F0BC0A
:1009A000FFF732BE32F81300F0BC70471088F0BC7D
:1009B000704700BF094B1B880C2B09D8084A80B22E
:1009C00052F8232028B143F6FE73984203D9108CC5
:1009D0007047108870470349FFF716BE909BFF1FB2
:1009E000A00F0100A4110100374A38491088384A85
:1009F000F8B5384B12881B68834248DB9342A8BF86
:100A0000134698420B60C8BF002342DD101AB0F5B0
:100A1000804FAABF9B03C3EB8333013093FBF0F0FD
:100A2000FFF7C8FF2C4B2D4F1C883B68C0F3C61541
:100A300005FB04F47F2CA8BF7F249D42064608D006
:100A4000274B1B88002B38D1264B1B88002B30D11D
:100A50003D60254D2B689E4205D0214B1B885A1FB7
:100A6000032A1DD92E60214D2B689C420ED0204BAD
:100A7000188848B11A4B1F4A1B88D35C834203D0A5
:100A8000C0B2E1B207F0FCFC2C60F8BDF8BD034633
:100A900008609A42D4BFC0EB0203C0EB0303B5E782
:100AA000144AD05C2030C0B206F07F0107F0E8FCA9
:100AB000D8E7284607F058FDCAE70E4A2946D05C19
:100AC00007F0DEFCC0E700BF109CFF1F589BFF1F14
:100AD000BC9DFF1F5C9DFF1FA09BFF1FC49BFF1FB2
:100AE0004A9DFF1F069CFF1FC89DFF1F089CFF1FFC
:100AF000969DFF1F9889FF1F2DE9F04F172089B0A1
:100B00000CF08EFAAF4B186016200CF089FAAE4B41
:100B1000AE4A1B8810600C2B00F03B81AC4BAD4AF9
:100B200019880093AC4B52F8214000221A70AB4B4D
:100B3000AB4D1B88AB4A2E88013B32F91370002E57
:100B40005CD0A94BA94A1B88A9491278013B31F90D
:100B50001380002A40F0DF8011200CF061FAA54BD1
:100B60000193D3F800A00646B24540F3DF80A24BC4
:100B7000DFF8A4921B88A14A012BD9F80030B2F803
:100B800000B09F4A02922046C8EB030800F09A8208
:100B90000EF000FE029A52F82B100EF04FFE0146A6
:100BA00000200EF041FD0FF00FF8CAEB0802B0452F
:100BB000B8BFB0469042CAEB080880F2968200FBAC
:100BC0000888013298FBF2F08E4BDFF850820293D6
:100BD000D8F80030034403EBD3735B10C8F800303F
:100BE0002B88012B12D1884BDFF834B20393874B4B
:100BF000DBF8005004934FF0000A47E07D4B01936F
:100C0000DFF814927F4BDFF8148202937E4B03933C
:100C10001D460F200CF004FA2B689842824641DAF8
:100C2000754A1288012A00F01D82744A05931288C1
:100C3000734D049220460EF0ADFD049ADFF8E0B14A
:100C400055F82210DBF800500EF0F8FD01460020A8
:100C50000EF0EAFC0EF0B8FFEF1B059B5745A7EB23
:100C60000302B8BF5746FF1A9042BABF013200FBD9
:100C70000777474397FBF2F7D8F80020634B0493BC
:100C8000BB1803EBD3735B10C8F80030604B1B88B4
:100C9000013B032B00F2B082DFE813F06301A901EE
:100CA000C4008601594B04931B68984240F3C281EB
:100CB000514A1288012A00F0A682504A07931188EF
:100CC0004F4A0691204605920EF064FD059A06995A
:100CD000DFF84CB152F82110DBF800500EF0AEFDF9
:100CE0000EF072FF079B2F445745A7EB0302A8BFE6
:100CF0005746FF1AD8F800309042BABF00FB07777A
:100D00000132474397FBF2F73B4403EBD3735B108D
:100D1000C8F80030BAE715200BF03EFA354B0193C6
:100D2000D3F800A00646B2453FF721AF354B0293FA
:100D3000D3F800A0B24580F289812F4BDFF8D8901C
:100D40001B882E4A012BD9F80030B2F800B02C4A8B
:100D500003922046984400F070820EF01BFD039A27
:100D600052F82B100EF06AFD0EF02EFFB045CAEBC4
:100D70000802A8BFB046CAEB08089042B6BF00FB05
:100D8000088800FB08F8013298FBF2F0DFF88C804D
:100D90001EE7204B1B78002B3FF4C0AE0C4B0D4AD6
:100DA000198800930C4B52F8210001221A700EF0A2
:100DB000F1FC4FF07C510EF041FD0EF005FF0446B2
:100DC000B5E600BFBC9BFF1F929DFF1FD89DFF1F74
:100DD000C09BFF1F5889FF1F629BFF1FA489FF1F35
:100DE000049DFF1F8C130100AA89FF1F709DFF1F28
:100DF00080110100DC9DFF1FF49BFF1F8C9BFF1FD8
:100E0000A4130100E89BFF1F849DFF1FFC9CFF1F94
:100E10002E89FF1F489DFF1F509BFF1F9C9DFF1F9A
:100E2000809DFF1F28460EF0B5FCB2490EF006FD6E
:100E3000054650460EF0AEFCAF490EF0FFFC0146F1
:100E400028460EF0F3FB0EF0BFFE0546CBF800502F
:100E5000D9F800000EF09EFCA6490EF0EFFC074604
:100E600030460EF097FCA4490EF0E8FC01463846E7
:100E70000EF0DCFB0EF0A8FEC9F800009F4AA04B64
:100E8000168819889F4AA04B12681B889F4FC6EB93
:100E9000050E3544039EC6F800E0461A084404993E
:100EA0000D6001990E6002993E8808609A4280F2B6
:100EB00089810025C3EB060E954974450F6880F2C1
:100EC0007681611C9F4205FB01F50EF1010E95FB39
:100ED000FEF5C0F2BE81BE42A8BF3E46F61A01FB37
:100EE00006F494FBFEF49A4200F33681BB42C0F252
:100EF0003381884C20680EF04DFC87490EF09EFC33
:100F000086490EF093FB0EF05FFEA0F5FF531C3BED
:100F1000082B98BF4FF40050D8F800301844002830
:100F20002060C0F24281B0F5804F80F252817C4B4C
:100F30001B781BB1B0F5005F40F05381794D2B78E1
:100F4000002B40F05481784D20682B68714C9842FA
:100F500004D080B207F072FB23682B6009B0BDE8B3
:100F6000F08F28460EF016FC70490EF067FC05461F
:100F700050460EF00FFC6E490EF060FC014628460C
:100F80000EF054FB0EF020FE0546CBF80050D9F8C9
:100F900000000EF0FFFB65490EF050FC074630469E
:100FA0000EF0F8FB62495FE728460EF0F3FB5A4962
:100FB0000EF044FC054650460EF0ECFB5D490EF089
:100FC0003DFC014628460EF031FB0EF0FDFD0546C6
:100FD000CBF80050D9F800000EF0DCFB4E490EF0C3
:100FE0002DFC074630460EF0D5FB52493CE728461B
:100FF0000EF0D0FB50490EF021FC054650460EF095
:10100000C9FB4E490EF01AFC014628460EF00EFBB5
:101010000EF0DAFD0546CBF80050D9F800000EF0CE
:10102000B9FB45490EF00AFC074630460EF0B2FB0C
:10103000424919E7D8F80030DFF810B103EBD37359
:101040005B10DBF80050C8F800301FE6DFF80081C5
:10105000DFF80091D8F8003003EBD3735B10C8F8C9
:101060000030BDE5364A06931188364A0591204680
:101070000492DFF8D8B00EF08DFB049A0599DBF8E6
:10108000005052F821100EF0D9FB0EF09DFDEF1B21
:10109000069B5745A7EB0302B8BF5746FF1AD8F87F
:1010A00000309042BABF013200FB0777474397FBFD
:1010B000F2F73B4403EBD373234A04925B10C8F866
:1010C0000030E3E50EF066FB029A52F82B100EF0AA
:1010D000B5FB0EF079FDCAEB0802B045B8BFB046CB
:1010E0008242CAEB08083FF76AAD00FB08F898FB9C
:1010F000F2F069E5CDCC4C3FCDCC4C3EA689FF1F2C
:101100002C89FF1FBC9BFF1F5A9DFF1FA29BFF1F27
:10111000D89DFF1F8C89FF1F9A99193FCDCC4C4554
:101120008E9EFF1F059CFF1F2089FF1F3333733FD7
:10113000CDCC4C3DCDCCCC3E6666663FCDCCCC3DD7
:101140008C9BFF1FA4130100FC9CFF1F809DFF1FB1
:101150009C9DFF1F509BFF1F009B1B88002B3FF493
:10116000C8AE2B1B002BB8BF5B42092B47DD05F532
:1011700000500130001B0EF00DFB3B493B4C0EF0C4
:101180005DFB054620680EF005FB39490EF056FB65
:10119000014628460EF04AFA0EF016FDD8F8003047
:1011A000184400282060BFF6BEAE002213E09F4224
:1011B00005FB04F5B8BF002195FBFEF54BDA91FB6A
:1011C000FEF490E6B242D4BFC3EB0205C3EB0605C2
:1011D00070E643F6FF72274B22601B78002B3FF42A
:1011E000ADAE04F009FC244B01221A70ABE604F00A
:1011F000FFFB00232B70A6E6D9F800003EE64FF473
:1012000000501A4C88E61D491D4A069320460D8859
:1012100005920EF0BFFA059ADFF868B052F8251073
:10122000DBF800500EF00AFB014600200EF0FCF93E
:101230000EF0CAFC2F44069B56E50EF0ABFA039A5B
:1012400052F82B100EF0FAFA014600200EF0ECF9DD
:101250008AE51E4642E6B742D4BFC3EB0701C3EBA3
:10126000060104FB01F1AAE7CDCCCC3E8C89FF1F1F
:101270009A99193F8E9EFF1F059CFF1F8C9BFF1F95
:10128000A4130100809DFF1F08B5244B1B88FBB1F0
:10129000234B1B78FBB1234B1B78E3B1224B1B780C
:1012A000CBB1224B1B78B3B1214B22481A78C2B97B
:1012B000214A22490088128809680244B1EB620F72
:1012C00009DD01221A706420BDE8084004F0A8BBC3
:1012D000174A117801B908BD1370BDE8084007F03E
:1012E00077B9154A16490088128809680244B1EB9B
:1012F000620FF0DD00221A7007F06AF9642004F032
:101300008FFB642004F08CFB642004F089FB4FF415
:101310001670BDE808400BF091BC00BF069DFF1F92
:10132000E59DFF1FB69DFF1FB79DFF1FB89DFF1FC7
:101330008E9BFF1FA29BFF1F5A9DFF1FBC9BFF1F81
:10134000D89DFF1F38B5114C232025780AF024FFC3
:101350000F4A42F82500131F02F1C400002253F87F
:10136000041F83420A44FAD123780A4907480A4CE9
:101370000133DBB2322B81FB025108BF0023D217AD
:10138000C2EB21120370226038BD00BF7A9BFF1FA1
:10139000209CFF1F1F85EB517C9DFF1F2DE9F04F07
:1013A000B84CB94D2068B94F83B00EF0F3F9B84985
:1013B0000EF044FA064610200BF032FE0EF0EAF969
:1013C000B4490EF03BFA31460EF030F90EF0FCFB5A
:1013D0002988206088423B8843DA9E465B1A7F2B2F
:1013E0004FF0000247DDD2015E1C92FBF6F2AA4EDE
:1013F000DFF8C882B6F800C0C8F80020BCF1190FA9
:1014000000F0DF80BCF11A0F00F01781BCF11E0F55
:1014100000F020810126B146A04A1288002A00F07F
:101420009D808842C0F207817045D4BFC1EB0000A7
:10143000C1EB0E009A42BABF02FB000001335043D9
:1014400090FBF3F3964A1360964B1888C0B9964AFE
:101450001288AAB9954B197801B11A7003B0BDE88A
:10146000F08F9842D4BFC1EB0002C1EB03029E464D
:101470005B1A7F2BB7DCC2EBC21292FBF3F2B6E72A
:101480002988D4F800E0DFF80082DFF8F8A1714580
:101490006CDCDFF818C29CF80020002A2ED14FF037
:1014A000010B04288CF800B028D1002E40F0948164
:1014B0007D4B18880028D1D0B9F1000FCED0236819
:1014C0002C883A88A34280F265810023141B7E2C6D
:1014D000774DD5BFC3EB8313C3EBC3135B0001345C
:1014E00093FBF4F42B680134A34203D0C0B2E1B201
:1014F00006F0C6FF2C6003B0BDE8F08F012800F0B5
:10150000F680022800F0EB800328D1D1694B1B88BC
:10151000092BCDD0002ECBD023682E883A88B34239
:1015200080F27B810023961B7E2EDFF88CA1D5BF35
:10153000C3EB8313C3EBC3135B00013693FBF6F6D7
:10154000DAF800300136B34203D0F1B24A2006F097
:1015500097FFCAF80060ABE716469146BCF11E0F34
:101560007FF472AF0022DFF858817EE04F4B1A788B
:10157000002A3FF473AF002401281C7000F0A480FF
:10158000022840F00E81002E00F0A3804A4D2B6807
:10159000002B00F09E800420214606F071FF424B94
:1015A0002C60188800283FF459AFB9F1000F3FF4C0
:1015B00055AFC0B2002106F063FF3D4B00221A6018
:1015C0004CE7DFF8FC8098F80020C2B1DFF8D89033
:1015D000B9F800A0BAF1000F11D0DFF8E89099F83F
:1015E00000B0934578D05FFA8AF07F2106F048FF7B
:1015F00098F80030B6F800C089F8003010E0DFF845
:10160000C49099F800A0924566D0274B0021187825
:1016100006F036FF98F80030B6F800C089F80030C0
:101620001E4B1A88002A97D0BCF11E0F40F006818D
:101630000026B14619E00020FCE6DFF8848098F827
:101640000020002A0BBF012600264FF000094FF0B2
:101650000109E1E6DFF86880104B98F800601A880D
:10166000B6FA86F676094FF0000998F80030002B9C
:101670003FF4E8AE2988B7F800E02068C1EB0E031C
:10168000CFE600BFB49BFF1F0C9DFF1F089DFF1FEF
:101690009A99193FCDCCCC3E929DFF1FC49DFF1F50
:1016A000189CFF1FBA9BFF1FA29DFF1F999DFF1F44
:1016B000989BFF1F4A9DFF1F1C9CFF1F749DFF1FCF
:1016C000489DFF1F7E9BFF1F1EB1614D2B68002BA5
:1016D0007BD1604B188865E70026B1469CE6002E5A
:1016E0003FF4E6AEDFF868A1DAF800202EE0002E25
:1016F0003FF4DEAEB7F80080F045D4BFC1EB08027E
:10170000C1EB0E02C1EB0808B8F17E0FDFF840A173
:10171000D5BFC2EB8212C2EBC212520008F101081F
:1017200092FBF8F8DAF8002008F10108424506D0EB
:101730005FFA88F10120009306F0A2FE009B188852
:10174000CAF8008002287FF4DFAE42462168B5F86F
:1017500000803888414559DA0021C8EB0008B8F10B
:101760007E0FD3BFC1EB8111C1EBC11108F101089C
:10177000490091FBF8F808F10108904506D05FFA9E
:1017800088F10420009306F07BFE009B1888CAF8BD
:101790000080B9E69342D4BFC4EB0303C4EB020359
:1017A00094E6032827D12C4B1B88092B91D0002EBF
:1017B0008FD0274D2B68002B8BD04A20214606F076
:1017C0005FFE244B2C601888ECE6214606F058FE9C
:1017D000204B2C601888E5E640207F218DE80C0026
:1017E00006F04EFE019B009A188858451CD002282E
:1017F0007FF48AAE76E704287FF46BAF002E3FF4C7
:1018000068AF2146402006F03BFE62E78142D4BF2C
:10181000C8EB0101C8EB00019FE79342D4BFC6EBC0
:101820000303C6EB02037EE6B8F80010DAF800E026
:10183000B7F800808E45FFF665AF5DE72988B7F8F9
:1018400000E020680026C1EB0E03B146E9E500BFC9
:101850001C9CFF1FA29DFF1F4A9DFF1F08B50F4B39
:101860001B88022B0FD0032B12D0042B03D00C4B60
:1018700001221A7008BD7F21092006F001FE084BE5
:1018800001221A7008BD7F21412006F0F9FDEEE724
:101890004021092006F0F4FDE9E700BF149CFF1F7A
:1018A000D49BFF1F38B51C4B1B881D2B26D01B4B10
:1018B0001B88012B25D01A4A1A4B14881B681A4A18
:1018C000A342128818DB9342D4BFC4EB0303C4EBDA
:1018D0000203141B7F2CC6BFDB010134C3EBC3130F
:1018E00093FBF4F4114D2B689C4203D0E1B2052028
:1018F00006F0C6FD2C6038BD0023EAE70C4B1C88BF
:10190000F0E70C4B0C4A0D491B6812680C689B1AD7
:101910001C1B84F30704E5E7929DFF1F049DFF1F36
:10192000789DFF1F649BFF1F909DFF1F5C9BFF1F07
:10193000B09BFF1FD09DFF1F2889FF1F109DFF1F19
:1019400010B50F4C23685BB90E4B1B88022B11D0CE
:10195000033B012B09D90C4A00231370236010BDEF
:101960000021052006F08CFDEEE70021092006F09D
:1019700087FDF0E70021412006F082FDEBE700BF84
:101980005C9BFF1F149CFF1FD49BFF1F08B5274BB8
:101990001B78ABB115200AF0FFFB254A254B1288B6
:1019A00018601D2A15D0244A1288EAB1012A25D0D0
:1019B000224B1B78002B34D0BDE80840FFF7C0BF96
:1019C00011200BF02DFB1A4A1A4B128818601D2AA1
:1019D000E9D11B4B1B78002BEAD0184B1B780BB3BB
:1019E000BDE80840FFF75EBF164A1288002ADFD024
:1019F000154A1B6812889A42DADCEEE70F200BF0DA
:101A00000FFB104B114A1B88106033B1104B114A69
:101A10001B6812689B1A9842DFDD084B1B78002B6D
:101A2000CAD108BDFFF71AFFDAE700BF709DFF1F9C
:101A3000929DFF1F649BFF1F049DFF1FD49BFF1FF0
:101A4000489DFF1F149CFF1F789DFF1F109DFF1FC7
:101A5000D09DFF1F2889FF1F2DE9F04F8BB007ADE8
:101A6000B54F2C460AAE611BC9B2B44808F0D2FB90
:101A70003B88834294BF0020012004F8010BA6425A
:101A8000F1D1AF48AF4A9DF81C70AF4907709DF87F
:101A90001E00AE4D10709DF820209DF82430AC4EF5
:101AA000AC4C0A709DF82210297000253370257007
:101AB00073B9002940F00581A7491AB10B78002BB2
:101AC00040F0EC81002800F0BF810223237005E084
:101AD000002A40F0A78005239F492370DFF8D0B289
:101AE000DFF8D0829DF81D209DF82100DFF8C89214
:101AF000DFF8C8A2994D9A4F9A4E0B709DF81FC0FF
:101B00009DF823109DF827309DF826E08BF80020E3
:101B100088F800009DF82520297001203A70337064
:101B200089F800C08AF800E00BF07AFA8E4A8F4BF1
:101B300011688842CCBF012200221A7076DD8C4BDE
:101B40001B88182B72D88B4AB2F800E00C3B00932C
:101B5000BEF1000F72D1884A9BF800C092F800B025
:101B600098F8008099F800209AF8009094F800A066
:101B70002C78ABEB4C0BC2EB0B0BA8EB880EDE44C6
:101B8000C9EB897BC9EB8B09DFF8F4B1F14497F815
:101B900000E0BBF800B009EB44093478CE4404FB04
:101BA0000BEE4FF00C09754C19FB0AEEC4F800E07F
:101BB000B8F1000F0BD036784EB1714E3688042E36
:101BC0000CBF0EF1020E0EF1040EC4F800E06D4CD5
:101BD000DFF8EC912488B9F800A06B4EDFF8E491AF
:101BE0003688D9F80090009B033C04EB4404CAEB10
:101BF000CA0A0EEB84043444D144644E0C3C56F8BB
:101C000029601C44A319BCF1000F28D02C7834B3F0
:101C1000002A5AD1B8FA88F85D4C4FEA581884F86F
:101C2000008023E0062323704B4957E7514AB2F85E
:101C300000E000230093BEF1000F8CD0BEF1010F35
:101C400047D0BEF1020F00F0C1804C4C9BF800C0A1
:101C500099F8002098F80080D4F800E0A8E74C4CF0
:101C6000002525700AB13A781ABB0022494C8842F7
:101C700022704949C4BF494AC2F800E00A68934249
:101C800013D0474A474C10680590059820601268A9
:101C90000692454C069A24880B60121AA24284BF11
:101CA000424A13600BB0BDE8F08F3E483C4A0068E2
:101CB000EDE7BCF1000FD8D1B8F1000FD5D101226A
:101CC000D4E704232370244908E7314A0024147020
:101CD000CBE7294A9BF800C092F800E098F8008012
:101CE00099F8002094F800B09AF800902C780194AC
:101CF000AEEB4C0EC2EB0E0EA8EB88047444C9EB9D
:101D0000C909D944A31EDFF878A0DFF8BCE0019C24
:101D100097F800B05EF829E0BAF800A096F80090B5
:101D200003EB44045C4409FB0A4909F11809134C0C
:101D3000CE44C4F800E03BE7B49DFF1F049CFF1FA6
:101D4000B69DFF1FB79DFF1FB89DFF1FB99DFF1FC9
:101D5000BA9DFF1F019DFF1F0A9DFF1FE69DFF1FEC
:101D6000E79DFF1F989DFF1F9489FF1F489DFF1F40
:101D7000929DFF1F609BFF1FA889FF1F509DFF1FA3
:101D8000C29BFF1F649DFF1F7C9BFF1FD40F0100A0
:101D9000CC9DFF1FCD9DFF1FCC9BFF1FAC9BFF1F4A
:101DA000D09EFF1FF09BFF1FA09DFF1FD49DFF1F14
:101DB000E29DFF1FE49DFF1FE39DFF1FE59DFF1FA9
:101DC000889DFF1F189CFF1F54130100374A9BF882
:101DD00000C092F800B0247899F8002098F80080AC
:101DE0000394ABEB4C049AF80090314B95F800A0AB
:101DF000CDF804A0A8EB880BA41A5C444FF0050BA7
:101E00001BFB094B039C97F800A0CDF808A0C9EB79
:101E1000C909B3F800A009EB0403BDF80490029CC3
:101E20000BF1050B1EFB09BE96F800B0DFF8A4907D
:101E3000A6440BFB0AEE59F823901E4C0EF10C0E33
:101E4000CE44C4F800E0B3E65FBB0B78012B2BD97E
:101E5000194A23701288002A3FF440AE174A1288AC
:101E6000013A92B2062A3FF639AE154A1278002A94
:101E70003FF434AE134A1268012A7FF42FAE1248A1
:101E8000124A0068124E82FB0025C217C2EB65029F
:101E900002EB4202A0EB820232801FE60323237092
:101EA0001CE60123237019E63B4617E6A889FF1FAD
:101EB000C29BFF1F509DFF1FE09DFF1F169DFF1F30
:101EC000129CFF1F8C9DFF1FD49DFF1FABAAAA2A47
:101ED000549DFF1F7C1501002DE9F04F3A4B1B78F4
:101EE0008BB0002B6AD10E200AF056F90DF052FC8F
:101EF00001463648364E374DFEF71CFB3348FEF799
:101F0000EFFA0DF061FE80F30C003060FFF7A4FDE6
:101F10002C68012C7AD0022C00F0AB82032C00F04C
:101F2000B9832D4E33682D4A2D4E0993099B316894
:101F300012882C4C591A013A9142236000F2948283
:101F4000294E32689A1A0D2A00F28782274E32688B
:101F50009A1A132A00F27C82254E32689A1A252A90
:101F60001AD9244B1B88002B40F06881224B1B7828
:101F7000002B40F06381FFF7E5F9204B1B881B3BEA
:101F80009BB2022B04D81E4B1B78002B40F05981CA
:101F900003F058FD236833601A4D2A689B1A502BB2
:101FA00000F21282184B1B88012B00F02A8206F0E7
:101FB000FBFA06F029F90BB0BDE8F08F07F054FBEF
:101FC0000BB0BDE8F08F00BF949BFF1F289DFF1F43
:101FD0005C9DFF1F8C9DFF1FD09EFF1F9089FF1FE0
:101FE0000C9CFF1F249DFF1FFC9BFF1FDC9BFF1F02
:101FF000E09BFF1F069DFF1F8E9BFF1F929DFF1FF3
:10200000489DFF1F189DFF1F609DFF1FDFF828934D
:10201000A34AB9F800001378834204D0C3B218462B
:10202000137006F0FDF9DFF80C839E4AB8F8003013
:102030001178994204D09C4F3978002940F0FD86F0
:102040009A4A336812889A4E9A42C0F2FF80994A9F
:102050001278002A40F0FA80DFF8E0A2BAF80030E7
:1020600023B9954B1B88002B00F0FC84934A944BBA
:1020700011881B88934A0B4412685B109342924A62
:10208000126880F29E8400219342B4BF01230B4664
:1020900004910093ACBF4FF0010B8B4605910E20CD
:1020A0000AF07AF8894B8A4A1B6817680393013350
:1020B000A7F25232002B8446029240F3CF86802B47
:1020C000A8BF8023834A844912780191002A00F036
:1020D000C7800978914200F0C380B8F80010DFF89B
:1020E00054E2994201F0A7806F49AEF800307B4B73
:1020F0004FF0010E81F800E01978DFF844E2019B0F
:102100008EF800101A70009B002B00F01B81BAF8AB
:102110000030002B00F01681714B1B685A1C002AFE
:1021200040F3A086802A00F39C866E4C6E496F486F
:102130002488098800682144B0EB610FC1F2EE8267
:10214000A3F148020F2A02D8473BA9F800300E201D
:102150000AF022F86FF454731F44874202DC644B88
:1021600000221A7000200AF05BFF624A624B11687D
:10217000624C1B888842D4BF002201222270002BAF
:1021800000F016845E4B1C78944240D088423EDDBD
:102190005C490C78002C00F017875B4991F800C06F
:1021A000BCF1000F40F00E87584F0097584F594828
:1021B0000297564F007887F800C0554F4FF0010E38
:1021C00087F800C081F800E0002841F0B48052494F
:1021D0000978002900F0D887504903910C46097806
:1021E000002940F0CE874E48494F007839700121D0
:1021F0000297217058B1454843490090002008706B
:102200000099029F0870039901243C7008701A70AD
:10221000444B1B88A3F11B02012A40F2E9851D2BC8
:102220007FF480AE3E4F3B78002B41F04B803E4C1C
:102230002378002B40F08984237073E6FFF724F89D
:1022400099E62B68012B7FF4A3AEA3E63168374AE9
:10225000069106983649106002220B602A60FBE660
:102260001E49DFF8DCE0097800293FF448AF9EF80A
:10227000000081423FF443AF03984B2840F3A2870C
:102280001833802BB8F80000A8BF802398423FF491
:1022900036AF284803800448012303702FE700BFAE
:1022A000FA9CFF1FE49BFF1F829BFF1F109CFF1FD8
:1022B000D09EFF1F8E9BFF1F029CFF1FA29BFF1F34
:1022C0005A9DFF1FBC9BFF1FD89DFF1FAC9BFF1F8C
:1022D000689BFF1FCC9DFF1FC89BFF1FCD9DFF1F4D
:1022E000509DFF1F0C9DFF1F089DFF1FB49BFF1FEC
:1022F000009DFF1F9489FF1F169DFF1FA89BFF1FB6
:10230000549BFF1FE59DFF1F589DFF1FA49DFF1FAE
:10231000129CFF1FE69DFF1FE29DFF1F559BFF1FA5
:10232000489DFF1F929DFF1F7E9BFF1FD89BFF1F95
:10233000209DFF1F949DFF1F149DFF1FD09BFF1F1B
:10234000C99BFF1F029B9C45BFF601AF864B1B88B4
:10235000002B3FF4FCAEBBF1000F7FF4DDAE834BEE
:102360001B881BB1059B002B7FF4D6AE049B002B72
:102370003FF4EDAE7E4B1A78002A7FF4E8AEDFF82A
:10238000649299F8004001221A70002C40F03783C3
:10239000784B1B78002B02F03780774B1B78002B93
:1023A00002F00283754B1B78002B7FF4D0AE744B88
:1023B0001B78002B3FF4CBAEB8F8003071490A3BD4
:1023C000A8F800300A70C2E604F03EFE6E4B1B789F
:1023D00073B96E4B1B785BB96D4B1B7843B96D4B72
:1023E0001B782BB96C4B1B7813B903F001FB01E090
:1023F00003F00AFB23682B60684B1B88012B7FF4DA
:10240000D6AD674A674B116867481A78A1F118037F
:102410002A2101FB03F10160002A00F0B382634C22
:102420002368994200F35C8310DA61480278002A3D
:1024300040F03E875F4A1068D0F17F0048BF03300C
:10244000801001301B1A994242F3428621609BE2C0
:10245000FFF79CFA236833607EE5FEF74DFBFEF73D
:102460009DFF2368336071E5FEF7BEFA2368336091
:1024700066E5514A34681188A14204DB464B1B785B
:10248000002B00F05D834D4E4D48336807934D4B54
:10249000079A00681B88121A9A4200F2A980002B42
:1024A00000F0A680484B1A88002A3FF43BAD474B0A
:1024B00047481B680088A342B8BF2346994241F3AE
:1024C0002681444B1960DFF8208188F80020344FC2
:1024D000FEF78AFA38687F2840F370853E4B7F38D4
:1024E00083FB0032C317C3EB620303EB4303A0EB90
:1024F00083007330394B01931B883860002B40F008
:102500008C86234B00931B78002B00F0CD83344C3A
:102510002378002B00F0C883DFF8D090DFF8B8A054
:102520004FF0000B0CE003F17300C0B298F80010FC
:1025300005F0CEFF23780BF1010B5B4540F3B4832C
:102540003B6859F8040F1844A0F17F038AFB03216C
:10255000DA17C2EB610202EB42027F28A3EB82038F
:10256000E1DCFEF779F8E0E7029CFF1F1C9DFF1FEE
:10257000009DFF1FE29DFF1FE39DFF1FE49DFF1FC6
:10258000E59DFF1F829BFF1F129CFF1F589DFF1F91
:10259000A49DFF1F559BFF1F8E9BFF1F609DFF1F6C
:1025A000D49DFF1FD49BFF1FC09DFF1F889BFF1F53
:1025B000A59DFF1F5C9BFF1F109CFF1FD09EFF1F50
:1025C000D89BFF1F009CFF1F809BFF1F209DFF1FAC
:1025D000BC9DFF1F589BFF1FABAAAA2AB89BFF1FD9
:1025E0005489FF1F019DFF1FF69BFF1F2C89FF1FB2
:1025F000554B564A1B681088554AA342B8BF23461C
:10260000994200F38482534C12888342A8BF034648
:102610002360002A7FF457AF9942C8BF134640F3A6
:102620007D82401AB0F5804FAABF9B03C3EB833372
:10263000013093FBF0F0FEF7BDF9C0F3C6100DF0CA
:10264000A9F8454B044618880DF0A4F843490746FD
:1026500020460DF0F3F8014638460DF0EFF821461C
:102660000CF0E4FF4FF07E5104460DF085FA00288F
:1026700041F031803A4920460DF09CFA002840F0A4
:10268000548620460DF0C6FAC0B2DFF8F48088F810
:1026900000001CE7334B34681988A14274DD324BCB
:1026A0001B78002B70D1DFF8DC9099F800007F28B0
:1026B00040F3FA85A3F155337F3803F1004383FBE0
:1026C0000032C317C3EB620303EB4303A0EB8300A9
:1026D0007330264B01931B88C0B289F80000002B91
:1026E00040F0EB87224B00931B78002B00F099847D
:1026F000204C2378002B00F094841F4FDFF87C805F
:102700004FF0000A0AE003F17300C0B205F008FFC1
:1027100023780AF1010A534540F3838457F8043FB4
:1027200099F800001844A0F17F0388FB0321DA1711
:10273000C2EB610202EB42027F28A3EB8203E2DCE0
:10274000FDF78AFFE1E700BF209DFF1FBC9DFF1F33
:10275000809BFF1F589BFF1FCE9DFF1FCDCCCC3D04
:102760000000FE42109CFF1F8E9BFF1FB89BFF1FA7
:10277000A49DFF1F5489FF1F2C89FF1FABAAAA2A03
:10278000F69BFF1F4C9DFF1FB84F38687F2840F312
:10279000CC81B74B7F3883FB0032C317C3EB620396
:1027A00003EB4303A0EB83007330DFF8249399F825
:1027B00000A0824500F01F82AE4B1B88002B43D146
:1027C000AD4AAE4812680088914205DC8242D4BF0F
:1027D000C1EB0203C1EB0003411AB1F5804FA6BF64
:1027E0009B030131C3EB833393FBF1F0FEF7E2F877
:1027F000C0F3C6100CF0CEFFA14B044618880CF0B5
:10280000C9FFA049804620460DF018F80146404611
:102810000DF014F821460CF009FF4FF07E510446EC
:102820000DF0AAF9002840F0C286974920460DF025
:10283000C1F9002840F0768520460DF0EBF9C0B2D2
:10284000DFF8908288F80000BAF17F0F40F3B2837E
:102850008748AAF17F0A80FB0A304FEAEA73C3EB8C
:10286000600000EB4000AAEB80007330874B0093C0
:102870001B78C0B289F80000002B40F01283844B13
:1028800003931B78002B40F0F584824B02931B7856
:10289000002B40F03487804B0193029B1B78FBB1E7
:1028A0007E4B1B88012B00F00086022B00F059871D
:1028B000032B01F0EB80042B01F0EB82052B01F0E0
:1028C0000784062B01F06085072B01F0D185082BCA
:1028D00002F02A80092B02F02F810A2B02F082825B
:1028E000009B1B78002B00F05F84019B6A4C1988C9
:1028F000002900F0B58438687F2840F3CF825C4B14
:102900007F3883FB0032C317C3EB620303EB43033F
:10291000A0EB830073303860002940F06484009B92
:102920001B78002B00F072815D4C2378002B00F0A7
:102930006D81DFF8A4A1DFF89C814FF0000B0CE063
:1029400003F17300C0B298F8001005F0C1FD2378C0
:102950000BF1010B5B4540F359813B685AF8040FBA
:10296000434A1844A0F17F0382FB0321DA17C2EB2C
:10297000610202EB42027F28A3EB8203E0DCFDF759
:102980006BFEDFE7474B1960474B1B68A92202FB30
:1029900003F3002BBCBF03F57F533F339B13543B22
:1029A000194481F30C01282009F07CFFFFF7FFBADE
:1029B000384C3E483549364A237003700B7013700B
:1029C00026E493424FF0000B80F2B2800123CDF851
:1029D00000B0CDF814B00493FFF761BB344B1B7803
:1029E000002B7FF4B4AB039B324A243B83F34703B1
:1029F000D9B25B20136005F043FD99F80040032C29
:102A000030D1DFF8D88098F80030002B42F02181D7
:102A1000294F3B78002B42F00F81254C2378002B67
:102A200042F0FD80254B1B78002B42F0EB80244ABE
:102A30001380244B1B78002B42F017810D4B7F2213
:102A40001A8098F800306BB93B785BB923784BB9A2
:102A50001D4A7F210720138005F012FD7F210B20E6
:102A600005F00EFD194B1F68FFF771BBD49DFF1FCA
:102A7000ABAAAA2A809BFF1F589BFF1FBC9DFF1F6C
:102A8000CE9DFF1FCDCCCC3D0000FE42A49DFF1F7C
:102A9000559BFF1F129CFF1FB89BFF1F169DFF1F1A
:102AA0005489FF1F889BFF1F8C89FF1F589DFF1FA4
:102AB000E59DFF1FB09DFF1FE49DFF1FE39DFF1FCE
:102AC000069CFF1FE69DFF1F4A9DFF1F689BFF1F7F
:102AD0004C9DFF1FF69BFF1F2C89FF1FE29DFF1FD0
:102AE000B04A1078002840F04383AF4A1268D2F110
:102AF0007F0248BF033203EBA202531CAB4A2360A0
:102B00009942B8BF1160FFF63FAF19463CE7A84BAA
:102B100012881960002A7FF4D6AC0B469842D4BFC5
:102B2000C1EB0003C1EB03037BE5FDF795FD3CE63C
:102B30000123CDF810B0CDF800B00593FFF7AFBA80
:102B400001232B609B4EFFF7EDB99B4B6A20198840
:102B500005F01AFE3B782370FFF7E4B9029B1B785F
:102B6000FBB1964B1B88012B00F01884022B00F060
:102B70007686032B01F00080042B01F0AF81052B3A
:102B800001F02A82062B01F01484072B01F0C08586
:102B9000082B01F07D86092B01F0EF870A2B02F04C
:102BA000B281019B1B88002B00F02683009B1B78C1
:102BB0003BB9039B1B7823B9029B1B78002B00F0C9
:102BC00054877F4B1B78002B00F035817D490B78B3
:102BD000082B00F230817C483A6800687B4C013356
:102BE000DBB25F1E101A44F827000B70784B346874
:102BF000198889F800208C426E4E7FF793A93268BD
:102C0000744B0892089A1A60FFF78CB9039B1B78E3
:102C1000002BA3D03B68A3F10C007F2840F327834F
:102C20006D488B3B80FB0320DA17C2EB600000EBA2
:102C30004000A3EB800303F17300DFF8AC81C0B266
:102C400098F8001005F044FC009B1B78002B85D001
:102C50005C4C2378002B81D0DFF890A14FF0000B63
:102C60000CE003F17300C0B298F8001005F030FCDE
:102C700023780BF1010B5B457FF770AF3B685AF887
:102C8000040F554A1844A0F18B0382FB0321DA1785
:102C9000C2EB61020C3802EB42027F28A3EB8203F5
:102CA000DFDCFDF7D9FCDEE7454B1B78002B40F05D
:102CB000A9823B68494A1278002A45D0A3F10C004A
:102CC0007F2840F3EE82444A8B3B82FB0321DA17D4
:102CD000C2EB610202EB4202A3EB820303F1730039
:102CE000C0B298F8001005F0F3FB009B1B7853B3BB
:102CF000344C23783BB3DFF8F490DFF8DCA04FF0DE
:102D0000000B0BE003F17300C0B298F8001005F05F
:102D1000DFFB23780BF1010B5B4514DD3B6859F8B1
:102D2000040F1844A0F18B038AFB0321DA17C2EBCE
:102D300061020C3802EB42027F28A3EB8203E1DC44
:102D4000FDF78AFCE0E73B68254A1278FAB11B4A96
:102D50001288012A00F02E84022A00F00186032A3C
:102D600000F08387042A01F0E080052A01F0188230
:102D7000062A01F02A83072A01F01984082A01F0A3
:102D80005786092A01F09B860A2A02F08880019A58
:102D90001288002A00F04882124903220B702A6030
:102DA000FFF7C0B8A59DFF1F5C9BFF1F889BFF1FFF
:102DB000589BFF1FD09EFF1FB09BFF1F169DFF1F3C
:102DC000589DFF1F5489FF1F849BFF1F3089FF1FE1
:102DD000109CFF1F789EFF1FABAAAA2A559BFF1FBE
:102DE000129CFF1F4C9DFF1FF69BFF1F2C89FF1F8E
:102DF000B04F3B78002B3FF41AAAAF4C207802F07A
:102E000071FEAE4B1B78002B00F0748223887E2B62
:102E100000F27082AA4A0133108899B221800028FA
:102E200000F07882C9B2C0B2A64C05F029FB3B780D
:102E30002370FFF777B83A68D8E6DBB2184613700C
:102E400005F0FCFAA04BA1491A46A14B18460023F5
:102E50000B703B7013700370FFF7F2B80123FFF79C
:102E600031B980249B499C4B9C4A09881B88126875
:102E70000B44B2EB630FBFF66AA98E4B1B78002B95
:102E800040F0DF81B8F80030954AA3423FF45FA9D3
:102E9000944B148001221A70FFF759B9FDF7DCFB3F
:102EA00039E5914B01931B88002B42F00B81884B35
:102EB00003938E4B02938E4C23786BB3DFF84082E2
:102EC000DFF830A24FF0000B09E003F17300C0B24D
:102ED00005F026FB23780BF1010B5B451CDD58F850
:102EE000043F99F800001844A0F17F038AFB0321F6
:102EF000DA17C2EB610202EB42027F28A3EB8203E6
:102F0000E3DCFDF7A9FBE2E7784B029305F008FB51
:102F1000009B1B78002BCED1039B1B78002B3FF42A
:102F2000BCAC99F80030A3F10C007F2840F3B681C7
:102F300070488B3B80FB0320DA17C2EB600000EB8C
:102F40004000A3EB800303F17300C0B205F0E8FA80
:102F5000009B1B78002B00F09681654C2378002B9A
:102F600001F04B82DFF89881DFF888A14FF0000B69
:102F70000AE003F17300C0B205F0D2FA23780BF136
:102F8000010B5B457FF789AC58F8043F99F80000C6
:102F90001844A0F18B038AFB0321DA17C2EB61020C
:102FA0000C3802EB42027F28A3EB8203E1DCFDF741
:102FB00053FBE0E75046FDF74FFB57E4FDF74CFBB2
:102FC000FFF798BA002008704B49087840B13E4995
:102FD00000910978002900F0AB81009F0021397031
:102FE0004649097800297FF4F7A8002C40F0CC80EE
:102FF000002840F0C9802F4C334F94F800E0344C47
:1030000003943A4C0294324C30492070374C00976C
:10301000087038702070BEF1000F7FF4EFA8FFF742
:10302000F6B82B4B1B78002B6CD099F80030A3F12D
:103030000C007F2840F37B832E4A8B3B82FB0321CD
:10304000DA17C2EB610202EB4202A3EB820303F147
:103050007300C0B205F064FA009B1B78002B51D0BE
:10306000234C2378002B4DD0254FDFF888804FF07C
:10307000000A09E003F17300C0B205F051FA2378A9
:103080000AF1010A53453DDD57F8043F99F8000065
:103090001844A0F18B0388FB0321DA17C2EB61020D
:1030A0000C3802EB42027F28A3EB8203E2DCFDF73F
:1030B000D3FAE1E7489DFF1FB09BFF1FE79DFF1F6D
:1030C000EC9BFF1F7E9BFF1FA49DFF1F589DFF1FB2
:1030D000559BFF1F0C9DFF1F089DFF1FB49BFF1FEB
:1030E000949DFF1F829BFF1FB89BFF1F129CFF1F19
:1030F0005489FF1FABAAAA2AE69DFF1FE29DFF1F6E
:103100002C89FF1F924B1B78FBB1924B1B88012B24
:1031100000F03886022B00F03287032B01F0AB80E1
:10312000042B01F05D81052B01F09783062B01F044
:103130003084072B01F0BC85082B01F07B86092B1E
:1031400001F088870A2B01F06587019B1B88002B03
:1031500000F0BC82804B1B78002B40F0B2827F4B8A
:103160007F4A198834680020012310602B6042E5F3
:103170000130C0B2022886BF0021117010701946BC
:1031800002E40398002101707649097800293FF490
:103190003EA86F4902910978002900F0168702982D
:1031A00000210170FFF733B8039B1B78002B7FF4DD
:1031B0009CAB029B1B78002B7FF497AB019B19887B
:1031C000FFF799BB243B002BB8F8000040F347847D
:1031D00098423EF494AF9BB26348A8F800300123B4
:1031E0000370FEF78CBFDFF88481C0B298F800103E
:1031F00005F06EF9FFF793BB5C4B3878197805F052
:1032000067F9D3E47F21402005F03AF95849594A3B
:103210003B680B60002111704CE5C0B298F80010BB
:1032200005F056F9FFF76DB9D8B298F8001005F01F
:103230004FF93B68B0E5504BDFF85CE11978FEF7D9
:103240005EBF4B2C40F34A821834802CB8F8003013
:103250004A4AA8BF8024A3427FF41AAEFEF777BF84
:1032600099F8000005F05CF92188FFF744BBFDF7F1
:10327000F3F9E2E4424B01931B88002B7FF444AE48
:10328000334B02934DE6029B1B78002B7FF408AB77
:10329000039B1B78002B7FF428AB8FE7FDF7DCF94D
:1032A00053E6FDF7D9F91BE5FDF7D6F9FFF711BA9B
:1032B0000132D2B2022A40F23D8200220270194647
:1032C000FFF762BB2F4C207802F00CFC2E4B1B78D2
:1032D0001BB123887E2B41F23B802C4B1B7823B102
:1032E0002388284A002B41F05880294C3B782370D2
:1032F000FEF718BE254B1B78002BF6D02388214AF9
:10330000002BF2D02349013B088899B21180002894
:103310007FF488ADC8B21E4C05F026F93B782370C7
:10332000FEF700BE7F20FFF78BBA7F20FFF7ADB915
:10333000074F094902974FF0000C81F800C0009F29
:1033400002994FF0010E87F800E081F800C047E6CF
:10335000129CFF1F169DFF1F589DFF1F109CFF1FF3
:10336000589BFF1F489DFF1F829BFF1FF69BFF1F5F
:10337000849BFF1F5489FF1FCD9DFF1F949DFF1F3E
:10338000B89BFF1FB09BFF1FE79DFF1FE69DFF1F20
:103390007E9BFF1FEC9BFF1FC99BFF1FDFF8B0A3A5
:1033A0003868BAF80030E54AE54CC31A82FB031EC0
:1033B000D917C1EB6E0101EB4101A3EB810303EBD4
:1033C000430354F8233018447F2840F3C9847F38DE
:1033D00082FB0032C317C3EB620303EB4303A0EB92
:1033E00083007330DFF86C83DFF86CB398F800105B
:1033F000C0B205F06DF8BBF80030022B7FF6D1AB00
:103400003968BAF80030CD4ACB1A82FB030ED817C0
:10341000C0EB6E0000EB4000A3EB800303EB430323
:1034200004EB8303586808447F2840F320877F38E3
:1034300082FB0032C317C3EB620202EB4202A0EB35
:1034400082007330C0B298F8001005F041F8BBF864
:103450000030032B7FF6A5AB3968BAF80030B74AC5
:10346000CB1A82FB030ED817C0EB6E0000EB4000B6
:10347000A3EB800303EB430304EB8304A06808443D
:103480007F2840F36B817F3882FB0032C317C3EB88
:10349000620202EB4202A0EB8200733098F8001047
:1034A000C0B205F015F8FFF77CBBDFF8A4A299F8CD
:1034B0000000BAF80030A14AA14CC31A82FB031ED7
:1034C000D917C1EB6E0101EB4101A3EB810303EBC3
:1034D000430354F8233018447F2840F33D847F3859
:1034E00082FB0032C317C3EB620303EB4303A0EB81
:1034F00083007330DFF860B2C0B205F011F8BBF89A
:103500000030022B7FF6ECA999F80010BAF80030D1
:103510008A4ACB1A82FB030ED817C0EB6E0000EB71
:103520004000A3EB800303EB430304EB83035868E1
:1035300008447F2840F397867F3882FB0032C31708
:10354000C3EB620202EB4202A0EB82007330C0B216
:1035500004F0E6FFBBF80030032B7FF6C1A999F811
:103560000010BAF80030754ACB1A82FB030ED81748
:10357000C0EB6E0000EB4000A3EB800303EB4303C2
:1035800004EB8304A06808447F2840F3CA807F3896
:1035900082FB0032C317C3EB620202EB4202A0EBD4
:1035A00082007330C0B204F0BBFFFFF799B901206D
:1035B000FFF746B9DFF898A16049BAF80020604CDF
:1035C0009A1A81FB020ED017C0EB6E0000EB400090
:1035D000A2EB800202EB420254F8220018447F283A
:1035E00040F3C283A0F17F0381FB0321DA17C2EB12
:1035F000610000EB4000A3EB80007330DFF858B1AE
:1036000098F80010C0B204F063FFBBF80030022B42
:1036100050D93968BAF80030484ACB1A82FB030EF9
:10362000D817C0EB6E0000EB4000A3EB800303EB68
:10363000430304EB8303586808447F2840F37E86E5
:103640007F3882FB0032C317C3EB620202EB4202F7
:10365000A0EB82007330C0B298F8001004F038FF7D
:10366000BBF80030032B25D93868BAF80030334A4C
:10367000C31A82FB031ED917C1EB6E0101EB410196
:10368000A3EB810303EB430304EB8304A368184417
:103690007F2849DD7F3882FB0032C317C3EB62020B
:1036A00002EB4202A0EB82007330C0B298F8001027
:1036B00004F00EFF3B68FFF76ABB04F031FFFFF731
:1036C00011B80021402004F0DBFE48E599F8000025
:1036D00004F026FF3EE50120FEF7D7BF243C002C76
:1036E000B8F8003040F35685A3423EF430ADA4B2A2
:1036F000144BA8F8004001221A70FEF728BD124BA7
:1037000001931B88002B7FF401ACFFF7C6B80F496B
:103710008342A8BF03460B60FEF7D5BE1446FFF7F1
:10372000ACBBFCF799FF3DE7FCF796FFBDE7FCF764
:1037300093FF8EE402701946FFF726B9ABAAAA2AB6
:10374000F0100100829BFF1FB89BFF1F589BFF1FBB
:10375000549DFF1FF69BFF1F929BFF1FFCF77CFFF2
:103760009CE6DFF81CA399F80000BAF80030C24AC2
:10377000C24CC31A82FB031ED917C1EB6E0101EBC9
:103780004101A3EB810303EB430354F823301844B6
:103790007F2840F3C7837F3882FB0032C317C3EB17
:1037A000620303EB4303A0EB83007330DFF8D4B272
:1037B000C0B204F0B5FEBBF80030022B7FF690A833
:1037C00099F80010BAF80030AB4ACB1A82FB030E0E
:1037D000D817C0EB6E0000EB4000A3EB800303EBB7
:1037E000430304EB8303586808447F2840F30186B1
:1037F0007F3882FB0032C317C3EB620303EB430342
:10380000A0EB83007330C0B204F08AFEBBF8003036
:10381000032B7FF665A899F80010BAF80030964A95
:10382000CB1A82FB030ED817C0EB6E0000EB4000F2
:10383000A3EB800303EB430304EB8304A068084479
:103840007F287FF76EAF7F3882FB0032C317C3EB50
:10385000620303EB4303A0EB83007330A2E6DFF8BF
:1038600020A23868BAF80030834A844CC31A82FB1D
:10387000031ED917C1EB6E0101EB4101A3EB8103DC
:1038800003EB430354F8233018447F2840F371833B
:103890007F3882FB0032C317C3EB620303EB4303A1
:1038A000A0EB83007330DFF8E081DFF8D8B198F83F
:1038B0000010C0B204F00CFEBBF80030022B7FF603
:1038C00070A93968BAF800306B4ACB1A82FB030E34
:1038D000D817C0EB6E0000EB4000A3EB800303EBB6
:1038E000430304EB8303586808447F2840F374853E
:1038F0007F3882FB0032C317C3EB620303EB430341
:10390000A0EB83007330C0B298F8001004F0E0FD23
:10391000BBF80030032B7FF644A93868BAF80030B2
:10392000554AC31A82FB031ED917C1EB6E0101EB86
:103930004101A3EB810303EB430304EB8304A3687E
:1039400018447F287FF70AAF7F3882FB0032C31705
:10395000C3EB620303EB4303A0EB830073309DE5ED
:10396000DFF81CA14449BAF80020444C9A1A81FBA4
:10397000020ED017C0EB6E0000EB4000A2EB8002FD
:1039800002EB420254F8220018447F2840F3F482EC
:10399000A0F17F0381FB0321DA17C2EB610000EB8A
:1039A0004000A3EB80007330DFF8D8B098F8001027
:1039B000C0B204F08DFDBBF80030022B7FF67AAE6A
:1039C0003968BAF800302C4ACB1A82FB030ED8179C
:1039D000C0EB6E0000EB4000A3EB800303EB43035E
:1039E00004EB8303586808447F2840F3EA847F3857
:1039F00082FB0032C317C3EB620303EB4303A0EB6C
:103A000083007330C0B298F8001004F061FDBBF879
:103A10000030032B7FF64EAE3868BAF80030164AF5
:103A2000C31A82FB031ED917C1EB6E0101EB4101E2
:103A3000A3EB810303EB430304EB8304A368184463
:103A40007F287FF771AE7F3882FB0032C317C3EB4C
:103A5000620303EB4303A0EB8300733025E60128E8
:103A60003EF44DAB0123FFF7B7BB99F8000004F01B
:103A700057FDFFF7A6B800BFABAAAA2AEC110100B8
:103A8000549DFF1F929BFF1FF69BFF1FDFF8E8A2CC
:103A900099F80000BAF80030B54AB64CC31A82FB58
:103AA000031ED917C1EB6E0101EB4101A3EB8103AA
:103AB00003EB430354F8233018447F2840F3DD819F
:103AC0007F3882FB0032C317C3EB620202EB420273
:103AD000A0EB82007330DFF8A4B2C0B204F020FD86
:103AE000BBF80030022B7EF6FBAE99F80000BAF866
:103AF00000309F4AC31A82FB0321DA17C2EB61022E
:103B000002EB4202A3EB820303EB430304EB8303C8
:103B10005B6818447F2840F327847F380C2290FB91
:103B2000F2F302FB13007330C0B204F0F9FCBBF8EF
:103B30000030032B7EF6D4AE99F80000BAF80030BE
:103B40008B4AC31A82FB0321DA17C2EB610202EB34
:103B50004202A3EB820303EB430304EB8304A36859
:103B600018447F287FF7DDAD7F380C2290FBF2F3FD
:103B700002FB1300733015E5DFF8FCA13868BAF8D2
:103B800000307B4A7B4CC31A82FB031ED917C1EB62
:103B90006E0101EB4101A3EB810303EB430354F8F6
:103BA000233018447F2840F365817F3882FB003240
:103BB000C317C3EB620202EB4202A0EB8200733038
:103BC000DFF8BC81DFF8B4B198F80010C0B204F09F
:103BD0007FFCBBF80030022B7EF6E3AF3868BAF802
:103BE0000030634AC31A82FB0321DA17C2EB610279
:103BF00002EB4202A3EB820303EB430304EB8303D8
:103C00005B6818447F2840F3A0837F380C2290FB28
:103C1000F2F302FB13007330C0B298F8001004F006
:103C200057FCBBF80030032B7EF6BBAF3868BAF800
:103C300000304F4AC31A82FB0321DA17C2EB61023C
:103C400002EB4202A3EB820303EB430304EB830486
:103C5000A36818447F287FF781AD7F380C2290FB42
:103C6000F2F302FB1300733018E4DFF80CA14049B3
:103C7000BAF800203F4C9A1A81FB020ED017C0EB15
:103C80006E0000EB4000A2EB800202EB420254F80F
:103C9000220018447F2840F3F380A0F17F0381FBCA
:103CA0000321DA17C2EB610101EB4101A3EB8100B3
:103CB0007330DFF8C8B098F80010C0B204F008FC08
:103CC000BBF80030022B7FF6F5AC3868BAF800304C
:103CD000274AC31A82FB0321DA17C2EB610202EB07
:103CE0004202A3EB820303EB430304EB83035B6811
:103CF00018447F2840F345837F380C2290FBF2F371
:103D000002FB13007330C0B298F8001004F0E0FB1F
:103D1000BBF80030032B7FF6CDAC3868BAF8003022
:103D2000134AC31A82FB0321DA17C2EB610202EBCA
:103D30004202A3EB820303EB430304EB8304A36877
:103D400018447F287FF7F0AC7F380C2290FBF2F309
:103D500002FB13007330A8E4FCF77EFCFFF7CABB3C
:103D6000FCF77AFCFFF73EBBFCF776FC46E400BFAD
:103D7000ABAAAA2A7C120100549DFF1F929BFF1F31
:103D8000F69BFF1FDFF83CA399F80000BAF800305B
:103D9000C44AC54CC31A82FB0317D917C1EB67018C
:103DA00001EB4101A3EB810303EB430354F8233000
:103DB00018447F286ADD7F3882FB0032C317C3EBCB
:103DC000620202EB4202A0EB82007330DFF8F8B22D
:103DD000C0B204F0A5FBBBF80030022B7FF6B5A9FA
:103DE00099F80000BAF80030AE4AC31A82FB0321EA
:103DF000DA17C2EB610202EB4202A3EB820303EB90
:103E0000430304EB83035B6818447F2840F3B682C6
:103E10007F380C2290FBF2F302FB13007330C0B228
:103E200004F07EFBBBF80030032B7FF68EA999F8D7
:103E30000000BAF800309B4AC31A82FB0321DA174C
:103E4000C2EB610202EB4202A3EB820303EB4303EA
:103E500004EB8304A36818447F2814DD7F380C2208
:103E600090FBF2F302FB13007330C0B204F058FB76
:103E7000FFF76BB9FCF7F0FBA2E6FCF7EDFB2AE6D7
:103E8000FCF7EAFB15E7FCF7E7FBEEE7FCF7E4FBE2
:103E90009CE7DFF830A299F80000BAF80030814AB8
:103EA000824CC31A82FB031ED917C1EB6E0101EBD2
:103EB0004101A3EB810303EB430354F8233018447F
:103EC0007F28DADD7F3882FB0032C317C3EB620341
:103ED00003EB4303A0EB83007330FCE5DFF8E4A1C0
:103EE0003868BAF800306F4A704CC31A82FB031E60
:103EF000D917C1EB6E0101EB4101A3EB810303EB89
:103F0000430354F8233018447F28B3DD7F3882FB05
:103F10000032C317C3EB620303EB4303A0EB830040
:103F200073304DE6FCF798FB40E4DFF898A15D495B
:103F3000BAF800205D4C9A1A81FB020ED017C0EB34
:103F40006E0000EB4000A2EB800202EB420254F84C
:103F5000220018447F2893DDA0F17F0381FB032119
:103F6000DA17C2EB610000EB4000A3EB8000733076
:103F70009FE6FCF771FB96E4FCF76EFB14E5DFF8B7
:103F800044A199F80000BAF80030464A484CC31AD8
:103F900082FB0317D917C1EB670101EB4101A3EBCA
:103FA000810303EB430354F8233018447F287FF741
:103FB0006DAF7F3882FB0032C317C3EB620303EBA4
:103FC0004303A0EB8300733000E73A4800903A487F
:103FD0003A490390FEF712B9DFF8E8A03868BAF85A
:103FE0000030304A364CC31A82FB0321DA17C2EB89
:103FF000610202EB4202A3EB820303EB430354F89A
:10400000233018447F2840F3B6817F380C2290FB80
:10401000F2F302FB13007330DFF8B080DFF8A8B0D2
:1040200098F80010C0B204F053FABBF80030022B2D
:104030001AD93868BAF800300C22C11A91FBF2F391
:1040400002FB131302FB03435B6818447F2840F311
:1040500067847F3890FBF2F302FB13007330C0B229
:1040600098F8001004F034FABBF80030032B7EF609
:1040700098ADBAF8003038680C22C11A91FBF2F3FF
:1040800002FB131302FB0344A36818447F287FF745
:1040900065AB7F3890FBF2F302FB13007330FFF740
:1040A000FDB900BFABAAAA2AF01001005C14010000
:1040B000EC110100A49DFF1F559BFF1F589DFF1F82
:1040C000B4150100549DFF1F929BFF1FF69BFF1F1D
:1040D000DFF894A399F80000BAF80030D84AD94C18
:1040E000C31A82FB0321DA17C2EB610202EB420220
:1040F000A3EB820303EB430354F8233018447F28D7
:1041000040F320817F380C2290FBF2F302FB130076
:104110007330DFF858B3C0B204F002FABBF80030D5
:10412000022B19D999F80000BAF800300C22C11AF4
:1041300091FBF2F302FB131302FB03435B68184489
:104140007F2840F322847F3890FBF2F302FB1300B8
:104150007330C0B204F0E4F9BBF80030032B7EF6F4
:10416000BFABBAF8003099F800000C22C11A91FBDD
:10417000F2F302FB131302FB0344A36818447F28E5
:104180007FF7CFAA7F3890FBF2F302FB1300733066
:10419000FFF708BA012B3DF4DAAF0124FFF7A8BA04
:1041A000DFF8C4A2A649BAF80020A64C9A1A81FBEF
:1041B0000210D117C1EB600101EB4101A2EB8102BA
:1041C00002EB420254F8220018447F2840F3D080CA
:1041D000A0F17F030C2093FBF0F200FB1230733050
:1041E000DFF888B298F80010C0B204F071F9BBF89B
:1041F0000030022B1AD93868BAF800300C22C11AE4
:1042000091FBF2F302FB131302FB03435B681844B8
:104210007F2840F382837F3890FBF2F302FB130088
:104220007330C0B298F8001004F052F9BBF80030B7
:10423000032B7FF63FAABAF8003038680C22C11A67
:1042400091FBF2F302FB131302FB0344A36818442F
:104250007F287FF769AA7F3890FBF2F302FB1300F7
:104260007330FFF722BAFCF7F7F9FFF770B9FCF7E4
:10427000F3F9FFF7E7B8DFF8F0A199F80000BAF812
:1042800000306F4A704CC31A82FB0321DA17C2EB6D
:10429000610202EB4202A3EB820303EB430354F8F7
:1042A000233018447F2846DD7F380C2290FBF2F340
:1042B00002FB13007330DFF8B4B1C0B204F030F980
:1042C000BBF80030022B19D999F80000BAF8003079
:1042D0000C22C11A91FBF2F302FB131302FB0343FE
:1042E0005B6818447F2840F3A7807F3890FBF2F387
:1042F00002FB13007330C0B204F012F9BBF80030B7
:10430000032B7EF622AFBAF8003099F800000C2299
:10431000C11A91FBF2F302FB131302FB0344A368DF
:1043200018447F287FF7AFAD7F3890FBF2F302FB94
:104330001300733099E5FCF78FF9BCE7FCF78CF9B3
:10434000FFF789B9FCF788F9E3E6FCF785F963E440
:1043500001339BB22380D9B205203C4C04F090F885
:104360003B782370FDF7DEBDFCF776F9FFF7DCBB89
:10437000FCF772F934E7FCF76FF94DE6FCF76CF9DE
:104380004DE5FCF769F9BEE4DFF8DCA099F8000020
:10439000BAF800302A4A2E4CA2E6013B9BB2D9B2B1
:1043A00005202A4C138004F06BF83B782370FDF74E
:1043B000B9BDDFF8B4A03868BAF80030204A244C00
:1043C00011E6FCF749F9FFF71DBBDFF89CA01C497B
:1043D000BAF800201E4CE9E6FCF73EF9FFF793BA65
:1043E000DFF884A099F80000BAF80030144A194C9C
:1043F00049E7FCF731F9FFF706BA029B1B78002B5F
:104400007EF44EAAFEF771BA134B1B78002B00F016
:10441000DE82124B1B78002B7DF499AE104B1B787B
:10442000002B3DF494AEB8F800300E490A33A8F8DA
:1044300000300A70FDF78BBEFCF70EF95BE700BF9A
:10444000ABAAAA2AB41501007C1201007E9BFF1FB3
:10445000CC1301005C140100E39DFF1FE49DFF1FCE
:10446000E59DFF1F829BFF1F549DFF1F929BFF1F17
:10447000A14C2388002B40F05483DFF890B29F4971
:104480009F4A098899F80000B2F800E0DFF87882C6
:10449000C1EB000C0C229CFBF2F102FB11C14FF0AE
:1044A000900C0CFB0EFE02FB01E16FF00B0E58F8B6
:1044B000011008440EFB03007F2840F3EC84A0F1B8
:1044C0007F0393FBF2F002FB10307330C0B204F0B4
:1044D00027F8BBF8002023881344022B22DD874AEB
:1044E000874B118899F80000B3F800C0DFF818E294
:1044F000411A0C2291FBF2F302FB1311902303FBF0
:104500000CF302FB013373445B6818447F2840F3CB
:1045100050857F3890FBF2F302FB13007330C0B27A
:1045200003F0FEFFBBF8002023881344032B22DD99
:10453000724A734B118899F80000B3F800C0DFF895
:10454000C8E1411A0C2291FBF2F302FB13119023F4
:1045500003FB0CF302FB013373449B6818447F2870
:1045600040F338857F3890FBF2F302FB1300733081
:10457000C0B203F0D5FFBBF8002023881344042BFE
:104580007EF7AEA95F4B1B88012B7EF4A9A999F891
:104590000020A2F10C007F287FF7C3A88B3A0C20E3
:1045A00092FBF0F300FB13207330FEF7FBBF524C7D
:1045B0002288002A00F018835249DFF850B1098898
:1045C000BBF800000331884227DD4C484C49008885
:1045D000B1F800E0DFF830C1181A0C2190FBF1F9B6
:1045E00001FB19004FF0900909FB0EFE01FB00E0F2
:1045F0006FF00B0E5CF8000003440EFB02307F28C6
:1046000040F311847F3890FBF1F301FB130073300A
:10461000C0B298F8001003F05BFFBBF800202388BD
:104620001344022B23DD354B354A38681B88B2F81A
:1046300000C0DFF8D4E0C31A0C2193FBF1F201FBB8
:104640001232902303FB0CF301FB023373445B68CB
:1046500018447F2840F3A5847F3890FBF1F301FBD9
:1046600013007330C0B298F8001003F031FFBBF8AC
:10467000002023881344032B23DD204B204A386875
:104680001B88B2F800C0DFF880E0C31A0C2193FB4E
:10469000F1F201FB1232902303FB0CF301FB023316
:1046A00073449B6818447F2840F37F847F3890FBD5
:1046B000F1F301FB13007330C0B298F8001003F05F
:1046C00007FFBBF8002023881344042B7EF7F2AFCA
:1046D0000C4B1B88012B7EF4EDAF3A68A2F10C0065
:1046E0007F287FF721A88B3A0C2092FBF0F300FB88
:1046F00013207330FEF7D9BFF89BFF1F549DFF1F97
:10470000029DFF1FD29BFF1F600D0100929BFF1FA8
:10471000B84C2388002B40F06A82DFF810B3B6490A
:10472000B64A0988D7F80080B2F800E0B448C1EB77
:10473000080C0C229CFBF2F102FB11C14FF0900C13
:104740000CFB0EFE02FB01E16FF00B0E40588044A3
:104750000EFB03807F2840F36A83A0F17F0393FB65
:10476000F2F002FB10307330A64BC0B2197803F0A0
:10477000AFFEBBF8002023881344022B23DD9E4AA2
:104780009E4B11883868B3F800C0DFF874E2411A14
:104790000C2291FBF2F302FB1311902303FB0CF3A9
:1047A00002FB013373445B6818447F2840F30B8499
:1047B0007F3890FBF2F302FB13007330914BC0B2D1
:1047C000197803F085FEBBF8002023881344032BDF
:1047D00023DD894A894B11883868B3F800C0DFF8B7
:1047E00020E2411A0C2291FBF2F302FB13119023F9
:1047F00003FB0CF302FB013373449B6818447F28CE
:1048000040F3DE837F3890FBF2F302FB130073303A
:104810007C4BC0B2197803F05BFEBBF80020238804
:104820001344042B7EF7BDA9774B1B88012B7EF424
:10483000B8A93A68A2F10C007F2840F3B2808B3A05
:104840000C2092FBF0F300FB132073306D4BC0B2D1
:10485000197803F03DFEFEF7A4B9DFF89CA199F8A2
:104860000000BAF80030694CC11A0C2291FBF2F337
:1048700002FB131302FB03F3E35818447F287FF76E
:104880005AAD7F3890FBF2F302FB1300733012E550
:104890005F4B1A88182A13D03B681344A3F1180001
:1048A0007F2840F37B830C20973B93FBF0F200FBC7
:1048B000123303F17300534BC0B2197803F008FEB2
:1048C000544B55491A78022A94BF013200221A70BB
:1048D0001A7831F81200182810D10424022A02F1A3
:1048E0000100C2B288BF002231F81200182804D19A
:1048F000013CF3D11A70FEF754B91A703B680344B7
:10490000A3F118007F284CDD0C20973B93FBF0F2BD
:1049100000FB123303F1730098E7FBF79DFE80E480
:10492000FBF79AFEFFF79BBB394B1B88182B12D065
:1049300099F800201344A3F118007F2840F33D8329
:104940000C20973B93FBF0F200FB123303F1730052
:10495000C0B203F0E5FD2F4A2F4B127833F8123026
:10496000182B3DF4BDAF99F800201344A3F11800B3
:104970007F287EF7D6AE0C20973B93FBF0F200FB2E
:10498000123303F17300FEF70DBEFBF765FEFFF770
:10499000E0BBDFF864A099F80000BAF800301F4CC3
:1049A00062E7FBF759FE51E71D4B1B78002B7DF4A6
:1049B000CEAB1C4B1B78002B3DF4C9ABB8F80030D4
:1049C0001949013BA8F800300A70FDF7C0BB144B31
:1049D0001B78002B7EF402A8124B1B78002B3DF4B1
:1049E000B6ABB8F8003010490133A8F800300A70AF
:1049F000FDF7ADBBF89BFF1F549DFF1F029DFF1FDE
:104A0000600D0100F69BFF1FD29BFF1FB415010034
:104A10009E9BFF1FF79BFF1F689DFF1FCC1301008C
:104A2000E49DFF1FE59DFF1F829BFF1F929BFF1FC1
:104A3000944A1288182A12D01344A3F118007F2830
:104A400040F3CC820C20973B93FBF0F200FB123337
:104A500003F17300C0B298F8001003F039FD8A4BDF
:104A60008A491A78022A94BF013200221A701A78F1
:104A700031F81200182811D10424022A02F1010091
:104A8000C2B288BF002231F81200182805D1013CBB
:104A9000F3D11A703B68FEF77AB91A703B68034489
:104AA000A3F118007F287EF73FAE0C20973B93FBC5
:104AB000F0F200FB123303F17300FEF7F6BD744A07
:104AC0001288182A12D01344A3F118007F2840F34B
:104AD0007E820C20973B93FBF0F200FB123303F134
:104AE0007300C0B298F8001003F0F2FC664B6949FD
:104AF0001A78022A94BF013200221A701A7831F80B
:104B000012001828CAD10424022A02F1010294BF1B
:104B1000D2B2002231F812001828BED1013CF3D1E4
:104B2000B7E75D4ADFF884B11288BBF800100332A2
:104B300091427FF7CEACA2E4554B1B88182B12D0C4
:104B400099F800201344A3F118007F2840F3238232
:104B50000C20973B93FBF0F200FB123303F1730040
:104B6000C0B203F0DDFC484A4A4B127833F81230E9
:104B7000182B7FF4F8AEFDF7B3BE454B1A88182A00
:104B800013D03B681344A3F118007F2840F3F2814F
:104B90000C20973B93FBF0F200FB123303F1730000
:104BA0003E4BC0B2197803F093FC374B39491A7861
:104BB000022A94BF013200221A701A7831F81200CA
:104BC00018287FF49BAE0424022A02F1010294BF4C
:104BD000D2B2002231F8120018287FF48EAE013CC8
:104BE000F2D11A70FDF7DDBFDFF8C0B0EDE42A4A5C
:104BF000DFF8B8B01288BBF80010033291427FF79B
:104C0000B8AD8CE5264B01227F2107201A8003F0E6
:104C100037FC7F210B2003F033FCFDF70ABF214B4B
:104C200004227F2107201A8003F02AFC00210B2098
:104C300003F026FCFDF7F6BE1A4B02227F21072067
:104C40001A8003F01DFC7F210B2003F019FCFDF7F7
:104C5000E4BE144B002107201C8003F011FC7F21CF
:104C60000B2003F00DFCFDF7D3BE0F4B00227F217C
:104C700007201A8003F004FC7F210B2003F000FCC6
:104C8000FDF7DFBE9E9BFF1FF79BFF1F689DFF1F69
:104C9000A49BFF1FE89CFF1FD29BFF1FF69BFF1FDB
:104CA000069CFF1F4A9DFF1F809BFF1F929BFF1FBB
:104CB000CC4C2388002B40F06381DFF854B3CA4901
:104CC00099F80000C94A09881788DFF824E3411AD7
:104CD0000C2291FBF2FC02FB1C114FF0900C0CFB20
:104CE00007F702FB01716FF00B075EF8011001443A
:104CF00007FB03107F2840F340817F3890FBF2F3DD
:104D000002FB13007330C0B203F00AFCBBF80020B2
:104D100023881344022B21DDB34BB44A99F80000D9
:104D20001B88B2F800E0B24FC31A0C2193FBF1F2DA
:104D300001FB1232902303FB0EF301FB02333B44D1
:104D40005B6818447F2840F3B1817F3890FBF1F312
:104D500001FB13007330C0B203F0E2FBBBF800208C
:104D600023881344032B21DD9F4BA04A99F80000B0
:104D70001B88B2F800E09E4FC31A0C2193FBF1F29E
:104D800001FB1232902303FB0EF301FB02333B4481
:104D90009B6818447F2840F386817F3890FBF1F3AD
:104DA00001FB13007330C0B203F0BAFBBBF8002064
:104DB00023881344042B7EF7C8A98E4B1B88012B34
:104DC0007EF4C3A999F80020A2F10C007F287FF798
:104DD0005AA88B3A0C2092FBF0F300FB132073309F
:104DE000FFF743B8844B1B88182B12D099F800208A
:104DF0001344A3F118007F2840F35B810C20973BFC
:104E000093FBF0F200FB123303F17300C0B203F026
:104E100087FB7A4A7A4B127833F81230182B7FF4DA
:104E2000A2ADFDF75DBDFBF717FCFFF7F1BBFBF78C
:104E300013FC99E4734B1B88182B12D099F80020AF
:104E40001344A3F118007F2840F339810C20973BCD
:104E500093FBF0F200FB123303F17300C0B203F0D6
:104E60005FFB664A684B127833F81230182B3EF419
:104E70006CA999F800201344A3F118007F287FF74C
:104E800002A80C20973B93FBF0F200FB123303F1D6
:104E90007300FEF7EABFFBF7DFFBFFF717BB564ACD
:104EA0001288182A12D01344A3F118007F2840F367
:104EB00003810C20973B93FBF0F200FB123303F1CC
:104EC0007300C0B298F8001003F002FB4B4B4C4942
:104ED0001A78022A94BF013200221A701A7831F827
:104EE000120018287FF4DAAD0424022A02F101022C
:104EF00094BFD2B2002231F8120018287FF4CDAD51
:104F0000013CF2D1C5E53C4B1A88182A13D03B6806
:104F10001344A3F118007F2840F3C2800C20973B74
:104F200093FBF0F200FB123303F17300374BC0B276
:104F3000197803F0CDFA314B31491A78022A94BF1F
:104F4000013200221A701A7831F8120018287FF402
:104F5000D5AC0424022A02F1010294BFD2B200228D
:104F600031F8120018287FF4C8AC013CF2D11A7055
:104F7000FDF717BEFBF770FB12E6FBF76DFBC2E611
:104F80001C4ADFF88CB01288BBF800100332914243
:104F90007FF7BCAE93E6FBF75FFBE1E5FBF75CFB5D
:104FA00089E4FBF759FBFFF75DBBFBF755FBFFF708
:104FB00083BBFBF751FBFFF7B2BAFBF74DFBC7E42E
:104FC000FBF74AFB24E4FBF747FBFFF7F7BBFBF7D4
:104FD00043FB86E5FBF740FBFFF7CABAFBF73CFB58
:104FE00038E500BFF89BFF1F549DFF1F029DFF1F68
:104FF000600D0100D29BFF1FA69BFF1FF79BFF1FA9
:10500000F09CFF1F9E9BFF1F689DFF1FF69BFF1FCD
:10501000929BFF1F304B1B88182B11D099F8002052
:105020001344A3F118007F2834DD0C20973B93FB39
:10503000F0F200FB123303F17300C0B203F070FA18
:10504000264A274B127833F81230182B7FF411AF11
:10505000FEF77BB8234B1B88182B11D099F8002042
:105060001344A3F118007F2817DD0C20973B93FB16
:10507000F0F200FB123303F17300C0B203F050FAF8
:10508000164A194B127833F81230182B7FF4F1AE10
:10509000FEF75BB8FBF7E0FACFE7FBF7DDFAECE7EA
:1050A000FBF7DAFA42E7FBF7D7FA7CE6FBF7D4FA2C
:1050B00051E6FBF7D1FAA9E6FBF7CEFA01E7FBF7D9
:1050C000CBFACBE6094B0393094B0293FDF71EBFC6
:1050D00023601946FDF758BCA69BFF1FF79BFF1FD7
:1050E000F09CFF1FA49BFF1FE89CFF1F559BFF1F09
:1050F000129CFF1F38B507F0EBF80B4805F022F8BB
:1051000000234FF07E5201210848FBF7AFF9084B0E
:10511000084A0949802400251C7118461D60BDE815
:1051200038400AF097BD00BF049CFF1F289DFF1F59
:10513000A89DFF1F1C89FF1FFD05000043682A2052
:10514000198803F021BB00BF10B504462220636814
:10515000198803F019FBE36824201988BDE8104082
:1051600003F012BB10B504460A206368198803F0E7
:105170000BFBE3680C201988BDE8104003F004BB6A
:1051800010B5044606206368198803F0FDFAE36849
:1051900008201988BDE8104003F0F6BA10B504469F
:1051A00002206368198803F0EFFAE3680420198885
:1051B000BDE8104003F0E8BA70B50E4C84B012257B
:1051C0000422012306460390029320468DE8240022
:1051D0001423102106F0BAF906220923029303963C
:1051E0000195204600921423102106F0AFF904B077
:1051F00070BD00BF149EFF1F2DE9F041224D82B00B
:10520000012602B284B20092284601967823192121
:1052100006F0E2F804F10C0212B28DE844002846D0
:10522000A7197823192104F1020806F0D5F83FB236
:105230000FFA88F819233A46284619460196CDF800
:10524000008006F0C9F878233A4628461946CDF87A
:105250000080019604F10A070B3406F0BDF83FB256
:1052600024B278233A46284619468DE8500006F0C5
:10527000B3F8192300943A4601962846194606F0D9
:10528000ABF802B0BDE8F081149EFF1F2DE9F0419C
:105290001E4682B01446002A6AD0099B4D4A00EB94
:1052A000C305012C6F8929896868A7EB010382FB7C
:1052B00003E21A444FEAE373C3EBA21302887BD0E4
:1052C000042C38D112FA83F3994203DC9F42394609
:1052D000A8BF1946089A0180B6F90030BDF92080B0
:1052E0003D48971D4FF0000E3FB2194642460097C9
:1052F000CDF804E006F070F829896A896B68521AC3
:105300001B885C2AA3EB010359DD03EB4303013245
:10531000C3EB431393FBF2F303F11B0213B201201F
:10532000328019464246019000972B4806F054F807
:105330002A4B00221A702A4B022CB3F9001045D0D8
:10534000082C31D100221A8091422DD0089AB6F94A
:10535000003021480632012412B20092194601940D
:10536000BDF9202006F038F8204602B0BDE8F081F3
:105370001C4D1D4A2B681268CB1A93420F4617D951
:10538000164A338811781448012918BF0124147073
:10539000089A06321BB212B28DE814001946BDF904
:1053A000202006F019F82F60012002B0BDE8F0813E
:1053B000204602B0BDE8F0819BB2D31A84E75C219D
:1053C00001FB03F393FBF2F21B32A7E74A1C12B274
:1053D0001A80B9E7C94216B2149EFF1F8D9EFF1FA7
:1053E000F49DFF1F789EFF1F4025010030B583B05C
:1053F00000230C4605B2009326225B231C210C4897
:1054000005F03AFD294601232622094805F044F813
:10541000002C24B205DB214601232622044805F096
:105420003BF8044A044B15801C8003B030BD00BF1C
:10543000149EFF1FAC89FF1FAE89FF1F70B5944CEF
:10544000237882B01BB1934B4FF6FF721A80924BB8
:10545000B3F90030C3B9914A8E4B1068B3F90020FC
:1054600080F30C005B2303FB00F000131C3082422E
:105470005AD04FF0FF31FFF7B9FF894805F060FDC2
:105480000023237002B070BD012B32D0022B6AD0F2
:10549000032B4FD0042BF3D1272200258DE82400C5
:1054A00076231C217E487F4E05F096FF17E0B0F56D
:1054B000AF7FA8BF4FF4AF70323803FB00F386FB19
:1054C0000321DB17C3EB61111C3109B201231D4419
:1054D0002722734804F0E0FF0C2D00F08180E9B230
:1054E000714804F097FE31284FF05B03DFDC1C218C
:1054F000ECE76E4B1A68B2F52F7F32DB41F25C238A
:105500009342A8BF1346A3F52F735B22684802FBA2
:1055100003F380FB0320DB17C3EBA0201C305D4BA3
:10552000B3F900308342A4D1624BB3F900300133A8
:105530009FD1A5E7604B1B68B3F5FA7F11DBB3F58C
:105540007A6FA8BF4FF47A63A3F5FA725B485B23C6
:1055500003FB02F380FB0320DB17C3EB20201C308E
:10556000DDE71C20DBE7564B1B68B3F5FA7F33DB26
:10557000B3F57A6FA8BF4FF47A63A3F5FA724F4878
:105580005B2303FB02F380FB0320DB17C3EB20202C
:105590001C304C4B1B68B3F5FA7F1FDBB3F57A6FF9
:1055A000A8BF4FF47A63A3F5FA7244495B2303FB67
:1055B00002F381FB0321DB17C3EB21211C31354BA7
:1055C000B3F9003083427FF456AF3A4BB3F9003061
:1055D0008B427FF450AF53E71C20DAE71C21EEE743
:1055E000012007F01DFD6FF495733238364A03FB36
:1055F00000F082FB0023C017C0EB632303F5AF73F9
:10560000312B3ADDB3F5AF7FA8BF4FF4AF735B2208
:10561000323B244D02FB03F385FB0325DB17C3EB71
:1056200065151C35002007F0FBFC6FF495733238CC
:10563000254A03FB00F082FB0023C017C0EB632365
:1056400003F5AF73312B1ADDB3F5AF7FA8BF4FF46D
:10565000AF735B22323B134902FB03F381FB03214F
:10566000DB17C3EB61111C310A4BB3F90030AB42BD
:1056700007D02846FFF7BAFEFFE61C25D2E71C211B
:10568000F2E70C4BB3F900308B42F2D1F5E600BFE4
:10569000EA9DFF1FAC89FF1FF09DFF1F5C9DFF1F50
:1056A000149EFF1F4B48371B049CFF1F649BFF1F6A
:1056B000D3058541AE89FF1FB49BFF1F011FB812A0
:1056C000BC9BFF1FD89DFF1F67BBCF462DE9F04F46
:1056D000DFF8EC82B74CB8F900604D7854F82640FA
:1056E00087B08246039305B10D78DFF8FCB2002A3B
:1056F00034D19BF800308BBBAF4EB6F900000028C8
:1057000000F0CE80012800F02481012032232A46B7
:10571000019000935146A94B2046FFF7B7FD0025A5
:105720000746B6F90030022B40F3F48000233380A3
:10573000B8F90030A24A002BC0F2F880042BC4BF95
:1057400000231380039B002B40F0F680002D0CBF3C
:1057500038464FF0FF3007B0BDE8F08F964EE36853
:105760002268984804930027059237808BF80070D0
:1057700005F0DAFA1120FFF73FFD4FF00109192378
:105780002821CDF804900091242219468D4805F077
:1057900023FE782328212422CDF804900091894803
:1057A000194605F019FE4946864806F0ABF9022273
:1057B0001921844806F0A2F9DDF8149048460BF050
:1057C0001FF8494602467F4806F032FB7D4806F046
:1057D00045FB394614227B4806F090F903227A49AA
:1057E000784806F025FB774806F038FB3946232237
:1057F000744806F083F903227449724806F018FBD6
:10580000704806F02BFB049B002B72D10123704AD9
:1058100018461370FFF7D0FC208963896768191A4E
:105820005C293A885BDC131A5C2202FB03F292FBD0
:10583000F1F31B33674A6348138001271BB21A2216
:1058400019468DE88400142205F0C6FD049BDBB1E7
:10585000218A638AE768581A5C283A886FDD521AF1
:1058600002EB4202C2EB4212431C92FBF3F31B33E6
:10587000524A54481380012738221BB28DE8840015
:105880001946322205F0A8FD534A544BB6F90000E0
:10589000012111704FF6FF721A8000287FF432AF99
:1058A000DFF848914E4AD9F800301268C3EB0A037A
:1058B00093424CD9464B1A78012A18BF0120187020
:1058C0000127FFF779FCC9F800A0012D4ED0042D67
:1058D00059D0022D60D0082D64D0002521E7121A7E
:1058E00002EB4202C2EB42124B1C92FBF3F31B335E
:1058F000A0E72F20FFF780FC39463222314806F01E
:10590000FDF8032237492F4806F092FA2D4806F099
:10591000A5FA7BE77FF40CAFE368002B3FF406AFFA
:10592000B8F90030264A002BBFF608AF04231380D5
:10593000039B002B3FF40AAFFFF780FD06E7511AE7
:105940005C2202FB01F292FBF0F31B3390E7074667
:10595000BBE7002714238DE888002A4651461D4BDB
:105960002046FFF793FC3D460746DAE6B8F80030DC
:105970008BF800500133A8F80030636983B100252B
:1059800020469847CDE6B8F800300122013BA8F840
:1059900000308BF80020F0E7012333800025C7E6B4
:1059A0001D46BEE66369002232804FF0FF35002BB2
:1059B000E6D1BDE6B089FF1FF49DFF1FEE9DFF1FDE
:1059C000F09DFF1F149EFF1F741601007816010042
:1059D0008D9EFF1FEC9DFF1FEA9DFF1FAC89FF1FDF
:1059E000402501007C160100F29DFF1F789EFF1FDD
:1059F00001210D2007F0E6B800210D2007F0E2B8E4
:105A000001460D2007F0DEB808B50D2007F0E0F8DC
:105A1000B0FA80F149090D20BDE8084007F0D2B87E
:105A200010B5002144080D2007F0CCF8204607F0FF
:105A300005F90D20012107F0C5F82046BDE810400A
:105A400007F0FCB8214A224B10881B68984210B519
:105A500035DA204A1288141A9A42A8BF1A46B4F5B9
:105A6000157F22DA121A40F2532303FB02F393FB51
:105A7000F4F105310A2006F015FF174B197801B330
:105A8000164B17491B6840F2271283F3070302FBEA
:105A900003F381FB03211944DB17C3EBA11105318B
:105AA0000920BDE8104006F0FDBE131A4FF4157230
:105AB000611C02FB03F393FBF1F10531DAE70021EE
:105AC000D8E70920BDE8104006F0ECBE109CFF1F8F
:105AD000589BFF1FBC9DFF1FD49BFF1F5C9BFF1F9C
:105AE000090402817F2838B5A8BF7F200F4C4FF4EE
:105AF000167202FB00F284FB02311144D2170546F4
:105B0000C2EBA1110A2006F0CDFE7F3D4FF4967343
:105B100003FB05F384FB03211944DB17A3EBA1115D
:105B20000920BDE8384006F0BDBE00BF090402816F
:105B3000C368B3F9003030B583EAE374A4EBE374CF
:105B4000002BA0B218DB012300E0134603EB830215
:105B500052009442F9DA0A4D90FBF3F285FB03E41C
:105B600003FB1200DB173032D3EBA40380B201F841
:105B7000012BF1D10B7030BD2D230B700131E2E709
:105B80006766666638B5094D8224204602F016FE27
:105B900035F8021B00B28842204601D002F0F4FD25
:105BA0000234A4B28A2CF0D138BD00BFF09CFF1F94
:105BB000024B8020198802F0E7BD00BFA69BFF1FA3
:105BC00038B5094D7824204602F0F8FD35F8021B5F
:105BD00000B28842204601D002F0D6FD0234A4B2C1
:105BE000802CF0D138BD00BFE89CFF1F024B76200F
:105BF000198802F0C9BD00BFA49BFF1F38B5094D2D
:105C00004624204602F0DAFD35F8021B00B2884235
:105C1000204601D002F0B8FD0234A4B24E2CF0D1DF
:105C200038BD00BF689DFF1F024B4420198802F059
:105C3000ABBD00BF9E9BFF1F024B4E20198802F098
:105C4000A3BD00BFB89BFF1F024B9A20198802F02A
:105C50009BBD00BFF89BFF1F024B9820198802F0E4
:105C600093BD00BFD29BFF1F024B8C20198802F00E
:105C70008BBD00BF029DFF1F024B9C20198802F0C4
:105C800083BD00BF929BFF1F024BA020198802F02A
:105C90007BBD00BFE09DFF1F024B9620198802F0DC
:105CA00073BD00BF549DFF1F024B8A20198802F06C
:105CB0006BBD00BF169DFF1F08B5034B1020198850
:105CC00002F062FD012008BD149DFF1F024B102051
:105CD000198802F059BD00BF149DFF1F024B2C20F4
:105CE000198802F051BD00BF909BFF1F024B1E2080
:105CF000198802F049BD00BF8C9BFF1FC3680E20AE
:105D0000198802F041BD00BF024B2820198802F01B
:105D10003BBD00BF649DFF1F024B6220198802F04B
:105D200033BD00BFC29BFF1F024B6420198802F0E5
:105D30002BBD00BF609DFF1F024B5A20198802F047
:105D400023BD00BFA09BFF1F024B1620198802F045
:105D50001BBD00BF809BFF1F024B2E20198802F045
:105D600013BD00BF009CFF1F024B3020198802F0BA
:105D70000BBD00BFCE9DFF1F024B9E20198802F075
:105D800003BD00BF9089FF1F024B1820198802F045
:105D9000FBBC00BF149CFF1F024B1A20198802F0A5
:105DA000F3BC00BFC09BFF1F024B1C20198802F0F0
:105DB000EBBC00BFBA9BFF1F024B6620198802F0A4
:105DC000E3BC00BFA29DFF1F024B7220198802F0A6
:105DD000DBBC00BFC49DFF1F024B2020198802F0CE
:105DE000D3BC00BFA09DFF1F024B3220198802F0D8
:105DF000CBBC00BF929DFF1F024B6820198802F0A8
:105E0000C3BC00BFEC9BFF1F024B6C20198802F043
:105E1000BBBC00BF609BFF1F024B5220198802F0E1
:105E2000B3BC00BF2E89FF1F024B5020198802F01F
:105E3000ABBC00BFA489FF1F024B5420198802F09D
:105E4000A3BC00BFA689FF1F024B5C20198802F08B
:105E50009BBC00BFAA89FF1F024B5E20198802F07D
:105E600093BC00BF2C89FF1F024B6020198802F0F1
:105E70008BBC00BF049DFF1F024B5620198802F007
:105E800083BC00BFF49BFF1F244B1B880B2B43D804
:105E9000DFE803F00B10151A1F24292E33383D06B6
:105EA000084604221E490AF069BD084604221D491D
:105EB0000AF064BD084604221B490AF05FBD08468B
:105EC00004221A490AF05ABD0846042218490AF069
:105ED00055BD0846042217490AF050BD0846042261
:105EE00015490AF04BBD0846042214490AF046BD84
:105EF0000846042212490AF041BD0846042211490D
:105F00000AF03CBD084604220F490AF037BD084696
:105F100004220E490AF032BD704700BF549DFF1F96
:105F2000DC210100C01F0100741E0100902201004D
:105F3000781E0100782201007C1E0100801E0100F5
:105F4000E4200100841E0100E8210100881E0100F8
:105F5000064B074A10B41C88064B0846002C14BF99
:105F600011461946042210BC0AF008BDD09BFF1F41
:105F70008C1E0100901E0100064B074A10B41C88BD
:105F8000064B0846002C14BF11461946042210BCCB
:105F90000AF0F4BC029CFF1F8C1E0100901E010041
:105FA000064B074A10B41C88064B0846002C14BF49
:105FB00011461946042210BC0AF0E0BC069DFF1FE2
:105FC0008C1E0100901E0100064B074A10B41C886D
:105FD000064B0846002C14BF11461946042210BC7B
:105FE0000AF0CCBC1C9DFF1F8C1E0100901E0100FE
:105FF000064B074A10B41C88064B0846002C14BFF9
:1060000011461946042210BC0AF0B8BC569DFF1F69
:106010008C1E0100901E0100064B074A10B41C881C
:10602000064B0846002C14BF11461946042210BC2A
:106030000AF0A4BC069CFF1F8C1E0100901E0100EC
:106040001B4B1B880A2B0AD8DFE803F00A0E121636
:106050001A1E22262A2E0600164B18680860704762
:10606000154B186808607047144B18680860704733
:10607000134B186808607047124B18680860704727
:10608000114B186808607047104B1868086070471B
:106090000F4B1868086070470E4B1868086070470F
:1060A0000D4B1868086070470C4B18680860704703
:1060B000169DFF1FB81E0100901E0100941E0100D6
:1060C000981E01009C1E0100A01E0100A41E0100DC
:1060D000A81E0100AC1E0100B01E0100B41E01008C
:1060E000F0B52B4E2B4FDFF8C4E005460FCE87B03E
:1060F0006C460FC496E803003B68274A274F44F8D4
:10610000040B40F6CC308342C8BF3A46BEF800606C
:106110002180012E11889278ADF80D108DF80F2096
:106120002AD032D340F6CA02022E18BF00229A4269
:1061300026DCA3F698031A491A4AC3EB031381FB22
:1061400003011944DB17C3EB6123243382FB0321D2
:10615000DA17C2EBA10202EB8201A3EB4103303359
:1061600030328DF813308DF81120694628461622FA
:106170000AF004FC07B0F0BD40F698029A42D8DD60
:10618000094B1868CDF81100EFE740F6FC02CEE7A6
:10619000CC1E01007C9DFF1FC01E0100BC1E010023
:1061A0003B773B9867666666C41E0100F89CFF1F3C
:1061B000F8B5174C174E2278174D33782F888E4636
:1061C000003218BF012201467046FFF77FFA002314
:1061D00098423370237015DB14BF012000202B88F8
:1061E0009F420ED040F23A72A3F5AF730B490C4CAC
:1061F00002FB03F381FB0312DB17A3EB62133233C1
:106200002360F8BD0749012218460A702270E6E7AC
:10621000788AFF1F059EFF1FB49DFF1FB5814E1B8F
:106220009489FF1F8C9EFF1F014B187802F044BA1F
:10623000749EFF1F014B187802F058BA2090FF1F80
:10624000134BB3F9003030B583EAE374A4EBE37485
:10625000002BA0B218DB012300E0134603EB8302FE
:1062600052009442F9DA0B4D90FBF3F285FB03E404
:1062700003FB1200DB173032D3EBA40380B201F82A
:10628000012BF1D10B7030BD2D230B700131E2E7F2
:106290002090FF1F67666666144BB3F9003070B537
:1062A00083EAE375A5EBE375002BACB21ADB01239F
:1062B00000E0034603EB830040008542F9DA0C4E10
:1062C00094FBF3F086FB03E503FB1044DB1730304F
:1062D000D3EBA503A4B201F8010BF1D105480B7073
:1062E000106070BD2D230B700131E0E7A09BFF1FF4
:1062F00067666666E41E0100134BB3F9003030B5E3
:1063000083EAE374A4EBE374002BA0B218DB01234F
:1063100000E0134603EB830252009442F9DA0B4D7E
:1063200090FBF3F285FB03E403FB1200DB17303232
:10633000D3EBA40380B201F8012BF1D10B7030BD77
:106340002D230B700131E2E79089FF1F67666666B7
:10635000134BB3F9003030B583EAE374A4EBE37474
:10636000002BA0B218DB012300E0134603EB8302ED
:1063700052009442F9DA0B4D90FBF3F285FB03E4F3
:1063800003FB1200DB173032D3EBA40380B201F819
:10639000012BF1D10B7030BD2D230B700131E2E7E1
:1063A0002E89FF1F67666666134BB3F9003030B560
:1063B00083EAE374A4EBE374002BA0B218DB01239F
:1063C00000E0134603EB830252009442F9DA0B4DCE
:1063D00090FBF3F285FB03E403FB1200DB17303282
:1063E000D3EBA40380B201F8012BF1D10B7030BDC7
:1063F0002D230B700131E2E7A489FF1F67666666F3
:10640000134BB3F9003030B583EAE374A4EBE374C3
:10641000002BA0B218DB012300E0134603EB83023C
:1064200052009442F9DA0B4D90FBF3F285FB03E442
:1064300003FB1200DB173032D3EBA40380B201F868
:10644000012BF1D10B7030BD2D230B700131E2E730
:10645000A689FF1F67666666134BB3F9003030B537
:1064600083EAE374A4EBE374002BA0B218DB0123EE
:1064700000E0134603EB830252009442F9DA0B4D1D
:1064800090FBF3F285FB03E403FB1200DB173032D1
:10649000D3EBA40380B201F8012BF1D10B7030BD16
:1064A0002D230B700131E2E7AA89FF1F676666663C
:1064B000134BB3F9003030B583EAE374A4EBE37413
:1064C000002BA0B218DB012300E0134603EB83028C
:1064D00052009442F9DA0B4D90FBF3F285FB03E492
:1064E00003FB1200DB173032D3EBA40380B201F8B8
:1064F000012BF1D10B7030BD2D230B700131E2E780
:106500002C89FF1F6766666608B5702002F056F991
:10651000044B1988884204D07020BDE8084002F07E
:1065200033B908BDF89CFF1F08B5742002F046F986
:10653000044B1988884204D07420BDE8084002F05A
:1065400023B908BD889DFF1F054B1B880846042200
:1065500013B904490AF012BA03490AF00FBA00BF8E
:10656000B89BFF1FEC1E0100E81E01000E4B1B88AC
:10657000032B17D8DFE803F0110C070208460422AA
:106580000A490AF0FBB90846042209490AF0F6B99B
:106590000846042207490AF0F1B9084604220649D0
:1065A0000AF0ECB9704700BF029DFF1FFC1E0100FE
:1065B000F81E0100F41E0100F01E010010B40A4B89
:1065C0000A4C0A4693E8030083B0238802AC04E92E
:1065D000030004EB8303104653F8081C052203B0A4
:1065E00010BC0AF0CBB900BF04170100609DFF1F6B
:1065F00030B40A4B0A4D0C4693E8070084B02B8850
:1066000004AD05E9070005EB8303204653F80C1C95
:10661000042204B030BC0AF0B1B900BF0C1701006D
:10662000F89CFF1FF0B40C4D0C4F0E460FCD8CB0F4
:1066300001AC0FC40FCD0FC495E807003B8884E878
:1066400007000CAA02EB8303304653F82C1C0422EB
:106650000CB0F0BC0AF092B9181701004A9DFF1F58
:10666000F0B40A4D0A4F0E460FCD86B001AC0FC4F0
:106670002A683B88226006AA02EB8303304653F85F
:10668000141C042206B0F0BC0AF078B944170100CB
:10669000149CFF1FF0B40A4D0A4F0E460FCD86B072
:1066A00001AC0FC42A683B88226006AA02EB830370
:1066B000304653F8141C0C2206B0F0BC0AF05EB948
:1066C00058170100BA9BFF1FF0B40A4D0A4F0E463F
:1066D0000FCD86B001AC0FC42A683B88226006AAA1
:1066E00002EB8303304653F8141C042206B0F0BCBE
:1066F0000AF044B96C170100889DFF1F164B1B88D8
:106700000BB31BB283EAE370A0EBE370002B30B550
:1067100084B21DDB012300E0134603EB8302520029
:106720009042F9DA0D4894FBF3F280FB03E503FB9A
:106730001244DB173032D3EBA503A4B201F8012BCE
:10674000F1D10B7030BD0846042205490AF016B994
:106750002D230B700131DDE7EC9BFF1F676666663A
:10676000001F010030B40A4B0A4D0C4693E80700A5
:1067700084B02B8804AD05E9070005EB83032046B0
:1067800053F80C1C042204B030BC0AF0F7B800BF68
:1067900080170100609BFF1F054B1B881BB9054B31
:1067A0001868086070470846042203490AF0E6B8F2
:1067B000F89BFF1F901E01008C1E0100164B1B88CA
:1067C0000BB31BB230B583EAE374A4EBE374002B84
:1067D000A0B21CDB012300E0134603EB830252004E
:1067E0009442F9DA0D4D90FBF3F285FB03E403FBD1
:1067F0001200DB173032D3EBA40380B201F8012B77
:10680000F1D10B7030BD064B1868086070472D231E
:106810000B700131DEE700BF8C9BFF1F6766666669
:10682000901E0100164B1B880BB31BB230B583EAD8
:10683000E374A4EBE374002BA0B21CDB012300E0A3
:10684000134603EB830252009442F9DA0D4D90FB9C
:10685000F3F285FB03E403FB1200DB173032D3EBCA
:10686000A40380B201F8012BF1D10B7030BD064BAF
:106870001868086070472D230B700131DEE700BFF8
:10688000969DFF1F67666666901E0100164B1B886B
:106890000BB31BB230B583EAE374A4EBE374002BB3
:1068A000A0B21CDB012300E0134603EB830252007D
:1068B0009442F9DA0D4D90FBF3F285FB03E403FB00
:1068C0001200DB173032D3EBA40380B201F8012BA6
:1068D000F1D10B7030BD064B1868086070472D234E
:1068E0000B700131DEE700BF809BFF1F67666666A5
:1068F000041F0100174B1B881BB31BB270B583EA42
:10690000E375A5EBE375002BACB21EDB012300E0C1
:10691000034603EB830040008542F9DA0E4E94FBF8
:10692000F3F086FB03E503FB1044DB173030D3EBB9
:10693000A503A4B201F8010BF1D108480B70106057
:1069400070BD074B1868086070472D230B7001312C
:10695000DCE700BF009CFF1F67666666081F01003A
:10696000901E0100164B1B880BB31BB230B583EA97
:10697000E374A4EBE374002BA0B21CDB012300E062
:10698000134603EB830252009442F9DA0D4D90FB5B
:10699000F3F285FB03E403FB1200DB173032D3EB89
:1069A000A40380B201F8012BF1D10B7030BD064B6E
:1069B0001868086070472D230B700131DEE700BFB7
:1069C000CE9DFF1F67666666901E0100164B1B88F2
:1069D0000BB31BB230B583EAE374A4EBE374002B72
:1069E000A0B21CDB012300E0134603EB830252003C
:1069F0009442F9DA0D4D90FBF3F285FB03E403FBBF
:106A00001200DB173032D3EBA40380B201F8012B64
:106A1000F1D10B7030BD064B1868086070472D230C
:106A20000B700131DEE700BFA29DFF1F676666663F
:106A3000901E0100164B1B880BB31BB230B583EAC6
:106A4000E374A4EBE374002BA0B21CDB012300E091
:106A5000134603EB830252009442F9DA0D4D90FB8A
:106A6000F3F285FB03E403FB1200DB173032D3EBB8
:106A7000A40380B201F8012BF1D10B7030BD064B9D
:106A80001868086070472D230B700131DEE700BFE6
:106A9000C49DFF1F67666666901E0100174B1B882A
:106AA0001BB31BB270B583EAE375A5EBE375002B4E
:106AB000ACB21EDB012300E0034603EB8300400081
:106AC0008542F9DA0E4E94FBF3F086FB03E503FBF7
:106AD0001044DB173030D3EBA503A4B201F8010B4F
:106AE000F1D108480B70106070BD074B1868086042
:106AF00070472D230B700131DCE700BFA09DFF1F05
:106B000067666666081F0100901E0100074B1B8820
:106B1000022B06D0012B0CBF054B064B18680860F2
:106B20007047054B18680860704700BF049DFF1F41
:106B3000101F0100141F01000C1F0100054B1B88D2
:106B40001BB1054B186808607047044B1868086053
:106B5000704700BFF49BFF1F1C1F0100181F01009E
:106B6000184B1A8852B3184A128830B50A80B3F904
:106B70000030002B83EAE374A4EBE374BCBF2D2345
:106B80008B70A0B2ACBF02310331012300E0134689
:106B900003EB830252009442F9DA0C4D90FBF3F2BE
:106BA00085FB03E403FB1200DB173032D3EBA403B5
:106BB00080B201F8012BF1D10B7030BD044B186885
:106BC00008607047C09BFF1F201F01006766666654
:106BD000901E010070B53C4D2B780646002B35D138
:106BE0001C4673780BB9204670BDFAF735FF374A5B
:106BF000374B3848127831781B78007802EB430322
:106C00004A1E03EB80030E2AEDD801A050F822F0B3
:106C1000796C00009B6C0000E76B0000796C000051
:106C2000E76B0000E76B0000E76B0000676C00009B
:106C3000E76B0000E76B0000E76B0000E76B00000C
:106C4000E76B0000E76B0000636C0000AE21224898
:106C500003F01AFE204804F067F800232B7001248B
:106C6000BFE706F0FDFAAF211B4803F00DFE1B4AFB
:106C7000012313702B70B6E783B9194803880429E0
:106C80004FF6FF7103F1FF320CBF01230B46134493
:106C900003F07F03013303800FE073B1013B114A1E
:106CA00032F813304BB10E4E0F481049104A338062
:106CB0000123002606700B701370084A022101237D
:106CC00011702B70204670BD788AFF1FE69DFF1F54
:106CD000E79DFF1F989DFF1F149EFF1F8C9EFF1FA7
:106CE000949DFF1F6C9BFF1FE49BFF1F829BFF1F58
:106CF0008F9EFF1F10B5064B064C1A8820460121B7
:106D000001F030FD21884220BDE8104001F03CBD7B
:106D1000D09BFF1F9C9BFF1F10B5064B064C1A888B
:106D20002046022101F01EFD21884220BDE81040CE
:106D300001F02ABD029CFF1F9C9BFF1F10B5064B54
:106D4000064C1A882046042101F00CFD21884220BF
:106D5000BDE8104001F018BD069DFF1F9C9BFF1F62
:106D600010B5064B064C1A882046062101F0FAFCA5
:106D700021884220BDE8104001F006BD1C9DFF1F88
:106D80009C9BFF1F10B5064B064C1A88204600211D
:106D900001F0E8FC21884220BDE8104001F0F4BC7D
:106DA000569DFF1F9C9BFF1F08B5122001F006FD9A
:106DB000054B1988884206D0122001F0E5FCBDE899
:106DC000084001F0F9BB08BD4A9DFF1F08B55820D7
:106DD00001F0F4FC054B1988884206D0582001F0D8
:106DE000D3FCBDE8084001F0E7BB08BD969DFF1F3E
:106DF00008B5142001F0E2FC054B1988884206D042
:106E0000142001F0C1FCBDE8084001F0D5BB08BD6D
:106E1000069CFF1FF0B480EAE075A5EBE075002842
:106E2000ACB21FDB1DBF2B230B704E1C0E46012383
:106E300000E0134603EB830252009542F9DA0B4F50
:106E400094FBF3F287FB030503FB1244DB1730329C
:106E5000D3EBA503A4B206F8012BF1D13370084699
:106E6000F0BC70472D230B704E1CE0E7676666662A
:106E7000174B18880C2813D0192815D01A2817D0AA
:106E80001B2819D01C281BD01D281DD01E2803D05C
:106E90000C3800B2FFF7BEBF0E4A1068086070479A
:106EA0000D4A1068086070470C4A10680860704707
:106EB0000B4A1068086070470A4A106808607047FB
:106EC000094A106808607047084A106808607047EF
:106ED000929DFF1F401F0100281F01002C1F010071
:106EE000301F0100341F0100381F01003C1F01004A
:106EF000034B1888A0EB8000400000B2FFF78ABF68
:106F0000749EFF1F024BB3F90000FFF783BF00BF61
:106F1000C29BFF1F024B1888033800B2FFF77ABFED
:106F2000649DFF1F024B18880C3800B2FFF772BF38
:106F30007C9BFF1F024B1888183800B2FFF76ABF0E
:106F4000A69BFF1F024B1888183800B2FFF762BFDC
:106F5000A49BFF1F024B1888183800B2FFF75ABFD6
:106F60009E9BFF1FC3681888183800B2FFF752BFF6
:106F7000054B1B881BB9054B18680860704708460D
:106F80000422034909F0FABCE09DFF1F901E010096
:106F90008C1E0100054B1B881BB9054B1868086047
:106FA000704708460422034909F0E8BCD29BFF1F42
:106FB000901E01008C1E010030B5134C85B00125D8
:106FC0002B463C2202212046009503F0D3FC2046AC
:106FD00003F0AAFE00224021802320460191009365
:106FE00011460A4B029504F04DFB204603F0A8FF22
:106FF00007480849084A0023036083800B608B80A0
:107000001360938005B030BD149EFF1FCC170100A4
:10701000F89DFF1F0C9EFF1F7C9EFF1F10B500EB0D
:10702000C00000F10F02D2B293B284B09C1E981C33
:107030003D2303918DE819003921024804F086FAB6
:1070400004B010BD149EFF1F014B01221A7070473F
:10705000059EFF1FF0B5694B694C6A4F6A4E6B4D38
:1070600085B004228DE80C0002932046684B402234
:10707000802103F087FA2046664A6749674C08F08A
:10708000E9FD674A674B9761674FD761674F9F611B
:10709000674FDF61674FB761674FF761674FAF6158
:1070A000674FEF61674FA7616748684FE761684FB7
:1070B00087616849684FC761684F8F61684A694F47
:1070C000CF61694F9761694B694FD761694F9F6184
:1070D000694E6A4FDF616A4F6A4DB7616A4FF76167
:1070E0006A4F6B4CAF616B4FEF616B4F6B48A761A1
:1070F0006B4FE7616B4F6C4987616C4FC7616C4F99
:107100006C4A8F616C4FCF616C4F6D4B97616D4FC7
:10711000D7616D4F6D4E9F616D4FDF616D4FB761F0
:107120006D4D6E4FF7616E4FAF616E4C6E4FEF61FC
:107130006E4FA7616E486F4FE7616F4F87616F4970
:107140006F4FC7616F4F8F616F4A704FCF61704F44
:107150009761704B704FD761704F9F61704E714F48
:10716000DF61714FB761714D714FF761714FAF6161
:10717000714C724FEF61724FA7617248724FE761B5
:10718000724F73498761734FC761734F734A8F6141
:10719000734FCF61734F744B9761744FD761744FC6
:1071A000744E9F61744FDF61744F754DB761754FB9
:1071B000F761754F754CAF61754F76487649EF6151
:1071C000764F774DA761DFF808E2E561754F764DA0
:1071D000764C774A774B8761C5618C61764E774FE5
:1071E000774D784CC1F81CE0774878499761D561B4
:1071F0009C61D861B16005B0F0BD00BF40420F0096
:10720000149EFF1F256F0000F08DFF1FE08BFF1FF6
:107210003C90FF1F1C89FF1FDDA50000A48EFF1FEF
:10722000E889FF1F808EFF1FFD5C0000156F0000C6
:10723000095D0000515F0000F56C0000795F0000FF
:10724000196D0000A15F00000C8AFF1F3D6D00005A
:10725000056F0000708CFF1F195D0000C95F000002
:10726000008DFF1F616D0000BD6500004C8CFF1F8D
:10727000295D0000F15F0000DC8CFF1F856D0000C0
:10728000F16E0000B88CFF1F29620000416200000F
:107290005C8EFF1F35620000F1650000748BFF1FDC
:1072A0000965000025660000108FFF1FA96D000012
:1072B00025680000288CFF1FCD6D0000996200003A
:1072C000308BFF1F395D0000196000007C8FFF1FAD
:1072D000F16D00008D680000048CFF1F495D000007
:1072E000F5680000248DFF1F595D000065690000EE
:1072F000BC8BFF1F695D0000F9620000A08AFF1FC0
:10730000795D000061660000948CFF1F895D0000BC
:10731000616B0000388EFF1F995D000095660000CC
:10732000FC8FFF1FA95D0000CD690000CC8DFF1F01
:10733000B95D0000356A0000C48AFF1FC95D000006
:10734000C9660000348FFF1F296500009D6A000098
:10735000148EFF1FD95D0000716E0000E88AFF1FC8
:10736000E95D0000FD6600007C8AFF1FF95D0000FA
:1073700065670000CC8FFF1F095E000051630000AD
:10738000988BFF1F195E0000A9630000548AFF1F3D
:10739000295E00000C8BFF1FC88EFF1F01640000D8
:1073A000395E000059640000495E0000B1640000CD
:1073B000308AFF1FC489FF1FF08FFF1F0D6B000075
:1073C000695E00003D6B0000795E000059790000A5
:1073D000595E0000F0B5461C83B00D46012703231B
:1073E00036B22AB2044631468DE888002448ADB250
:1073F00004F042F80C23AA1C12B200930197052353
:1074000021B21F4804F038F81E4A1F4B12881B682F
:10741000BA422AD023D3022A10D11C4CA3F6CA03A5
:1074200084FB03241C44DB17C3EB24140A2CA8BFE1
:107430000A2424EAE474A2B223B202E000231A462A
:107440001C460D35AA1A01200093019012B2314654
:1074500003230B4803F08EFF204603B0F0BD0C4C15
:10746000A3F6FC0384FB0324DDE7084CA3F6980392
:1074700084FB03241C44DB17C3EBE404D6E700BF02
:10748000149EFF1FF89CFF1F7C9DFF1F8988888822
:107490001F85EB512DE9F0438FB283B0DFF84C80AC
:1074A000BD1D461D2DB204B236B24FF001090AB21D
:1074B0002346314640460095CDF8049003F08CFFFA
:1074C0002A463346214640468DE8200203F084FFD9
:1074D00007F10C020095334612B22146CDF8049014
:1074E000404603F079FF03B0BDE8F083149EFF1F10
:1074F0002DE9F043804685B0002956D1012130485E
:1075000004F000FB2F4998F8062098F8083011F88D
:107510000290994522DA4FEA89064D460C24D8F8A4
:107520000C3027489B595F6822B2002104F0E6FA2C
:10753000384609F065F939460246214804F078FCDE
:107540001F4804F08BFC98F8083001350934AB4231
:10755000A4B206F1040601DD422CE0D1B9F1000F1E
:1075600013D109F1060999450CDA3C2301213B228C
:10757000039102930093019239233F223A2110484C
:1075800003F0E4FF05B0BDE8F0830F2301213B22A7
:10759000039102930093019239230C223A21084867
:1075A00003F0D4FF98F80830DBE700213423009380
:1075B00001913F230C22024803F0DCFE9EE700BF4E
:1075C000149EFF1F0C9EFF1F10B5104C012120467A
:1075D00004F09EFA2046012104F094FA2046342259
:1075E000552104F08BFA20460222094904F020FCC0
:1075F00020460522074904F01BFC204604F02EFC1F
:107600002046BDE8104003F09BBC00BF149EFF1F46
:10761000441F0100481F010070B50D46064609F0E1
:10762000EFF800EB40008400002D36D0284609F02A
:10763000E7F800EB4000400023185B1003F1600105
:10764000091A282209B21748C3F1600404F056FA57
:107650000121144804F056FA284609F0D1F82946C9
:107660000246104804F0E4FB0E4804F0F7FB022148
:107670000C4804F047FA21B221220A4804F03EFAED
:10768000304609F0BDF831460246064804F0D0FB0A
:107690000448BDE8704004F0E1BB6410C4F160042C
:1076A000E5E700BF149EFF1F184B70B5B3F900301B
:1076B00083EAE374A4EBE374002B82B0A1B21EDB77
:1076C00068466D46012300E0134603EB8302520037
:1076D0009442F9DA0E4E91FBF3F286FB03E403FBCE
:1076E0001211DB173032D3EBA40389B205F8012B5A
:1076F000F1D119462B70FFF78FFF02B070BD2D231B
:107700008DF800300DF101056846DBE7149DFF1F81
:107710006766666610B50D4B1B5C51F823402378F5
:1077200084B013B1012004B010BD04AA01A942F82D
:10773000103D2046A3699847A38A9B07F2D401A86D
:107740000099FFF769FF012004B010BDF89DFF1FED
:107750002DE9F04F2F4DDFF8CCB0DFF8C4A0DFF8F3
:10776000C8900FCD91B003AC0FC40FCD0FC40FCD97
:107770000FC42B6823600025A8462F462E4600E044
:107780009846BAF8003024495BF823202846112394
:10779000F9F7FAF800EBC00400EB840089FB003431
:1077A0000444C017C0EB6434C4F13C00C6F13C0291
:1077B00007F14101012600B208F1410300901BB21C
:1077C000019612B209B2154803F006FE08EB060353
:1077D00005F211153C2B2646ADB24746D0D13422D6
:1077E0006B210E4804F08AF900210C4804F08AF954
:1077F0000B4B1B8810AA02EB830353F8344C204632
:1078000008F0FEFF02460548214611B0BDE8F04FE2
:1078100004F00EBB8C170100A4110100149EFF1F81
:10782000909BFF1FA00F01000900028010B5424C81
:10783000424882B003F078FA2378C3B906213F4862
:1078400004F060F92378012B37D90A22022B114664
:107850003A486BD004F052F939490322374804F012
:10786000E7FA364802B0BDE8104004F0F7BA354BED
:107870001A7801210523002A35D101910093114680
:107880002E4803F0F9FD304B1A78002A36D0052334
:1078900001220192009300220A21284803F06AFD88
:1078A0002A4B1A78002A35D1012105230191009332
:1078B0001421224803F0E0FDC0E7254C2388092B62
:1078C00032D9632B8CBF0A211F210A221B4804F0E6
:1078D00015F92188194804F011FB184802B0BDE8D9
:1078E000104004F0BBBA00220191009311461348E6
:1078F00003F040FD144B1A78002AC8D1052301215A
:10790000019100930A210D4803F0B6FD0F4B1A7840
:10791000002AC9D0012205230192009300221421DC
:10792000064803F027FD89E73021CEE704F0E6F8AA
:107930000322084992E700BF8F9EFF1F149EFF1F7E
:10794000541F0100E69DFF1FE79DFF1F989DFF1F2D
:10795000949DFF1F501F0100F8B56D4D287840B968
:107960006C4B1B6899425CD36B4A012313702B70DC
:10797000F8BD0C4600266948664F03F0D5F904F6B9
:10798000AC53324665483B6031212E7004F0B6F8A6
:1079900001216248624D04F0BBF831465F4804F0B3
:1079A000B1F805225F495D4804F042FA5B4804F0F3
:1079B00055FA0C221021594804F0A0F80B225A491C
:1079C000564804F035FA05225849544804F030FA74
:1079D000524804F043FA564B50481C68A4F69803EA
:1079E000C3EB031385FB03251D441021DB17202265
:1079F000C3EB652504F082F840F6CC339C4205F1D8
:107A000024054FF022014FF004000BDCFFF7E2FCED
:107A1000484B1C88064674B3012C46D0022C41D03A
:107A20000120F8BDFFF736FD092243493B4804F029
:107A3000FFF92A221021394804F060F83F4C3748FA
:107A400084FB0534EB17C3EBA404214604F056FA7B
:107A500001223B49314804F0EBF904EB8401A5EB2A
:107A600041012E4804F04AFA012236492B4804F01D
:107A7000DFF90120F8BD34491022284804F0D8F974
:107A8000264804F0EBF92A221021244804F036F8A5
:107A90003146224804F032FA07222C491F4804F0EC
:107AA000C7F9CBE70C222A49E7E70C2229491B48F2
:107AB00004F0BEF9194804F0D1F92A221021174820
:107AC00004F01CF8314615481C4E04F017FA072242
:107AD0001E49124804F0ACF986FB0536EB17C3EBE0
:107AE000A60631460D4804F009FA224614490B480F
:107AF00004F09EF906EB8601A5EB4101074804F06E
:107B0000FDF922460F49054804F092F92046F8BDD8
:107B1000788AFF1F909EFF1F8C9EFF1F149EFF1FE1
:107B20003B773B98581F0100601F0100481F010070
:107B30007C9DFF1FF89CFF1F6C1F01006766666637
:107B4000D026010048260100781F01008C1F01008B
:107B5000A41F0100941F01002DE9F041754C22780B
:107B6000002A05460F4614BF4FF001084FF00008E9
:107B70004ED1714E3368CB1AB3F5FA6F04D86B78D7
:107B8000A3B94046BDE8F0816C4B6D486D49DFF804
:107B9000D0E11A70012303700988237026208EF823
:107BA000002000F0F1FD6B78002BEAD03760F9F788
:107BB00053FF654A654B6649127828781B78097827
:107BC00002EB4303421E03EB81030E2AD9D801A125
:107BD00051F822F0C57C0000917C0000837B0000FE
:107BE000C57C0000837B0000837B0000837B00005A
:107BF000797C0000837B00002B7C0000837B0000ED
:107C0000837B0000837B0000837B0000277C0000D7
:107C1000AF215048484E02F037FEFFF707FE002321
:107C200037602370ABE705F01BFB4A4803F07CF894
:107C30000221484803F066FF0F222321454803F044
:107C40005DFF05224449434804F0F2F8414804F03E
:107C500005F91E2223213F4803F050FF05223F492A
:107C60003C4804F0E5F83B4804F0F8F8394803F0E4
:107C700067F900F0ADFC84E7394D2B78012B50D922
:107C8000304B2620198800F07FFD00232B7078E709
:107C9000002B3FF476AF013B324A32F81330002B11
:107CA0003FF46FAF274C304825492D4A23804FF0D1
:107CB00001080023037081F8008082F80080FFF73C
:107CC000B5FD5EE793B1013B264A32F8131019B3B4
:107CD0001C4B254D1A4C224A1980002601232620D0
:107CE0002E702370137000F04FFD15E0154C1E49E7
:107CF00022880B7004284FF6FF7002F1FF310CBF91
:107D0000012202460A440E4E154D02F07F02013256
:107D10000121228031702B70FFF788FD4FF00108A0
:107D20002FE70649064A01230020087013702370CC
:107D3000A6E700BF788AFF1F889EFF1F8C9EFF1F4B
:107D4000829BFF1F949DFF1FE69DFF1FE79DFF1F66
:107D5000989DFF1F149EFF1FB41F0100BC1F010050
:107D60008F9EFF1F6C9BFF1FE49BFF1F2DE9F04FB1
:107D700005468BB00F46AD480121164603F0C8FEFC
:107D8000AA8812F0010440F0B080DFF8CC8298F8A5
:107D90000030002B7DD1AB79A54AD15CA1B9DFF8C9
:107DA000BCA279781AF8039041B3397801390729D0
:107DB00000F2B780DFE811F0F1005401B5006C016A
:107DC000B500B500B500E9007C78002C00F0CA8051
:107DD0000139EC68387854F82170FC68411EB4F819
:107DE0000080072900F2A780DFE811F07401590133
:107DF000A5006C01A500A500A5009F00DFF854A216
:107E0000DAF80020B21AB2F5967F75D9894A10784F
:107E100001281ABF012010701170874A18BF01464F
:107E2000D05CC0EB0900C0B2FFF7F8F80124CAF833
:107E30000060AB889B0770D57B78002B6DD0F9F77D
:107E40000BFE7E4B7E4A7F481B781278397800788B
:107E5000022515FB02330A2903EB800300F04E8153
:107E60000C295AD1002B58D003F11900764E774ACD
:107E7000013B0021400080B226F813100123157049
:107E800088F8003000F080FC714B032220461A7005
:107E90002FE0664802F048FF0121644803F032FEFB
:107EA00062482246214603F029FEAB88580725D4B4
:107EB0002C68204608F0A4FC214602465B4803F0EB
:107EC000B7FF5A4803F0CAFF092201238DE80C00CE
:107ED00000217F23554803F07FFA00212846FFF751
:107EE00007FB002388F8003055E7AB683146384679
:107EF00098470BB0BDE8F08F0846FAE72B6804A856
:107F0000984704A808F07CFC04A90246474803F0FF
:107F10008FFF464803F0A2FFD6E720460BB0BDE82E
:107F2000F08F00240AF8039083E70021D1543846EB
:107F3000FB699847FC68A4F80080002725223C23B1
:107F40008DE8840041211822384803F013FAE968CB
:107F5000A879FFF7DFFB374A3E4B17701E600BB066
:107F6000BDE8F08F3B490A68B21AB2F5967FD4D9C2
:107F7000304F0E603E78012E00F0B480E96818465C
:107F800001233B70FFF7C6FBB3E7304AE979117074
:107F9000012288F800200024C4E72A7A013A4A45E1
:107FA000BFDD09F10104E4B2A145BAD0224E16F8B2
:107FB00003B0CBEB0900C0B20021FFF72FF82B7AFA
:107FC000052BD9461BD9CBEB0402042A40F3AE8023
:107FD000A4F1040BBBF1000FC0F2B080063B5B457F
:107FE000A8BF5B465FFA83F9AA791348B15C99424E
:107FF00005D000F8029001212846FFF779FAC9EB75
:108000000400C0B201210B4EFFF708F80021342311
:10801000019100930548317040230B223F21A14676
:1080200003F0A8F90124AB797CE700BF149EFF1F81
:108030007C9EFF1F8D9EFF1F0C9EFF1FE69DFF1F56
:10804000E79DFF1F989DFF1F6C9BFF1F8C9EFF1FCE
:108050008F9EFF1F789EFF1F788AFF1FF89DFF1FCE
:108060000FFA89F1E868604C50F8216021680491AA
:1080700034785E4904980860002C71D0012C7FF49C
:1080800050AF5B4A317A88F800401170002449E70C
:10809000B9F1000F50D009F1FF34E4B284E7B98A96
:1080A00001F0040189B200293FF440AF3B6A03921A
:1080B0009847039A00283FF43DAFAB79FC68002154
:1080C000D15438E77B8A43453CD908F101081FFAAF
:1080D00088F830E73B8A43453BD208F1FF381FFA66
:1080E00088F828E725238DE8180042483C703C2397
:1080F0001822412103F03EF93046FAE6002B3FF406
:108100000CAF3D4A3D4E1188394A03F11900013B3D
:10811000400080B226F81310012388F80030157053
:1081200000F032FB364B20461D70E2E6002A3FF796
:1081300055AF04F1FF3B4DE74C46F3E64FF0000925
:108140004B4651E7BB8ADA077FF5F5AEB7F81080EA
:10815000F1E6BB8AD9077FF5EEAEB7F81280EAE602
:108160002849C85CC0EB090009F1010EC0B2012129
:108170004FF0340B02F803E0FEF750FFB6681D48DD
:10818000019440230B223F210124CDF800B003F0DD
:10819000F1F840230B223F211648CDF800B001949E
:1081A00003F06AF92146134803F0ACFC304608F0AE
:1081B00027FBA0EB800000F15F0109B20F220D4800
:1081C00003F09CFC304608F01BFB31460246094890
:1081D00003F02EFE074803F041FEE968A879FFF797
:1081E00099FAAB799EE600BFD09EFF1F789EFF1FD5
:1081F0008C9EFF1F149EFF1F949DFF1F6C9BFF1FF3
:108200008F9EFF1F0C9EFF1F2DE9F047DFF808929D
:108210006D4B99F800601B68DFF800A282B0003651
:1082200001934FF0030018BF0126019F9AF80080C8
:1082300004F0CEFC0546042004F0CAFC04460520E8
:1082400004F0C6FC800040EA4404062004F0C0FCB0
:108250002C4364B25D4944EAC0000A7880F00F0301
:10826000DBB29A425A4A3CD01760002259480B7040
:1082700003788DF800808DF8012053B3564A1268B8
:108280004EF66021BA1A8A4219D8022B59D0012B16
:108290005FD0062B48D0032B63D0042B69D0052B6D
:1082A00077D0072B7DD0082B00F08380092B68D076
:1082B00016B14A4802F044FE02B0BDE8F087484AD1
:1082C000484C00230121237003701360938089F8C8
:1082D00000103A4669464448FFF748FD3043C6B2AD
:1082E000E6E71268BA1A1E2A6BD99AF80020934260
:1082F00022D0394C3D488AF80030012B276082EAB1
:10830000030207609846B1D0042BAFD1374800680C
:10831000381AB0F5C87FA9D9354C2068381A3228E8
:10832000A4D927601A46A1E73A4669463148FFF7C3
:108330001DFD3043C6B2BBE7012B4FF00002E3D175
:10834000E4E73A4669462C48FFF710FD3043C6B2D1
:10835000AEE73A4669462948FFF708FD3043C6B202
:10836000A6E73A4669462648FFF700FD3043C6B205
:108370009EE73A4669462348FFF7F8FC3043C6B209
:1083800096E73A4669462048FFF7F0FC3043C6B20C
:108390008EE73A4669461D48FFF7E8FC3043C6B20F
:1083A00086E73A4669461A48FFF7E0FC3043C6B212
:1083B0007EE73A4669461748FFF7D8FC3043C6B215
:1083C00076E7002252E700BFD09EFF1F949EFF1F5A
:1083D000009EFF1F8C9EFF1F849EFF1F149EFF1F89
:1083E0007C9EFF1F8E9EFF1FC81D0100989EFF1FD1
:1083F000089EFF1FF81D0100201D0100241C010024
:108400009C2501008C250100141C01007C1C01002E
:10841000041D0100F08FFF1F788AFF1F049EFF1FBD
:1084200028B11028044BA8BF102018607047024BD9
:1084300001201860704700BF9C9EFF1F38B50F4D8C
:108440002B78013B01381B02C4B203F47063200493
:1084500043F4404343F00C0300F4FE00184305F0DE
:108460001FFD2868013860F03F00C0B204F046FDEF
:108470002046BDE8384004F041BD00BF9C9EFF1F70
:1084800070B5124D2B78013B1B0203F47063064656
:1084900043F430430806320400F0FE4043F00B037F
:1084A000034302F4FE0018430C4605F0F9FC28686B
:1084B000013860F04F00C0B204F020FD304604F0F7
:1084C0001DFD2046BDE8704004F018BD9C9EFF1FB6
:1084D00070B5124D2B78013B1B0203F47063064606
:1084E00043F410430806320400F0FE4043F0090351
:1084F000034302F4FE0018430C4605F0D1FC286843
:10850000013860F06F00C0B204F0F8FC304604F0AF
:10851000F5FC2046BDE8704004F0F0BC9C9EFF1FB7
:1085200038B5104D2B78013B1B0203F470630446F1
:1085300043F41043000443F0090300F4FE00184321
:1085400005F0AEFC2868013860F06F00C0B204F09E
:10855000D5FC204604F0D2FC0020BDE8384004F0F1
:10856000CDBC00BF9C9EFF1F38B50E4D2B78013B44
:108570001B0203F47063044643F45043000443F0C9
:108580000D0300F4FE00184305F08AFC286801384A
:1085900060F02F00C0B204F0B1FC2046BDE83840C6
:1085A00004F0ACBC9C9EFF1F08B5002005F042FD06
:1085B0000028FAD108BD00BF08B564210720FFF7E5
:1085C0005FFF7F210B20BDE80840FFF759BF00BFC8
:1085D00010B500217B20FFF753FF0024E0B2FFF726
:1085E0009FFF0134022004F029FB802CF6D110BD3E
:1085F00010B504464FF4406004F030FC04F088FCF1
:108600002CB1102C044BA8BF10241C6010BD024BD1
:1086100001241C6010BD00BF9C9EFF1F10B50446C6
:1086200041F0E00004F06AFC04F07F0004F066FC16
:10863000C4F3C610BDE8104004F060BC38B5134D5B
:108640002B78044641F6FF72A0F50050824203F1F8
:10865000FF33A8BF02461B0202F5005203F4706309
:10866000100443F4604343F00E0300F4FE00520490
:10867000184302F0FE42104305F012FC296801394C
:108680002046C9B2BDE83840FFF7C8BF9C9EFF1F17
:1086900038B504460D46F02004F030FC35B12544D1
:1086A00014F8010B04F02AFCAC42F9D1F720BDE824
:1086B000384004F023BC00BF00B50B4B83B002462A
:1086C000998818680090032AADF8041002D903B005
:1086D0005DF804FB684606218DF80520FFF7D8FFFA
:1086E00003B05DF804FB00BF0826010000B50B4B8A
:1086F000024683B0186899880090131F4C2BADF880
:10870000041002D903B05DF804FB684606218DF819
:108710000520FFF7BDFF03B05DF804FB1026010044
:10872000030203F4FE43C0F3C6101843704700BFB2
:1087300003784078DB0103F47E5300F07F00184398
:10874000704700BF82B002AA114642F8040D002013
:1087500012F8013B03F07F03914243EA0020F7D176
:1087600002B07047003210B403884FF0010404FADD
:1087700001F418BF012202FA01F123EA04020A43BC
:10878000028010BC704700BF70B5CEB20C460546E3
:1087900003F0E6FD864203D03146284603F0FAFD99
:1087A0000135284603F0DCFD240A844205D0214629
:1087B0002846BDE8704003F0EDBD70BD38B50546F4
:1087C00003F0CEFD4FF0000460F30704681C03F0D3
:1087D000C7FD60F30F24A0B238BD00BFF8B5044652
:1087E0000020FFF7EBFF002C00F051814FF4AF6148
:1087F0000220FFF7C9FF04204FF47A61FFF7C4FF9E
:108800000B2004F0E5F9002840F05E864FF49661F5
:108810000620FFF7B9FF4FF4FA610820FFF7B4FF15
:108820004FF4AF610A20FFF7AFFF40F6FC010C20C8
:10883000FFF7AAFF4FF496612220FFF7A5FF4FF440
:1088400016612420FFF7A0FF7D212A20FFF79CFF5F
:108850000C210E20FFF798FF01211020FFF794FF55
:1088600002211220FFF790FF00211420FFF78CFF58
:1088700000211620FFF788FF02211820FFF784FF50
:1088800001211A20FFF780FF02211C20FFF77CFF47
:1088900004211E20FFF778FF14212020FFF774FF2A
:1088A00001212620FFF770FF03212820FFF76CFF2E
:1088B00004212C20FFF768FF14212E20FFF764FF0E
:1088C00000213020FFF760FF0C213220FFF75CFF12
:1088D00000213420FFF758FF00213620FFF754FF16
:1088E00000213820FFF750FF00213A20FFF74CFF0E
:1088F00000213C20FFF748FF00213E20FFF744FF06
:1089000000214020FFF740FF00214220FFF73CFFFD
:108910001F214420FFF738FF13214620FFF734FFC3
:108920000E214820FFF730FF11214A20FFF72CFFCE
:108930000A214C20FFF728FF00214E20FFF724FFDB
:1089400006215020FFF720FF02215220FFF71CFFD5
:108950000C215420FFF718FF00215620FFF714FFC9
:1089600000215820FFF710FF01215A20FFF70CFFCC
:1089700003215C20FFF708FF0A215E20FFF704FFB8
:1089800000216020FFF700FF04216220FFF7FCFEBA
:1089900001216420FFF7F8FE00216620FFF7F4FEB6
:1089A0000B216820FFF7F0FE7F216A20FFF7ECFE25
:1089B00000216C20FFF7E8FE00216E20FFF7E4FEA7
:1089C00000217020FFF7E0FE00217220FFF7DCFE9F
:1089D00000217420FFF7D8FE1F217620FFF7D4FE78
:1089E00013217820FFF7D0FE0E217A20FFF7CCFE6E
:1089F00011217C20FFF7C8FE0A217E20FFF7C4FE6C
:108A00001F218020FFF7C0FE13218220FFF7BCFE4C
:108A10000E218420FFF7B8FE11218620FFF7B4FE57
:108A20000A218820FFF7B0FE00218A20FFF7ACFE64
:108A300001218C20FFF7A8FE00219620FFF7A4FE5D
:108A400000219820FFF7A0FE00219A20FFF79CFE4E
:108A500005219C20FFF798FE06219E20FFF794FE3B
:108A60000021A020FFF790FE27210020FFF78CFEB9
:108A70000220FFF7A3FEB0F5805F034616D34FF444
:108A8000AF610220FFF780FE4FF4AF630EE04FF6B8
:108A9000FF7398423FF4AAAE272840F021850220B8
:108AA000FFF78CFEB0F5805F0346E8D2D24A04207F
:108AB0001380FFF783FEB0F5805F034680F051849A
:108AC000CE4A06201380FFF779FEA0F52F739BB2E4
:108AD000B3F57A6F024606D940F628210620FFF743
:108AE00053FE40F62822C64B08201A80FFF766FE88
:108AF000A0F52F739BB2B3F57A6F024606D940F604
:108B0000E4410820FFF740FE40F6E442BD4B0A2056
:108B10001A80FFF753FEA0F5FA739BB240F6AC51F2
:108B20008B42024606D94FF4AF610A20FFF72CFEB4
:108B30004FF4AF62B44B0C201A80FFF73FFEA0F554
:108B4000FA739BB240F6AC518B42024606D940F60E
:108B5000FC010C20FFF718FE40F6FC02AB4B0E2088
:108B60001A80FFF72BFE1828034600F21584A84A46
:108B700010201380FFF722FE431E9BB20F2B0246EC
:108B800004D901211020FFF7FFFD0122A14B122083
:108B90001A80FFF713FE0A28034600F2F7839E4A65
:108BA00014201380FFF70AFE0128034604D9002190
:108BB0001420FFF7E9FD0023984A16201380FFF7E1
:108BC000FDFD7F28034600F2DB83954A18201380C1
:108BD000FFF7F4FD0428034600F2CC83914A1A20E3
:108BE0001380FFF7EBFD0C28034600F206848E4A43
:108BF0001C201380FFF7E2FD0428034600F2F783F0
:108C00008A4A1E201380FFF7D9FD0928034600F287
:108C1000E883874A20201380FFF7D0FD46280346CB
:108C200000F2D983834A22201380FFF7C7FDA0F505
:108C3000FA739BB240F6AC518B42024606D94FF410
:108C400096612220FFF7A0FD4FF496627A4B242014
:108C50001A80FFF7B3FDA0F5FA739BB240F6AC5152
:108C60008B42024606D94FF416612420FFF78CFD93
:108C70004FF41662714B26201A80FFF79FFD7F2864
:108C8000034600F2A2836E4A28201380FFF796FD68
:108C90000628034600F293836A4A2A201380FFF7CE
:108CA0008DFDA0F132039BB2B3F5967F024604D945
:108CB0007D212A20FFF768FD7D22634B2C201A803E
:108CC000FFF77CFD0C28034600F273835F4A2E20D9
:108CD0001380FFF773FD1E28034600F264835C4A8D
:108CE00030201380FFF76AFD0928034600F2E6836F
:108CF000584A32201380FFF761FD1E28034600F218
:108D0000D783554A34201380FFF758FD7F28034648
:108D100000F2C883514C36202380FFF74FFD7F2897
:108D2000034600F2B98338206380FFF747FD7F28B0
:108D3000034600F2AB833A20A380FFF73FFD7F2874
:108D4000034600F29D833C20E380FFF737FD7F2838
:108D5000034600F28F833E202381FFF72FFD7F28FB
:108D6000034600F2818340206381FFF727FD7F28BF
:108D7000034600F273834220A381FFF71FFD384DA5
:108D800028804420FFF71AFD3028034600F2608354
:108D9000344A46201380FFF711FD3028034600F2C5
:108DA0005183314C48202380FFF708FD30280346CB
:108DB00000F242834A206380FFF700FD302803461B
:108DC00000F234834C20A380FFF7F8FC30280346E0
:108DD00000F226834E20E380FFF7F0FC01280346D3
:108DE00004D900214E20FFF7CFFC00231F4A50205A
:108DF0001380FFF7E3FC3BE0109CFF1FBC9DFF1FAF
:108E0000789DFF1F909DFF1F5A9DFF1FA29BFF1F74
:108E10007C9BFF1F149DFF1F4A9DFF1F069CFF1F89
:108E2000809BFF1F149CFF1FC09BFF1FBA9BFF1F4F
:108E30008C9BFF1FA09DFF1F0C9DFF1F089DFF1F08
:108E4000949DFF1F649DFF1FB49DFF1F909BFF1FFC
:108E5000009CFF1FCE9DFF1F929DFF1F6C9BFF1F5D
:108E60009C9BFF1F9E9BFF1F689DFF1FB89BFF1FC2
:108E7000431E9BB20B2B024604D906215020FFF75C
:108E800083FC0622CD4B52201A80FFF797FC042862
:108E9000034600F2BF82CA4A54201380FFF78EFCBB
:108EA000431E9BB21D2B024604D90C215420FFF710
:108EB0006BFC0C22C34B56201A80FFF77FFC012865
:108EC000034604D900215620FFF75EFC0023BE4A6A
:108ED00058201380FFF772FC7F28034600F294822B
:108EE000BA4A5A201380FFF769FC431E9BB2092B34
:108EF000024604D901215A20FFF746FC0122B44B57
:108F00005C201A80FFF75AFC431E9BB2102B0246CE
:108F100004D903215C20FFF737FC0322AD4B5E2010
:108F20001A80FFF74BFC431E9BB21D2B024604D94F
:108F30000A215E20FFF728FC0A22A74B60201A8036
:108F4000FFF73CFC0228034600F2F981A34A6420A3
:108F50001380FFF733FC0128034604D90121642064
:108F6000FFF712FC01239E4A62201380FFF726FCC4
:108F7000C31E9BB2012B024604D904216220FFF7D5
:108F800003FC0422974B66201A80FFF717FC7F280A
:108F9000034600F2CE81944A68201380FFF70EFC4E
:108FA0007F28034600F2BF81904A6A201380FFF7B2
:108FB00005FC7F28034600F2B0818D4A6C201380A7
:108FC000FFF7FCFB0228034600F2A181894A6E20CC
:108FD0001380FFF7F3FB1928034600F29281864ABB
:108FE00070201380FFF7EAFB0228034600F283811A
:108FF000824A72201380FFF7E1FB0628034600F245
:1090000074817F4A74201380FFF7D8FB042803463D
:1090100000F265817B4A8A201380FFF7CFFB0A2884
:10902000034600F25681784A8C201380FFF7C6FB76
:109030000428034600F24781744A98201380FFF702
:10904000BDFB0128034604D900219820FFF79CFBB3
:1090500000236F4A9A201380FFF7B0FB01280346D4
:1090600004D900219A20FFF78FFB0023694A96203C
:109070001380FFF7A3FB0B28034600F21E81664A0C
:109080009C201380FFF79AFB831E9BB2032B0246A2
:1090900004D905219C20FFF777FB05225F4B762042
:1090A0001A80FFF78BFB3028034600F200815C4AF0
:1090B00078201380FFF782FB3028034600F2F1800E
:1090C000584C7A202380FFF779FB3028034600F2C2
:1090D000E2807C206380FFF771FB3028034600F2BA
:1090E000D4807E20A380FFF769FB3028034600F27E
:1090F000C6808020E380FFF761FB3028034600F242
:10910000B880494A82201380FFF758FB3028034675
:1091100000F2A980454C84202380FFF74FFB3028C4
:10912000034600F29A8086206380FFF747FB3028D1
:10913000034600F210818820A380FFF73FFB302810
:10914000034600F20281A020E380FFF737FB0128ED
:10915000034604D90021A020FFF716FB0023344A60
:109160009E201380FFF72AFBC31E9BB20C2B04D951
:109170009E200621FFF708FB06202B88DFF8D0E0B1
:109180002C4F2D4A2D4D2E4E2E4C2F4903F0010C05
:10919000AEF800C0C3F3400EA7F800E0C3F38007A9
:1091A0001780C3F3C007294A2F70C3F30017C3F316
:1091B0004015C3F38013378025804BE0A489FF1F3F
:1091C0002E89FF1FA689FF1FF49BFF1F969DFF1F7F
:1091D000A09BFF1FAA89FF1F2C89FF1F049DFF1F53
:1091E000609DFF1FC29BFF1FA29DFF1FEC9BFF1FE7
:1091F000B09BFF1F609BFF1FE89DFF1FF89CFF1F98
:10920000C49DFF1F889DFF1F169DFF1F029DFF1F0E
:10921000D29BFF1FF89BFF1F549DFF1F929BFF1FB8
:10922000A49BFF1FE89CFF1FA69BFF1FF09CFF1F36
:10923000E09DFF1FD09BFF1F029CFF1FFB9CFF1F99
:10924000069DFF1F629DFF1F1C9DFF1F9089FF1F32
:10925000569DFF1F0B801080F8BD0E218420FFF764
:1092600093FA0E235FE713218220FFF78DFA132371
:1092700050E71F218020FFF787FA1F2341E70A21CB
:109280007E20FFF781FA0A2333E711217C20FFF7C4
:109290007BFA112325E70E217A20FFF775FA0E23BA
:1092A00017E713217820FFF76FFA132308E71F2130
:1092B0007620FFF769FA1F23F9E600219620FFF7D1
:1092C00063FA0023DBE601218C20FFF75DFA01231E
:1092D000B2E600218A20FFF757FA0023A3E6002117
:1092E0007420FFF751FA002394E600217220FFF763
:1092F0004BFA002385E600217020FFF745FA002392
:1093000076E600216E20FFF73FFA002367E6002192
:109310006C20FFF739FA002358E67F216A20FFF717
:1093200033FA7F2349E60B216820FFF72DFA0B2340
:109330003AE600216620FFF727FA00232BE60021FA
:109340006020FFF721FA002300E60A218820FFF7BA
:109350001BFA0A23F7E611218620FFF715FA1123DD
:10936000E9E64FF47A610420FFF70EFA4FF47A63CE
:10937000FFF7A6BB02211820FFF706FA02232DE40F
:1093800000211620FFF700FA00231EE4022112201C
:10939000FFF7FAF9022302E40C210E20FFF7F4F99B
:1093A0000C23FFF7E4BB14212E20FFF7EDF9142363
:1093B00095E404212C20FFF7E7F9042386E4032138
:1093C0002820FFF7E1F9032366E401212620FFF7B7
:1093D000DBF9012357E414212020FFF7D5F91423EA
:1093E00020E404211E20FFF7CFF9042311E4022119
:1093F0001C20FFF7C9F9022302E401211A20FFF71C
:10940000C3F90123FFF7F3BB00215820FFF7BCF994
:10941000002365E502215220FFF7B6F902233AE561
:109420000A214C20FFF7B0F90A23D3E411214A2086
:10943000FFF7AAF91123C5E40E214820FFF7A4F98C
:109440000E23B7E413214620FFF79EF91323A8E467
:109450001F214420FFF798F91F2399E400214020A1
:10946000FFF792F9002386E400213E20FFF78CF9F4
:10947000002378E400213C20FFF786F900236AE40A
:1094800000213A20FFF780F900235CE40021382016
:10949000FFF77AF900234EE400213620FFF774F934
:1094A000002340E400213420FFF76EF9002331E46B
:1094B0000C213220FFF768F90C2322E40021302030
:1094C000FFF762F9002313E440F628210620FFF796
:1094D0005BF940F6E4410820FFF756F9FFF7A0B921
:1094E00017287FF683A919287FF6F2A91B287FF693
:1094F0000FAA1C283FF424AA1E287FF629AA1F2899
:109500003FF42EAA20283FF447AA21283FF450AA6E
:1095100022283FF455AA23283FF45EAA24283FF4CA
:109520008FAA25283FF494AA26287FF49DAAFFF746
:1095300093BA00BFF8B5B32006F0C6FB204B214A12
:10954000054603CB1368C5F803001A0CA220C5F822
:1095500007102B80AA70FFF7E3F82E46002426F8A8
:109560000B0FA0B2FFF72AF9FFF7DAF80234A22CAA
:1095700026F8020FF5D16C1E05F1AE064FF0FF3054
:1095800014F8013F082758400F4B40F300017A1EA2
:109590000B4012F0FF0783EA5000F5D1B442EFD13F
:1095A000C043FFF7CFF83A46C5F8AF00B3212846CD
:1095B00004F0C4FC2846BDE8F84006F08DBB00BFAF
:1095C0001C260100182601002083B8EDF0B50E4BD3
:1095D0000E4C054693E8070085B024682E88AD78C8
:1095E00001AB83E80700270C184600220B21ADF8D9
:1095F00004408DF80670ADF80C608DF80E5004F044
:109600009DFC05B0F0BD00BF282601001826010012
:10961000F0B5124B124D1E68124F0FCD87B06C463D
:109620000FC495E8030044F8040B38683B79CDF883
:109630000D00320C272021808DF802208DF811308A
:10964000ADF80060FFF76CF80022ADF80B001221B6
:10965000684604F073FC07B0F0BD00BF1826010097
:1096600034260100481F0100002004F0E3BC00BFC5
:1096700002F02EBE70B5124C82B000254023064683
:1096800029462046009301958023202201F072FE96
:1096900020222946204602F031FA2046012102F01C
:1096A00037FA304607F0ACF831460246204602F061
:1096B000BFFB204602B0BDE8704001F041BC00BFD6
:1096C000149EFF1FF0B5B22983B075D90546441E1C
:1096D00000F1AE064FF0FF3014F8012F082750407C
:1096E000404A40F300017B1E0A4013F0FF0782EA64
:1096F0005000F5D1B442EFD1C043FFF723F8014643
:10970000D5F8AF000190019A914202D0B2F17F2FBB
:109710000BD105F10B00FFF70BF8A2280BD0324854
:10972000FFF7A8FF002003B0F0BD3048FFF7A2FF0D
:10973000384603B0F0BD05F10D00FEF7F9FF27280C
:1097400040D1002440F6AC5613E004281AD0062875
:1097500021D008281FD00A2828D00C2822D1A1F512
:10976000FA7292B2B24201D8FFF70EF80234A22C7C
:109770000ED004F10D002844FEF7DAFF022C01465A
:10978000A0B2E2D1B1F5805FEED30234A22CF0D1C9
:10979000012003B0F0BDA1F52F7292B2B2F57A6F3D
:1097A000E4D8E1E7222801D0242811D1A1F5FA72EA
:1097B00092B2B242DAD8D7E70D48FFF75BFF00203C
:1097C00003B0F0BD0B48FFF755FF002003B0F0BD1C
:1097D0002A28C9D1A1F1320292B2B2F5967FC5D83A
:1097E000C2E700BF2083B8ED78260100642601009F
:1097F0004C2601008C26010003290CD970B5461CAB
:1098000082B005460C46304603222A4907F066F826
:1098100010B102B070BD70470B2C05D90522264946
:10982000281D07F05BF840B12448FFF723FF2448C8
:1098300002B0BDE87040FFF7C9BE05F1090103227F
:1098400001A807F09BF801A803221E4907F046F87B
:10985000D8B103221C4901A807F040F808B301A8B9
:1098600003221A4907F03AF8B0B91948FFF702FF86
:10987000A11E89B23046FFF725FF0028C9D0154840
:1098800002B0BDE87040FFF7F5BE1348FFF7F2FEE7
:10989000FFF750FE1148F3E71148FFF7EBFE1148C0
:1098A000C6E71148FFF7E6FE02B0BDE87040FFF7DB
:1098B000AFBE00BF18260100581F0100A4260100FA
:1098C000B8260100BC260100E4260100FC260100A8
:1098D0000027010014270100C0260100D426010042
:1098E000282701003C270100E82601002DE9F0436C
:1098F000174D2B6883B081460F469046F3B1154E45
:1099000034880A1992B218461146328006F05AFD80
:1099100028603A464946204402F06CFDB8F1000F39
:1099200009D031882868FFF767FF286806F0D4F966
:1099300000232B60338003B0BDE8F083054E019314
:109940000846318006F0C0F9019B28601C46E0E71C
:10995000A49EFF1FA09EFF1F10B51F4C4FF4FA706E
:10996000FCF75EF8204601F0DFF9002211462046A0
:1099700002F0C4F82046012102F0CAF82046002176
:1099800002F0C0F80B221549204602F051FA204699
:1099900002F064FA0F221249204602F049FA2046EA
:1099A00002F05CFA0F490722204602F041FA2046F5
:1099B00002F054FA204601F0C3FA0B4B0B4A1A602E
:1099C0004FF4FA70FCF72CF8FFF722FE0848BDE8C8
:1099D0001040FFF74FBE00BF149EFF1F402701003D
:1099E0004C2701005C2701005CA0FF1FED980000E0
:1099F000642701000020704790F8392090F8380063
:109A0000101A704790F8383090F839209A4205D9EA
:109A10005A1C034480F83820187E70474FF0FF30FE
:109A2000704700BF90F8383090F839209A4286BFCE
:109A30001B18187E4FF0FF30704700BF704700BF03
:109A400038B50546B0F85E0090B195F85D30144623
:109A5000C3F1210294420CD805F13B001844224680
:109A600002F0C8FC95F85D30234485F85D3020464F
:109A700038BD012014462871EEE700BFB0F85E3013
:109A80006BB190F85D30202B07D8C218013380F8F5
:109A90005D30012082F83B107047012303710020E4
:109AA000704700BF0023426980F8383080F83930B1
:109AB00080F85C3080F85D3080F85E3080F85F3090
:109AC00006CA30B40D68046943662A4383660A6097
:109AD000A370426990F861301649146813441D7AE6
:109AE0005B7B01EBC5051B026D6803F4E06343F08B
:109AF00064032B6090F8623013449D7CDB7D01EBA6
:109B0000C5011B02496803F4E06343F064030B6082
:109B100021685368194205D0036927225A700369E6
:109B200004229A71036920225A71036980229A7073
:109B300030BC70479832010043690CCB12681A425E
:109B40000CD0094B99420AD9084B9942036994BF3A
:109B50001A220D225A70036904229A717047036910
:109B600027225A70F7E700BF7F1A06003F420F0016
:109B700010B50269D378DBB2D90604463DD5102171
:109B80005806D17038D503F0040303F0FF02002B10
:109B900051D03D49626E00230B7084F85D30002A7D
:109BA0005BD0904794F85D30002B56D02369D022CB
:109BB0009A70236994F83B201A712369012284F872
:109BC0005C200222DA7010BD304B84F860009C42A9
:109BD0004AD02F4B9C4252D094F8391013791F2948
:109BE000DBB207D82848007820B16018013184F82A
:109BF000391003760223D37010BD5906C3D491786F
:109C000001F0100101F0FF000029DDD013F0010385
:109C10001ED194F85C1094F85D00884281BF4B1C03
:109C2000091984F85C3091F83B3013712369D02214
:109C30009A702269DEE7236984F83920C0229A707D
:109C40002369114A1979012111700222DA7010BDBD
:109C5000C023937022691379CCE70122002384F892
:109C60005D2084F83B30A1E7626994F861300949CE
:109C700013440322187A02F043FD2269ACE76269BB
:109C800094F861300449F3E7A89EFF1F3C90FF1F42
:109C9000A890FF1FF99C0000059D00000369DB7878
:109CA00003F0200373B190F860300133DBB2012B75
:109CB00080F860301AD9426990F861301344187AFC
:109CC00002F09ABD70B5426903F0FF0590F861306B
:109CD00013440446187A02F08FFDA36E5BB184F83A
:109CE000385094F83900BDE87040184790F85F305C
:109CF000002BE0D0704770BD0148FFF7CFBF00BF19
:109D00003C90FF1F0148FFF7C9BF00BFA890FF1F8D
:109D10002DE9F047374FDFF8E0903B68026982B0E9
:109D200006460093DDF800800021A025D3789B062D
:109D30005BD53B680193019BC8EB03030F2BF5D95F
:109D400049B1102BF2D000209070336980229A70B4
:109D500002B0BDE8F087726996F8613013440521BE
:109D6000187A02F043FF726996F8613013440121BA
:109D700093F812A0504602F039FF09240021504602
:109D800002F020FF2B46013BFDD10121504602F09D
:109D900019FF2B46013BFDD1013CEFD1706996F8CC
:109DA000611001444FF4A0720C7A4B7B09EBC401A3
:109DB0001B02496803F4E06343F064030B6096F808
:109DC00062300344997CDB7D09EBC1011B024968C9
:109DD00003F4E06343F064030B60013AFDD13269A0
:109DE000D3789B064FF00101A3D4012002B0BDE857
:109DF000F08700BFD09EFF1F98320100F0B50369C5
:109E00001222DA700269937803F0200385B00446C9
:109E10000D46002B5ED0B42393703C4922690B6839
:109E20000093009E05E00B680193019B9B1B042B94
:109E300042D8D37803F0200303F0FF00002BF2D0C8
:109E400094F85D30002B31D04FF0000E4FF0020C33
:109E500004EB0E0393F83B3013710B680393039FDD
:109E6000206907E09B060DD50B680293029BDB1B64
:109E7000052B28D8C378DBB203F0020202F0FF06FC
:109E8000002AEFD080F803C02669F378DBB2DF0642
:109E900032462DD49F062BD5DB0731D40EF1010EAF
:109EA00094F85D305FFA8EFE7345D1D800201DBB5B
:109EB000002384F85E3004E09070236980229A7059
:109EC000042005B0F0BD86702369802204209A70BA
:109ED00005B0F0BD03F0FF06FFF71AFF10B904202C
:109EE00005B0F0BD236984F85F60B0229A7094E7F2
:109EF0008023B3700420DAE726698023B370D7E7A4
:109F0000BEF1000F0CBF02200320F6E7D09EFF1F1A
:109F10002DE9F04106690025122780F8385080F8B5
:109F20003950F770D0F810C09CF802E00EF0200E07
:109F300088B00446884615461E46BEF1000F49D03B
:109F4000B4238CF80230784B21691A680092DDF84E
:109F500000E006E01A6801920198CEEB00000428A8
:109F600030D8C87800F0200000F0FF070028F1D0BA
:109F70004FEA480242F00102D2B20A711A68029214
:109F8000DDF808E0206906E01A6803920399CEEB39
:109F9000010105292AD8C17801F0020101F0FF076B
:109FA0000029F1D04FF0020C80F803C02269D1786B
:109FB00011F0110722D12DBB002E0CBFA02380234E
:109FC000937003E08F70236980229A70384608B03E
:109FD000BDE8F0810EF0FF07FFF79AFE0028F5D0EC
:109FE000236984F85F70B0229A70ACE787702369A8
:109FF000802238469A7008B0BDE8F08180239370C3
:10A000000027E3E7012D75D0A021917021690A791D
:10A01000BE4667464FF0A80C1A680492049805E003
:10A020001A680592059A121A052A4AD8CA7802F0C7
:10A03000020202F0FF08002AF2D0CF702169CA782C
:10A04000D2B212F0100F08465AD1920658D5013DEF
:10A05000EDB2012D49D0BEF11F0F3BD90A79012D78
:10A06000DAD11A680692069D05E01A680792079AE7
:10A07000521B052A46D8C27802F0020202F0FF0104
:10A08000002AF2D00223C3702269D378DBB2D9064A
:10A090003AD49B0634D5B023BEF11F0F93703FD83E
:10A0A000226904EB0E0312791A760EF1010E5FFAA3
:10A0B0008EFE16B1236980229A7084F839E07746C3
:10A0C00084E781F80280236980229A70774684F8B9
:10A0D00039E07BE704EB0E0291F8048082F81880E7
:10A0E0000EF1010E5FFA8EFEB9E781F802C0216918
:10A0F0000846B0E7A82191702069BE460279B0E712
:10A10000774663E78170DEE71021A023D170013B21
:10A11000FDD12269937803F0F7037746937055E7F2
:10A1200023691B79C5E700BFD09EFF1F0148FFF7D9
:10A130001FBD00BF3C90FF1F0148FFF719BD00BFC6
:10A14000A890FF1F704700BF38B5144C0378012258
:10A150005B000546204684F83B3084F85E2084F896
:10A160005D20FFF78BFC20460021FFF747FE0B4CDC
:10A170002978012320461A46FFF7CAFE0128F6D1A6
:10A1800094F8383094F839209A4205D9E21801330E
:10A1900084F83830107E38BDFF2038BD3C90FF1F5A
:10A1A00038B51B4C037801225B000546204684F835
:10A1B0003B3084F85E2084F85D20FFF75FFC20468A
:10A1C0000021FFF71BFE124C2978204601230222B2
:10A1D000FFF79EFE0228F6D194F8382094F8391043
:10A1E0008A420FD2531CDBB2A018994284F838304F
:10A1F000007E0AD9234402321B7E84F8382040EACC
:10A20000032038BD4FF6FF7038BD40F47F4038BDA5
:10A210003C90FF1F0C2901D90020704702314900F2
:10A2200001F0FE01FFF7BCBF70B50C4C0378164679
:10A2300001255B00204684F83B3084F85E5084F8AA
:10A240005D50FFF71BFC31462046FFF717FC2946FF
:10A250002046BDE87040FFF7D1BD00BF3C90FF1F16
:10A26000F8B505460F461646412421463A4628468B
:10A27000FFF7DAFF611C0234C9B232462846E4B265
:10A28000FFF7D2FF592CF0D1F8BD00BF38B5044616
:10A290000D463548FFF706FC6322802120462570D5
:10A2A000FFF7C2FF012002F0C9FC204600225E2118
:10A2B000FFF7BAFF20465D21FFF746FF242801D0B3
:10A2C000002038BD204606220C21FFF7C9FF20469A
:10A2D00001222B21FFF7A8FF204601222C21FFF7A6
:10A2E000A3FF20460E222D21FFF79EFF20460022CD
:10A2F0002E21FFF799FF204601222F21FFF794FF1F
:10A30000204605223021FFF78FFF20460122312110
:10A31000FFF78AFF204600223221FFF785FF204603
:10A3200000223321FFF780FF204600223421FFF76F
:10A330007BFF204600223521FFF776FF20460022D2
:10A340005B21FFF771FF204610225C21FFF76CFFB5
:10A35000204620225D21FFF767FF20468F225E21E5
:10A36000FFF762FF012038BD3C90FF1F10B4047F4F
:10A370004160022CC26002D010BC01F0D7BB8368E0
:10A3800010BC184790E80C00F0B41C6859682568A8
:10A39000164F174E29432160164D17491760D66096
:10A3A00015611160417A154A5C180A3194F824400D
:10A3B00053F8215002EBC40149680D60017A5C1822
:10A3C00003EB8101247ECD6902EBC40149680D6075
:10A3D000817A581803EB810390F83000596B02EB37
:10A3E000C002F0BC53681960704700BF01401F00F5
:10A3F000011000380110007800001F809832010021
:10A40000704700BFF0B50C1EBDF8146034DBB0F926
:10A4100006701919B942C4BF3B1B1BB2002BA646DC
:10A420001CDD002A1146B8BFD11D02F00705CC1073
:10A43000826A012007FB04E1A840012E0A44C0B251
:10A440001ED00CD3022E09D1013B12FA83F3013A3C
:10A4500012F8011F41409A421170F9D1F0BDC0437A
:10A46000013B12FA83F3C0B2013A12F8011F014016
:10A4700093421170F9D1F0BD23441BB20024C6E70A
:10A48000013B12FA83F3013A12F8011F01439A4289
:10A490001170F9D1F0BD00BFF8B50D1E0EDB1446EA
:10A4A0001F46064601F03AFBA84207DD002C05DBFB
:10A4B000304601F037FBA04201DCF8BDF8BD304664
:10A4C00001F02AFB022853D003284BD0012806D1E3
:10A4D0006540F3886C406540013B5D1B2DB2012F48
:10A4E00003D02AD3022F14D0F8BD002C2246B6F98F
:10A4F0000630B06AB8BFE21D42F3CF0202FB03553B
:10A5000004F00704435D012101FA04F41C4344559F
:10A51000F8BD002C2246B6F90630B06AB8BFE21D7D
:10A5200042F3CF0202FB035504F00704435D01210F
:10A5300001FA04F45C404455F8BD002C2246B6F9FB
:10A540000630B06AB8BFE21D42F3CF0202FB0355EA
:10A5500004F00704435D012101FA04F423EA040432
:10A560004455F8BD3389013B591B25460CB2B6E76B
:10A57000F18832890139013A4D1B141B2DB224B2E6
:10A58000ADE700BF2DE9F041079E9DF91880089DB9
:10A5900004461F4600F0C0FF0D4B0E480E4984F8DC
:10A5A0003380FF22002F08BF1F4684F82F2000238E
:10A5B00084F8302084F8312084F832202060A665A9
:10A5C000E565676261652362A3622046BDE8F081AC
:10A5D0003C90FF1FF02701000110013810B5044620
:10A5E000806A034B236008B105F076FB204610BD5E
:10A5F000F0270100F8B5436ADBB190F82C20012563
:10A60000AA4083F83B2083F85E5083F85D500446EF
:10A61000406A03680E461B6800219847606A036819
:10A6200031461B6898472946606ABDE8F840FFF745
:10A63000E5BBC26BC56C1368046A23EA05031360AB
:10A640004CB122684FF00043D3625163D36A002BB0
:10A65000FCDA936BF8BD836B466B0825802410E011
:10A660003768426C3A4332601F68826C3A431A6022
:10A670001A68876C013D22EA07024FEA54041A6007
:10A6800007D02142ECD13268476C22EA07023260DF
:10A69000EAE7F8BD70B50446406A0D4600282BD0A5
:10A6A000A16DFFF749FA002D20460CBFA621A72176
:10A6B000FFF7A0FF606A20B1E16DBDE87040FFF7D1
:10A6C0003BBA216C226D0868236A02430A6093B189
:10A6D000DA7A82B1D00703D5224A99691160DA7A11
:10A6E000910703D5204AD9691160DA7A520702D559
:10A6F0001E4A1B6A136070BD236A002B2BD0D97AC7
:10A70000626DE1B172B6D97ACE0706D51848D9681C
:10A710000668314099610160D97A880706D51548E5
:10A72000196906683140D9610160D97A4E0705D5AB
:10A7300011485969066831401962016062B61B68A8
:10A74000D968914207D00D4818600D49DA6042F08F
:10A75000804018611960226C216D136823EA01039F
:10A760001360A0E700E100E004E100E008E100E0A0
:10A7700080E100E084E100E088E100E001403F008A
:10A7800000003F80436A2DE9F04105460E469046A1
:10A79000002B3ED090F82C100124A14083F83B10F0
:10A7A00083F85E4083F85D40406A036800211B68BF
:10A7B00008F1FF379847FFB2B8F1000F23D03744B4
:10A7C000A046013E686A16F8011F03681B68984797
:10A7D0000134B742E4B216D0202CF3D10121686ACB
:10A7E000FFF70CFB95F82C206B6A520083F83B2096
:10A7F00083F85E8083F85D80686A036800211B68C7
:10A8000098470124DEE7686A0121BDE8F041FFF7BF
:10A81000F5BAC26BC16C136823EA010306EB0804A6
:10A8200013604FF00048A6420ED02B6A16F801EBD9
:10A8300063B11A68C2F82C80C2F834E0D36A002BE6
:10A84000FCDAA642936BF0D1BDE8F081AB6BD5F892
:10A8500034C008208021DCF800206F6C1EEA010F54
:10A8600014BF3A43BA43CCF800201A68AF6C3A439D
:10A870001A601A68AF6C013822EA07024FEA5101E8
:10A880001A60E8D1CFE700BF70B50446406A0D46B4
:10A89000002828D0A16DFFF74FF920462946FFF781
:10A8A000A9FE606A20B1E16DBDE87040FFF744B9D0
:10A8B000216C226D0868236A02430A6093B1DA7A38
:10A8C00082B1D00703D5234A99691160DA7A9107DA
:10A8D00003D5214AD9691160DA7A520702D51F4A95
:10A8E0001B6A136070BD236A002B2BD0D97A626D6E
:10A8F000E1B172B6D97ACE0706D51948D96806688B
:10A90000314099610160D97A880706D515481969DF
:10A9100006683140D9610160D97A4E0705D51248E1
:10A920005969066831401962016062B61B68D968CE
:10A93000914207D00D4818600D49DA6042F080401E
:10A9400018611960226C216D136823EA01031360FA
:10A95000A3E700BF00E100E004E100E008E100E05F
:10A9600080E100E084E100E088E100E001403F0098
:10A9700000003F802DE9F041044686B0806A9DF8D2
:10A9800030801E460F461546B4F90830002800F006
:10A990004281DA1D48BF03F10E02B4F90630D2102D
:10A9A00003FB02F2002105F0BBFCB4F90820202AC9
:10A9B00000F39280B4F90610A34B0120203A7339BA
:10A9C00002EBD27201EBD1714FF0200E0290732096
:10A9D0008DE8014042F34F0241F34F01204600F061
:10A9E00051FE606A84F82D70002800F04D81002D22
:10A9F00040F08A80B4F90830202B14BF3D253C2557
:10AA000084F82C50B8F1000F40F0858006B394F91B
:10AA10003300002818DBC0B2012102F0E7F8012161
:10AA200094F8330002F0CEF8012002F007F900217B
:10AA300094F8330002F0C6F80A2002F0FFF8012172
:10AA400094F8330002F0BEF8606A002800F08280BB
:10AA5000A16DFFF771F804227C492046FFF792FEB2
:10AA6000217A0139C9B22046FFF7C4FD7849042292
:10AA70002046FFF787FE94F92D30012B14BF1421D7
:10AA800010212046FFF7B6FD042272492046FFF749
:10AA900079FEB4F90630802B00F09280602B00F034
:10AAA000A680D9212046FFF7A5FD94F92D30012B72
:10AAB00014BFF12122212046FFF79CFD20460622EB
:10AAC0006549FFF75FFE606A50B3E16DFFF734F848
:10AAD000012006B0BDE8F081B4F906105F4B0120FB
:10AAE000403A52394FF0400E029002EBD27252209F
:10AAF00001EBD1718DE8014042F34F0241F34F0168
:10AB0000204600F0BFFD6CE76DB284F82C50B8F120
:10AB1000000F3FF47BAFFEF7C5FF002E94D076E721
:10AB2000216C226D0868236A02430A6073B1DA7AE5
:10AB300062B1D00703D54A4A99691160DA7A910760
:10AB40007CD4520702D5474A1B6A1360012006B025
:10AB5000BDE8F081236A002B2BD0D97A626DE1B178
:10AB600072B6D97ACF0706D53F48D968056829401B
:10AB700099610160D97A8E0706D53C481969056844
:10AB80002940D9610160D97A4D0705D538485969FE
:10AB9000056829401962016062B61B68D968914254
:10ABA00007D0344818603449DA6042F080401861B8
:10ABB0001960226C216D136823EA010313604AE7D0
:10ABC000B4F90830202B00F08680402B7FF469AF69
:10ABD0002A4920460322FFF7D5FD94F92D30012B99
:10ABE00014BFCF219F212046FFF704FD59E7B4F998
:10ABF0000830102B7FF455AF214920460322FFF780
:10AC0000C1FD94F92D30012B14BFAF211021204636
:10AC1000FFF7F0FC45E7DA1D48BF03F10E02B4F977
:10AC20000630D21003FB02F21046059205F04CF8F4
:10AC3000A06200283FF44DAF059AB3E6114AD969E6
:10AC40001160DA7A7DE700BF48280100282A010058
:10AC50002C2A0100302A0100342A01003C2A01007C
:10AC600000E100E008E100E080E100E084E100E0D4
:10AC700088E100E001403F0000003F8044280100DF
:10AC8000FC2C010004E100E0012194F83100244F84
:10AC900001F0ACFF94F83200012101F0A7FF94F914
:10ACA000312094F9323057F83220E26357F83330CC
:10ACB000206A23640125E56425651A682A431A6021
:10ACC00078B1B8F1000F3FF428AFFFF75BFB002E1F
:10ACD0003FF4BAAE9BE6042212492046FFF752FD2C
:10ACE000DFE6294694F82F0001F080FF294694F80A
:10ACF000300001F07BFF94F92F2094F9303057F8A1
:10AD00003220626357F833306564A5641A68A36320
:10AD100022F001021A60002E3FF496AE77E600BFE3
:10AD20009832010040280100B0F90820D31D48BF27
:10AD300002F10E03B0F90620806ADB1002FB03F279
:10AD4000002105F0EDBA00BFF0B50029BDF81450A0
:10AD50002EDBB0F90660B1422ADA002A59DBB0F9DD
:10AD6000087014461C44BC42C4BFBB1A1BB2002B63
:10AD70001EDDD2B2D408D0F828E016FB041112F080
:10AD80000702DBB20EEB010421D0C2F10807FAB2D0
:10AD9000374F9342BF5C0CD2C3EB020CFF2646FA3E
:10ADA0000CF6012D07EA06073FD005D3022D36D059
:10ADB000F0BD012D39D030D21EF8016026EA070718
:10ADC0000EF801709342F3D3B0F906100C449A1AAE
:10ADD000D2B2072A10D9022D36D0002D14BFFF267B
:10ADE000002613462670083BB0F90610DBB2072B8D
:10ADF0000C44F7D802F00702002AD9D01D4B012DD0
:10AE00009B5C1DD017D3022DD2D1227853402370E2
:10AE1000F0BD13441BB20022A1E7022D25D11EF87C
:10AE2000016077400EF80170CCE71EF801603743EF
:10AE30000EF80170C6E7227822EA03032370F0BD02
:10AE4000227813432370F0BD11462378DB4323702F
:10AE50000839B0F90630C9B207291C44F5D812F0F8
:10AE60000702A5D0034B9B5CCFE73444AFE700BF9C
:10AE7000E0270100D027010070B4C47DBDF80C505C
:10AE8000022C18D0032C1FD0012C0BD0002A03DB7E
:10AE9000B0F90840944201DC70BC7047039570BC67
:10AEA000FFF7B0BAC4880395013CA41A0A4621B240
:10AEB00070BCFFF749BF0689C488013E641AB21A04
:10AEC000E41A12B221B2E1E704890395E41A641A84
:10AED000114622B270BCFFF737BF00BF70B4C57D0A
:10AEE000BDF80C60022D1AD0032D12D0012D03D015
:10AEF000039670BCFFF728BFC488E41AA41A0A4658
:10AF000021B2002A03DBB0F90840944213DC70BC84
:10AF100070470489013C641A114622B2F1E7C488E3
:10AF200005890396013CAD1AED1A621A11B22AB2D4
:10AF300070BCFFF709BF039670BCFFF763BA00BF90
:10AF40002DE9F8430446406A002863D0A16DFEF75E
:10AF5000F3FD052274492046FFF714FCA17901395D
:10AF6000C9B22046FFF746FBB4F90820E588A66A77
:10AF7000D31D48BF02F10E03DB10626A15FB03F517
:10AF80001FFA85F8002A7BD094F82C300125AB40BD
:10AF900082F83B3082F85E5082F85D50606A036848
:10AFA00040211B6808F1FF379847BFB2B8F1000F86
:10AFB00023D03744A846013E606A16F8011F036893
:10AFC0001B6898470135B742EDB216D0202DF3D15A
:10AFD0000121606AFEF712FF94F82C20636A520088
:10AFE00083F83B2083F85E8083F85D80606A0368A5
:10AFF00040211B6898470125DEE70121606AFEF7C2
:10B00000FDFE606A002800F08D80E16DBDE8F84328
:10B01000FEF792BD236A002B2BD0D97A626DE1B185
:10B0200072B6D97ACE0706D54048D9680568294056
:10B0300099610160D97A8D0706D53D48196905687F
:10B040002940D9610160D97A480705D5394859693D
:10B05000056829401962016062B61B68D96891428F
:10B0600007D0354818603549DA6042F080401861F1
:10B070001960226C216D136823EA0103136068E7ED
:10B08000E26BE36C1168276A0B4306EB0809136057
:10B090004FF0004E4E450DD016F801CB2FB33A6855
:10B0A000C2F82CE0C2F834C0D36A002BFCDA4E455B
:10B0B000936BF1D1226C236D11680B43136097B130
:10B0C000FB7A83B1D90703D51D4BBA691A60FB7AA5
:10B0D0009A0703D51B4BFA691A60FB7A5B0702D506
:10B0E000194B3A6A1A60BDE8F883A36BD4F8348030
:10B0F00008208021D8F80020656C1CEA010F14BFDD
:10B100002A43AA43C8F800201A68A56C2A431A608B
:10B110001A68A56C013822EA05024FEA51011A604B
:10B12000E8D1B7E7276AC5E7D827010080E100E04A
:10B1300084E100E088E100E001403F0000003F8042
:10B1400000E100E004E100E008E100E02DE9F04F5B
:10B1500085B09946BDF93870BDF83CA0BB1AC1EB6B
:10B16000090B002BB8BF5B42BBF1000FB8BFCBF19E
:10B17000000B5B450D4616460093804648DC4D4566
:10B180003A4633464CDC194613460A46C5EB0901DC
:10B190009B1A89B2002B0CB2B8BF5B4204EBD4748B
:10B1A000BE42ACBF4FF0FF3201224D4503910292E7
:10B1B0004FEA640429DC9BB201930DE0D8F80070DB
:10B1C000BF69B847019BE41AA3B21CB20135002C39
:10B1D0002DB211DBA94518DB009B5B452A4653467F
:10B1E00031464046EADCD8F80020534697692946A4
:10B1F00032464046B847E5E7029A1644039AA94505
:10B2000002EB030436B224B2E6DA05B0BDE8F08FF3
:10B210004A462B46B94635464D4517461E46B2DDD1
:10B22000304629463E464D4607468946AEE700BFB2
:10B2300010B404682469A44610BC604730B40468A4
:10B24000BDF808500295A46BA44630BC604700BF0F
:10B2500030B40468BDF808500295E46BA44630BCD5
:10B26000604700BF70B40468BDF90C60BDF81050B1
:10B2700003960495246CA44670BC6047704700BFD9
:10B2800010B582B0B0F90C20019101680092002243
:10B290000C6CB0F90A301146A04702B010BD00BFD7
:10B2A000704700BF01F003010129C17506D00329D1
:10B2B00004D0C28803894281838170470289C38890
:10B2C00042818381704700BF2DE9F0410568134E2C
:10B2D0006F6986B0B7420446BDF8308010D1013B9B
:10B2E00013441BB20093CDF804800B46AD6A204690
:10B2F000A8472368DB6AB3420AD106B0BDE8F081F3
:10B30000059304920391B84703A925680EC9E6E79F
:10B31000204606B0BDE8F041184700BF7DB20000EE
:10B320002DE9F0410568124E6F6986B0B7420446B8
:10B33000BDF830800FD1013BCDF804800B44009262
:10B340001BB2AD6A2046A8472368DB6AB3420AD124
:10B3500006B0BDE8F081059304920391B84703A9B4
:10B3600025680EC9E7E7204606B0BDE8F04118475A
:10B370007DB200002DE9F04F0568DFF858B06F6925
:10B3800085B05F450646BDF93890BDF83CA00C4637
:10B39000904615D11F19BC420CDACDF800A0214609
:10B3A00001342D6A4B464246304624B2A847BC427F
:10B3B0003568F2DBEB6A5B4507D105B0BDE8F08F7D
:10B3C0000393B8473568039BE4E7304605B0BDE812
:10B3D000F04F18477DB200002DE9F04387B0994245
:10B3E0000546BDF93840BDF83C6025D0A24212D0D8
:10B3F0000768DFF88080D7F81490C14532D18DE816
:10B4000050002846BC6AA0472B68DB6A434524D11C
:10B4100007B0BDE8F083994202DD084619460346AD
:10B4200028680E96C46B01335B1A1BB22846A446EB
:10B4300007B0BDE8F0436047A24202DD1346224652
:10B440001C4628680E96631C846B9B1A1BB2284608
:10B45000A44607B0BDE8F0436047284607B0BDE802
:10B46000F0431847059304920391C84703A92F6836
:10B470000EC9C4E77DB200002DE9F04FD0F800E01E
:10B48000DFF89090DEF814B083B0CB450446BDF9E8
:10B490003080BDF834A00D4617461E4631D1CDF898
:10B4A00000A0DEF824B0294633463A462046D84765
:10B4B0002368CDF800A008F1FF323A44D3F824B055
:10B4C000294612B233462046D8472368CDF800A05B
:10B4D0002946D3F820B03A4643462046D84720684C
:10B4E000CDF800A0711E29444346056A09B23A46C8
:10B4F0002046A8472368DB6A4B4506D103B0BDE868
:10B50000F08FD847D4F800E0C9E7204603B0BDE883
:10B51000F04F18477DB20000F0B4002401264FF62A
:10B52000FF75094F07600471C475C48104824476B5
:10B53000C4618675067685824582C180028141811B
:10B540008281F0BC704700BF082D01002DE9F04F4B
:10B5500085B00668BDF84450BDF93880CDF800804C
:10B5600004460195D6F848B00392BDF93C60BDF998
:10B57000407089469A46D84723680195009742460D
:10B580005146D3F8488020463346C0472068039B85
:10B590000E930F95856C4B463A4631462046AC4695
:10B5A00005B0BDE8F04F60472DE9F04F87B0174672
:10B5B000BDF9404000912546E91D059344BF2B4647
:10B5C00003F10E010268BDF8486053690294C91086
:10B5D00003912B49BDF9444001968B42824645D1E7
:10B5E000002C3CDD029B3C445E1EB6B24FF00009CD
:10B5F00023B2049301364D46029B002B28DD059BA8
:10B60000002403EB090806E0EDB22B0604F1010467
:10B6100011D4A6421CD0A1B211F0070F23B24FEAF9
:10B620004505F1D1002BB8BF0733DB10013418F802
:10B6300003502B06EDD5009BD2F818B019443A46BA
:10B6400009B2019B5046D847A642DAF80020E2D161
:10B65000039B01379944049B3FB2BB42CCD1D36AD0
:10B66000074A934206D107B0BDE8F08F9847DAF851
:10B670000020B5E7504607B0BDE8F04F184700BFBF
:10B680007DB2000070B4BDF90C60BDF91050BDF87A
:10B69000144003960495059470BCFFF785BF00BF66
:10B6A0002DE9F04F93B090460591C1691090BDF817
:10B6B00070000790BDF874909DF878A0049300295D
:10B6C00000F0CD800A7A0AC9894604998A1AD2B252
:10B6D00003EBC203BAF1010FDA780B9293F905205C
:10B6E0001E8893F802B00F9293F9064079D913B2ED
:10B6F000099323B20C93109B1A68A94B1193194616
:10B7000053698B4240F0A6800B9B002B55D01FFA4B
:10B7100088F300210D93C8462344DDF8409006913C
:10B720000E930F460C46BBF1000F3FD0BDF818102A
:10B730000C9B03971FFA8AF0CB1813FB00F30490BD
:10B740000E9801440D98034409B21BB20A91089364
:10B75000002505E00135EBB264009B45E4B222D937
:10B76000039B2B44590703D1731C18F806409EB263
:10B770002306EFD5099BBDF81000E91811FB00F175
:10B780000598BAF1010F0FFA8AF301441CD007980B
:10B7900001900093D26909B217464846089AB84703
:10B7A000D9F80020D6E7039F5F44FFB2069B0B99B0
:10B7B00001330693DBB29942B5D8D36A119A93420A
:10B7C00043D113B0BDE8F08F0F9B191893690A9A03
:10B7D00029441F4609B2079B4846B847D9F80020BC
:10B7E000B8E700230C93099385E70A9A0D9B013271
:10B7F000013B52B213F0FF030A920D936FD1DDF8B3
:10B800001890079BDDF83C80DDF820A04B4517D051
:10B81000BAF1010F00F0C8800B9A109DCDF804908A
:10B820000BEB8B014FEACB030A4400931146DEF881
:10B830001C405346424609B22846A047D5F800E0CE
:10B84000DEF82C30119A9342BBD0109813B0BDE8AB
:10B85000F04F1847109D284698472A6854E7109AD9
:10B860000598B2F90A308342ABDDB2F90C3043459A
:10B87000A7DD062313FB0A03002BA2DD08EBCA0396
:10B88000002B9EDD537E2BB9049BAF2B02D90133D5
:10B89000DBB20493109BD3F800E0414B11931A469E
:10B8A000DEF81430934240F08E801FFA88F30E9336
:10B8B00008339BB2BDF81420059305230D93002394
:10B8C0000A93CDF83C800FFA8AF3DDF84080CDF87A
:10B8D00018900B921FFA8AFBCDF820A099460A9A7D
:10B8E000BDF810000B9C0E9D0523194611FB00238B
:10B8F0002C481146C75C039702FB0B4214FA81F3F4
:10B9000012B21BB209920C932C462E461CE0089BE7
:10B910000999012B2AB24B4640462DD0079F01972B
:10B92000CDF80090DEF81CA0D047D8F800E0039BCB
:10B930005B0801340393059BA4B25D445E44A342BB
:10B94000ADB2B6B23FF451AF039BD807DFD4079B2B
:10B95000069A9342EBD0089B012B16D0069B0193CD
:10B96000CDF80090DEF81CA009994B4632B2404653
:10B97000D047D8F800E0DAE7DEF818A0079B0C996A
:10B9800022B2D047D8F800E0D1E7DEF818A00C9931
:10B990001346404622B2D047D8F800E0C7E700BFC0
:10B9A0007DB20000582D01000B99109DCDF800903C
:10B9B0000531DEF8204009B2424608232846A04758
:10B9C000D5F800E03CE7109C20469847D4F800E00A
:10B9D0006BE700BFF0B5C36985B004462BB30A29F5
:10B9E00068D00D294AD01A7A914247D3587A8842B2
:10B9F00044D35D688A1A05EBC205AA78002A50D0A4
:10BA0000E87800284DD0207E00283AD095F905E04E
:10BA1000B4F90E00A67DB4F90A70724406FB020266
:10BA2000BA4262DCB4F9102030E00A2956D00D2960
:10BA300024D0027E002A4BD0B0F90E00A57DB4F9C7
:10BA40000A60062212FB0502B2423EDD228AE38131
:10BA500002EBC50212B218462282A78A668A0295B4
:10BA60000B468DE8C00001462046FFF719FEA37D76
:10BA7000E28903EB430302EB4303E381012005B0BA
:10BA8000F0BDA67DB4F90E00B4F91020B4F814E0AE
:10BA9000678A02960B468DE8804001462046FFF7F4
:10BAA000FFFD2979E389A27D012001FB0233E381B7
:10BAB00005B0F0BD0022C2819A7A817D038A01FB24
:10BAC00002330382012005B0F0BDB4F91020C4E7B1
:10BAD000857DB4F91020B0F90E00BEE7028A817DA1
:10BAE000C38102EBC1030382C8E70020E0819B7A97
:10BAF000228A03FB062212B22282C7E7C181028298
:10BB0000704700BF002908BF01218175704700BF41
:10BB100081824182704700BFC07D7047B0F90A0042
:10BB2000704700BFB0F90C00704700BF10B4EFF3CE
:10BB3000108272B6437F33B9017F012907D00329F0
:10BB40000FD00123437702B962B610BC7047124C84
:10BB50002168A1B1114943610B6883610860586194
:10BB6000EFE70F4C216881B10E4943610B68836197
:10BB7000086058610C4B4FF080511960E1E7074BAA
:10BB80004161816120601860DBE7064B41618161A2
:10BB900020601860EEE700BFBC9EFF1FB89EFF1F2D
:10BBA000AC9EFF1FB09EFF1F04ED00E070B5EFF3E9
:10BBB000108272B60C4C206880B10C4E002543698F
:10BBC000236073B19D6102B962B645778368984777
:10BBD000EFF3108272B620680028F0D102B962B685
:10BBE00070BD3360EFE700BFAC9EFF1FB09EFF1F2C
:10BBF000FFF7DCBF184A30B41468002C27D0036864
:10BC000021688B420ED2CB1A00218460C160236070
:10BC1000E06010600223037530BC704711688B42EE
:10BC2000144608D3A2685B1A0360002AF6D182602A
:10BC3000C460A060EEE7D268C2608460E060C5685E
:10BC4000CB1A0222A8602360027530BC7047846062
:10BC5000C4601060DEE700BFB49EFF1FF8B5224E3F
:10BC600034682CB32368002B3AD1204F1D4604E0E2
:10BC70003468ECB12368002B32D1A36803B1DD60D6
:10BC800020693360036825751B68BB4221D1037F9F
:10BC90004560022BC46020D0FFF748FF6368002B8B
:10BCA000E6D023602046FFF7A5FF3468002CE1D1E1
:10BCB000EFF3108372B60E4A00211068116003B9C9
:10BCC00062B628B18468FFF795FF20460028F9D1B5
:10BCD000F8BD224600219847E0E783689847DDE7F2
:10BCE000013B2360E4E700BFB49EFF1F6DA300008B
:10BCF000C49EFF1F024A136801331360FFF7AEBFF3
:10BD0000D09EFF1F704700BF0368F0B4FBB1002551
:10BD100001249D60DC601B4C1A601C44241104F15A
:10BD200044056A11032692009E60174F0679174B4F
:10BD300047F8241002F1604202F5614205F01F0548
:10BD4000012000FA05F5E6541560F0BC7047104C70
:10BD5000236843F40003236000BF0E4B0E4DA4F58F
:10BD60008734A4F59E7401261E60234604609C68F7
:10BD7000002CD0D01033AB420360F8D10023036015
:10BD80001846E2E7008FFCBF1491FF1F44E400E077
:10BD90003C80044000700340407103400168A9B139
:10BDA0000B4BF0B40B441B110A4E0B4F0B4D46F8D6
:10BDB000237003F1440202F01F0401235211A34037
:10BDC000002445F822308C600460F0BC704700BF4E
:10BDD000008FFCBF1491FF1F05BD000080E100E053
:10BDE000024A034B012111601B6818470C71034084
:10BDF0001491FF1F024A034B012111605B68184731
:10BE00001C7103401491FF1F024A034B0121116072
:10BE10009B6818472C7103401491FF1F024A034B83
:10BE200001211160DB6818473C7103401491FF1F2A
:10BE3000F8B50E4671B17AB10746144600253B6845
:10BE400016F8011B1B6838469847013C0544F6D19B
:10BE50002846F8BD0846F8BD1046F8BD00B5064AAC
:10BE6000036812885B6883B001A9ADF80420022240
:10BE7000984703B05DF804FB58320100F0B507465F
:10BE80008BB0002A33D0012A08BF0A2251B32124E3
:10BE900000E0F4B2B1FBF2F502FB1511C8B20929BA
:10BEA00000F1300198BFC8B20AA988BF37302144D9
:10BEB00088BFC0B201F8240C661E2946002DE8D1C7
:10BEC00033B1013CE4B20AAB23442D2203F8242C05
:10BED0003B6801AA11195B683846C4F122029847F1
:10BEE0000BB0F0BD30228DF825202124E8E703684F
:10BEF000C9B21B6898470BB0F0BD00BF0029BABF9C
:10BF000049422D2300230A22FFF7B8BF374A384998
:10BF100013681B06FCD40B6813F08003F8D172B6CB
:10BF200034490A78002A5FD0334A3448F0B4344C9C
:10BF3000176806682568D4680C303E4414320068DF
:10BF40001268304F35442C4420440244C2F34E0260
:10BF50002D4E2E482E4D2F4C42F400423A60376849
:10BF600006682D682C4A24680C303E44006812682C
:10BF70002A4F35442C4420440244C2F34E02284E3A
:10BF80002848294D294C42F400423A603768066837
:10BF90002D68274A24680C303E4400681268254FFB
:10BFA00035442C4420440244C2F34E02224E23481E
:10BFB000234D244C42F400423A60376806682D68ED
:10BFC000214A24680C303E440068126835442C44F1
:10BFD00020440244C2F34E021C4842F40042026074
:10BFE0000B7062B6F0BC704762B6704724B0034075
:10BFF00024B00B40C99EFF1F38B003403CB0034043
:10C0000040B003402CB0034058B003405CB0034044
:10C0100060B0034064B003406CB0034030B00340F4
:10C0200038B00B403CB00B4040B00B4044B00B402C
:10C030004CB00B402CB00B4058B00B405CB00B40E8
:10C0400060B00B4064B00B406CB00B4030B00B40A4
:10C0500030B42948294A2A4B2A4D6024E121047032
:10C0600011701B78284C082B30D00A2B2748284900
:10C0700037D00C2B0CBF35223D2212232A602360BF
:10C0800002600B60234B24491B78244ABBB1012377
:10C090000B601360224B23491B78234A012B26D9BE
:10C0A000042B0FD9082B1ED9102B94BF862387236E
:10C0B0000B6013601D4B01221A7030BC70470B607F
:10C0C0001360E7E784230B601360F3E700F58E202D
:10C0D0000F490830012213232A60236002600B609D
:10C0E000D0E73922F7E785230B601360E2E780236E
:10C0F0000B601360DEE700BF0040074001400740CF
:10C100002491FF1F08B003400CB0034008B00B405F
:10C110000CB00B40CC9EFF1F20B0034020B00B4062
:10C120002591FF1F24B0034024B00B40C99EFF1F80
:10C130000C2830B417D91023984228BF18461C4643
:10C14000104A114D1178181A8C42287018D00F49D6
:10C1500013700B7823B10E490E4A00230B60136055
:10C1600030BCFFF775BF0A2802D90C231C46E7E74D
:10C17000082802D90A231C46E2E708231C46DFE709
:10C1800030BC70472491FF1FC89EFF1FC99EFF1F30
:10C1900024B0034024B00B4028282FD8334B2DE97E
:10C1A000F0411E5CFF2E2BD0314B1B78002B2AD187
:10C1B00032062CD472B62F4D2F4C2F460123266009
:10C1C0002B7062B672B623681B060CD43B781BB981
:10C1D000F4E72B78002BF1D062B602F09BF972B62F
:10C1E00023681806F5D5254B1B6800222A7062B615
:10C1F000234A107843FA00F0BDE8F0810020704730
:10C200000020BDE8F081FFF781FE3206D2D572B67C
:10C210001C4DDFF87C801C4C06F04007FFB206F096
:10C220003F06D8F80030DFB123F01003C8F8003023
:10C2300001232660134A2B7062B672B62368190672
:10C240000CD413781BB9ECE72B78002BE9D062B63D
:10C2500002F060F972B623681B06F5D50B4BC3E7F5
:10C2600043F01003C8F80030E2E700BF5C32010081
:10C27000C99EFF1FCB9EFF1F00B0034010B00340BC
:10C28000C89EFF1FCA9EFF1F00B00B4010B00B409E
:10C290000CB00B400A4A0B49136843F480531360F7
:10C2A0000B7843B9084BC0221A70084B80F30C007E
:10C2B00000B218807047044B80221A70F5E700BF67
:10C2C0002C800440CC9EFF1F21C00C4000C00C40BD
:10C2D000F0B51B4B1B4E596818689A68DB6885B02F
:10C2E0006C460FC4337899071DD5174A174C13783D
:10C2F000174913F0700318BF1370164A164B8027A6
:10C30000177000263320032226706D4608701A70BD
:10C3100072B6043C45F001052046A84762B6237872
:10C3200013F0700309D10D4B064901E0013B02D027
:10C330000A78D207FAD505B0F0BD237005B0F0BD7C
:10C340008832010001000240000002400400024067
:10C350000B000240070002400A000240410D0300AA
:10C36000B0F5006F0AD210B5094B1B78DB07044605
:10C3700006D504F1A0500078C0B210BD002070476F
:10C38000FFF7A6FF04F1A0500078C0B210BD00BFB7
:10C3900001000240B0F5006F17D238B50F4B1B7883
:10C3A000DA070D46044611D504F1A0500378AB42DC
:10C3B0000AD00B4A137813F0700318BF1370074AA2
:10C3C00005701378DB07FCD538BD7047FFF780FF99
:10C3D00004F1A0500378AB42EBD1F5E70100024035
:10C3E0000000024008B5F4F749F9F5F775FD02F0D1
:10C3F00091F8FAE7844641EA000313F003036DD194
:10C40000403A41D351F8043B40F8043B51F8043B17
:10C4100040F8043B51F8043B40F8043B51F8043B1E
:10C4200040F8043B51F8043B40F8043B51F8043B0E
:10C4300040F8043B51F8043B40F8043B51F8043BFE
:10C4400040F8043B51F8043B40F8043B51F8043BEE
:10C4500040F8043B51F8043B40F8043B51F8043BDE
:10C4600040F8043B51F8043B40F8043B51F8043BCE
:10C4700040F8043B51F8043B40F8043B51F8043BBE
:10C4800040F8043B403ABDD2303211D351F8043B5E
:10C4900040F8043B51F8043B40F8043B51F8043B9E
:10C4A00040F8043B51F8043B40F8043B103AEDD20D
:10C4B0000C3205D351F8043B40F8043B043AF9D25E
:10C4C000043208D0D2071CBF11F8013B00F8013B31
:10C4D00001D30B8803806046704700BF082A13D33E
:10C4E0008B078DD010F003038AD0C3F10403D21A56
:10C4F000DB071CBF11F8013B00F8013B80D331F88A
:10C50000023B20F8023B7BE7043AD9D3013A11F809
:10C51000013B00F8013BF9D20B7803704B78437074
:10C520008B7883706046704708B5104C08E023682C
:10C5300059050DD423681A050FD42368DB0411D4E0
:10C5400023685803F3D500F08DFE23685905F1D513
:10C5500002F044F823681A05EFD502F0D5F82368F5
:10C56000DB04EDD500F0F0FCEAE700BF34800440C6
:10C5700008B5FFF7D9FF00BF014B10221A807047A2
:10C5800000200540704700BF094908B50B6830B16D
:10C590006A461844A2F58052904202D208601846BA
:10C5A00008BD03F063FB0C2303604FF0FF3008BDB0
:10C5B0002891FF1FFEE700BFEFF3138070B9EFF380
:10C5C00010836BB9EFF305825AB94FF48070EFF323
:10C5D00011832BB1984228BF184670474FF0FF30A7
:10C5E00070470F2A01D81846F1E7014BD05CEEE7FF
:10C5F000F0E300E0F0B44D1E2E46002400E00134CC
:10C60000B0FBF2F302FB1300092800F130078ABFE8
:10C610003730F8B2C0B206F8010F1846002BEED141
:10C620000A1953704CB1107815F8016F2870013356
:10C63000E01A834202F80169F5DB0846F0BC704756
:10C64000704700BF10B40F4B53F8302092F880426F
:10C650002CB1012369B182F8803010BC704703EB24
:10C66000C0035B681A6841B922F002021A6010BC6C
:10C67000704782F8003110BC704742F003021A6024
:10C6800010BC7047983201001C4A02EBC00301291C
:10C690005B6811D004291BD052F83000002280F8CA
:10C6A000802229B1022920D0032922D01A607047A4
:10C6B0004FF480721A60704752F830004FF4A27243
:10C6C00080F880121A601A6822F020021A607047FF
:10C6D00052F830104FF4A272012081F880021A60E3
:10C6E0001A6842F020021A60704740F203121A6082
:10C6F00070474FF481721A60704700BF9832010092
:10C70000212848D8F8B5042A44D8DFE802F0484B7D
:10C710004E0345004FF410262B4B03EBC0030D4690
:10C720005C68216811F4E06148D0284B284A294907
:10C73000C3F89C2104F140422748C3F8A411A2F594
:10C740009221264FC3F8A0017C292548C3F8A8717F
:10C75000C3F8AC012CD9A2F594237C2B2AD9A2F5DD
:10C7600096237C2B28D9A2F598237C2B29D9A2F5D6
:10C770009A227C2A27D81B4872B6236823F4702398
:10C7800043F08072C4F384011643236040F82150C3
:10C79000266062B6F8BD70474FF43026BCE74FF410
:10C7A0000026B9E74FF44026B6E74FF42026B3E75A
:10C7B0000D48E1E70D48DFE70D48DDE7FFF764FFCF
:10C7C000B3E70C48D8E7F8BD983201000082FF1F9C
:10C7D000F188FF1F9988FF1FC588FF1F6D88FF1F05
:10C7E0004188FF1F0492FF1F2C91FF1F6491FF1FC0
:10C7F000B491FF1FE491FF1F1A4B03EBC00010B46C
:10C80000426802F14043A3F592217C2923D9A3F584
:10C8100094217C290DD9A3F596217C291FD9A3F554
:10C8200098217C2919D9A3F59A237C2B11D80E4C79
:10C8300000E00E4C72B613680D4823F08773C2F304
:10C84000840123F4803343F08073136044F82100A3
:10C8500062B610BC7047074CECE7074CEAE7074CA0
:10C86000E8E700BF983201000492FF1F6491FF1FA8
:10C8700041C600002C91FF1FE491FF1FB491FF1FE0
:10C8800030B4054B054D064C002210211A602A6079
:10C890002060196030BC704714D0034004D00340BE
:10C8A00000D00340282838B52ED0002904464FDD9B
:10C8B0005F4B1B78012505FA03F28A4202D8212832
:10C8C00037D938BD0338C2B2012A3AD9202C4AD010
:10C8D000192C48D0574A126802FB011222FA03F3BE
:10C8E0001D2800F29B80DFE800F0928B847D9999EF
:10C8F000766F99999999999999999968615A5399E3
:10C900004C99999999999945494B1B780B2B08D9C2
:10C910000C2B1CBF0C3B19410846BDE83840FFF703
:10C92000B9BCC3F10C0399400846BDE83840FFF795
:10C93000B1BC2946FFF786FE2946BDE83840FFF71F
:10C94000A3BE3D4A126802FB011222FA03F3C7E7B5
:10C950002128B6D80021FFF775FE20460121BDE849
:10C960003840FFF791BE354A126802FB011222FAE5
:10C9700003F3B5E73249334A0B604FF45173136048
:10C9800038BD3149314A0B604FF45173136038BDE3
:10C990002F49304A0B6040F24443136038BD2E49A2
:10C9A0002E4A0B6040F24443136038BD2C492D4A97
:10C9B0000B6040F24443136038BD2B492B4A0B6097
:10C9C00040F24443136038BD29492A4A0B6040F2C3
:10C9D0004443136038BD2849284A0B6040F2444361
:10C9E000136038BD2649274A0B6040F24443136068
:10C9F00038BD2549254A0B6040F24443136038BDD9
:10CA00002349244A0B604FF45173136038BD224907
:10CA1000224A0B604FF45173136038BD212C3FF64E
:10CA200050AF7F29D4BF00210121204693E700BFEA
:10CA30000C92FF1F088003400890034008800B40C1
:10CA400010800B4048A0044018800B404CA00440CC
:10CA50001880034008B004401080034004B0044034
:10CA60004080034018C004403880034014C0044094
:10CA70002880034010B00440208003400CB00440E4
:10CA80003080034010C00440488003401CC0044074
:10CA900018900340349004401090034030900440BC
:10CAA00038B1102828BF1020044AC3B21078137080
:10CAB0007047024A01231078137070470C92FF1FD1
:10CAC0002DE9F8430E4680463249334D304603F097
:10CAD00053F847F6122300281ABF1D464FF00209EB
:10CAE0004FF00109002425FA04F002F04FFE4FF048
:10CAF0005E51074602F0A2FE0146304603F050F8B0
:10CB000030B90134072CEED1E80902F03FFE0746A8
:10CB10003146384602F046FF4FF07C5102F084FD6A
:10CB200003F078F84FF6FF729042A8F1030328BF94
:10CB30001046012B29D9B8F1170F17D8174B23FA34
:10CB400008F303F0010383F0010223B9B8F1190FD0
:10CB50000FD0BDE8F883124B124D13491A6044EA16
:10CB6000C9042A6008601C60BDE8F883B8F1200F92
:10CB7000ECD10E4B0E4D0F49002244EAC9041A6055
:10CB80002A6008601C60BDE8F8830B4B0B4D0C4914
:10CB9000F2E700BF001BB740006CDC026006F0004B
:10CBA00000800340048003400880034000800B4065
:10CBB00004800B4008800B40009003400490034029
:10CBC00008900340212801D8FFF73CBD704700BF03
:10CBD000212806D8044B53F8303093F80002C0B235
:10CBE00070470020704700BF98320100212801D80B
:10CBF000FFF74ABD704700BF72B60C490C4B0D4A97
:10CC00001B680868126862B6520102D5322B88BFD1
:10CC100001300949C3F5BB334FF47A72FF33A1FBEE
:10CC2000031302FB00F000EB93107047D09EFF1F30
:10CC300018E000E004ED00E0ABAAAAAA2DE9F84351
:10CC4000054672B6204F214B214A1B683C6812688A
:10CC500062B6520102D5322B88BF013495B3C3F5B9
:10CC6000BB331C4EDFF86490DFF86480FF334FF471
:10CC70007A72A6FB031302FB04F404EB931472B65E
:10CC8000D9F800103A68D8F800E062B6C1F5BB33B5
:10CC9000FF33A6FB03031EF0806FC4EB93134FF426
:10CCA0007A7002D0322988BF013200FB0233B3F51B
:10CCB0007A7F04D3013D05D004F57A74DFE701F0F3
:10CCC00029FCDCE7BDE8F883D09EFF1F18E000E0F8
:10CCD00004ED00E0ABAAAAAAF8B52D4B2D49DFF868
:10CCE000D0E0DFF8D0C02C4E2C4D2D4C2D4A2E4FCD
:10CCF0004FF4000018604FF0807018604FF0007023
:10CD000018604FF0806018604FF0006018600020DD
:10CD1000086028234BF6FF71CCF80010CEF80030E5
:10CD2000336013602B6023603B60B362936209221F
:10CD300045F8242CC4F8D80F05F57F65C7F8D41F33
:10CD400007F5FF2707F5FA67C6F8F83F2B6006F5E9
:10CD5000FF26C4F8D42F05F5FD2504F5FF2438601F
:10CD600006F2F4761148316005F5FF6504F5FD64BF
:10CD70002B6023600260FFF76BF91920FFF75EFF5D
:10CD800000F0B6FF40F21310BDE8F840FFF756BFC1
:10CD900008E100E004800340148003402480034045
:10CDA0002C8003401C8003403480034000800B40F3
:10CDB0000C800340088003402DE9F84F214B1B688D
:10CDC00007460BB101221A70DFF888901E4D99F8C2
:10CDD0000040DFF884801D4E0134272C8ABF4FF0BD
:10CDE000000A5FFA84FA5446AB462B78A34216D168
:10CDF000FFF7E2FB40281FDC33791B06F5D59BF8D3
:10CE000000300133272B86BF00221346DAB218F810
:10CE10000330DBB2F3712A702B78A342E8D00C49BF
:10CE20000A4BFFB208F804700120AC22087089F8A0
:10CE300000A0DA70BDE8F88FFF28D6DD01F06AFBAC
:10CE4000D3E700BF489FFF1F459FFF1F00C006405C
:10CE5000449FFF1F4C9FFF1FDC9EFF1F1C4BDFF8F2
:10CE600094C01A681B49F0B542F480521A4D1A60FA
:10CE7000DFF884E0194F1A4E1A4C00238CF800306A
:10CE80004FF451722B701F2840F213358EF800308A
:10CE90003B70337025600A6012D819460124124A8B
:10CEA000124D11701248547000212C2740269372A5
:10CEB0004FF4003491701174D7702E700460F0BD7F
:10CEC000C0F34431C0F3471400F01F03E7E700BF8D
:10CED000348004400CC00440D99EFF1F459FFF1FB3
:10CEE000449FFF1F08C0044000C0064031E400E03A
:10CEF00004E100E0D89EFF1F4C9FFF1F034B1B68FF
:10CF0000DB0401D5FFF758BF704700BF34800440F1
:10CF100010B5044C237823B101F0FCFA2378002BE0
:10CF2000FAD110BD449FFF1F054A064B10781B78AD
:10CF3000C0B2DBB2984238BF4030C01A704700BF61
:10CF4000D89EFF1FD99EFF1F30B42B4B1A79940631
:10CF50001FD52A48DA790378294901333F2B09780C
:10CF6000C8BF00238B42D2B203D0264CD9B2E254C0
:10CF70000170254A116861B1244A1278D2B29342F5
:10CF800036BFC2F140029B1A9B18272BC4BF012356
:10CF90000B70194AD378DBB2180611D45A060DD596
:10CFA000154B1B795B0609D5194B1A491B680022E2
:10CFB0000A7003B11A70104B2C22DA7030BC704723
:10CFC00011790906EAD5144910480C780178C9B2DC
:10CFD0008C420DD04A1C272A84BF00210A460F4DDF
:10CFE000054C98BFD1B2AA5CD2B2E2710170D5E70C
:10CFF0006C21D170D2E700BF00C00640D89EFF1F51
:10D00000D99EFF1F049FFF1FD49EFF1F459FFF1F38
:10D01000489FFF1F449FFF1F4C9FFF1FDC9EFF1F69
:10D0200021282FD8184B195CFF292BD0174B184AF1
:10D03000DFF870C003EBC000F0B54368DFF868E0CC
:10D04000144F154D154E00241C60DEF800300120F1
:10D0500043F020038840CEF8003014604FF4A073F2
:10D0600038602E60C2F800C0013BFDD113689B05FB
:10D07000FCD42023013BFDD1094B09B233F8110048
:10D0800080B2F0BD00207047A83301009832010043
:10D0900000500440085004400450044000000203C3
:10D0A0000051044080014A0038800440431E032B95
:10D0B00014D872B60A4951F8230068B170B4094C0B
:10D0C000058834F81320466841F82360521B24F881
:10D0D000132062B670BC704762B67047002070477C
:10D0E000A89FFF1FECA1FF1F013803280BD872B6C1
:10D0F000074B53F8203043B100205B680130002B10
:10D10000FBD162B67047002070471846F9E700BFB0
:10D11000FC9FFF1F30B472B62B4A13781D0706D54B
:10D120002A4B196A002936D0996A002941D05378D0
:10D130001C0706D5254B196C00293ED0996C002997
:10D1400039D09378190705D5204B196E002936D0B0
:10D15000996E89B1D3781B0707D51C4BD3F8802073
:10D160007AB3D3F8882011213AB162B6184B002265
:10D170001A7030BC00F04ABE0D21154C154D2278B6
:10D1800043F8315003EBC1030830013A5860227074
:10D1900062B630BC704704220D4C0F4D217843F825
:10D1A000325003EBC20308304A1E5860227062B648
:10D1B000EFE70521E1E70921DFE70822ECE70C2290
:10D1C000EAE71022E8E700BFCC3301000080FF1F30
:10D1D00025A0FF1FC800400088004000431E032B0D
:10D1E0001DD81B4A400140F0100030B4104472B604
:10D1F000184CE25C032A1BD8DFE802F00212151774
:10D2000003220D88E25410F0080F14BFC8238823AE
:10D2100043EA054308310360416062B630BC7047A1
:10D2200008300222EDE70522EBE708300422E8E7A8
:10D23000094A52F8230038B1084A52F823004160E5
:10D2400042F8231062B6E9E742F82310034AF7E7F1
:10D250000080FF1F34A0FF1FFC9FFF1F0CA0FF1FBB
:10D2600000BE70472DE9F04FDFF818B3DFF818A3C0
:10D2700087B044E0AD4F4FEA930807EBC809013E81
:10D28000D9F8042003F00803F6B2A2F1080003F075
:10D29000FF04002B40F0018157F838301B0C99B285
:10D2A00022F8081C002B00F0EF80A14B22F8064C5E
:10D2B00042F8044C53F82620002A00F0CF819D4DFF
:10D2C00055F8263058609C4C45F8260034F8163046
:10D2D000194424F8161000F079FD002800F0C281EE
:10D2E000964A974B19F0080F00F1080018BF134633
:10D2F000C9F8040047F8383008238BF800309BF851
:10D300000040E4B265071CD58E4B1B78B3B18E4943
:10D310000A7802F0FF0322B1013BDBB20B7003B9C4
:10D3200000BE8A490A7802F0FF032AB1013BDBB252
:10D330000B70002B00F0688100F066FE04238BF870
:10D34000003004F0080303F0FF02002B00F0C98056
:10D350009AF80030DBB21E098CD19A08DFF8CC9124
:10D3600059F8321009EBC200C1F38301013940685A
:10D370000C2900F28580DFE801F07A7A83838383C9
:10D3800083834683838307000168714D4068714F32
:10D39000714E6860296088B240F281610024674B59
:10D3A00049F832304FF0010E88423C60C9F8104015
:10D3B000C9F8184086F800E05C4A00F2E780B0F552
:10D3C000D06F80F01B82B0F5817F00F0D98100F230
:10D3D0006981802800F02A82822840F0D781A988BC
:10D3E00001F07F01042900F2D1815C485C4A890088
:10D3F00008441470547001788C0740F1608382F8FF
:10D4000000E0022173E1534F3A682AB3554B524E64
:10D41000554819883478057840298E4645F0020829
:10D4200028BF4FF0400E002C84F001043470CEEB86
:10D4300001010CBF8824C82409EBC80689B285F015
:10D44000010544EA0E447260198049F8384072447C
:10D450000570002965D03A603D4B1A88B2F5A06F7F
:10D460000ED100219A785970404B1A7008E0384963
:10D470003F4C0D68A54200F09880304949F83210C1
:10D480003C4A0123137037E72C4A2D4B19F0080F43
:10D4900018BF134647F838302EE700F0B7FC364A7D
:10D4A000364952F82630002B00F0E38058688C5D36
:10D4B00042F8260003F10802C9F80420032C05D81D
:10D4C000DFE804F02C02292602228A551A8819F076
:10D4D000080F0CBF8823C82343EA024347F83830BB
:10D4E0000AE7E00700F19380210600F1D180A2074E
:10D4F00006D5234A234913780220DBB21370087043
:10D50000E30602D51F4B10221A7007B0BDE8F08F5A
:10D5100004228A55DAE705228A55D7E703228A557D
:10D52000D4E7BEF1400F18BF002294E70080FF1F30
:10D53000A89FFF1F549FFF1FECA1FF1FC8004000C2
:10D540008800400030A0FF1FB99FFF1FA4A0FF1F4D
:10D550001CA0FF1F509FFF1FB89FFF1FC020074048
:10D5600028A0FF1F649FFF1F24A0FF1F98200740D3
:10D570002109000394200740FC9FFF1F34A0FF1FD8
:10D58000882007408020074090200740B0F5106FAA
:10D5900000F07C8140F2A38040F62112904240F0DE
:10D5A0007B82A54A012313706AE74C68A3498C4229
:10D5B0007FF463AF0178A9297FF45FAF41784529F3
:10D5C0007FF45BAF8178C2297FF457AFC1786B29B4
:10D5D0007FF453AF9A489B4E0178347881F001056F
:10D5E000002C41F0020105700CBF8820C82084F097
:10D5F000010449F8310009EBC1019348347000255A
:10D6000005244D60047038E700F064FF94E68F4B0A
:10D6100089488B491A614FF0020E80F800E08C4F68
:10D620000A708C49196099608B4E8C4D8C4C9A61B4
:10D630000D213970FF213170DFF84CE22970227022
:10D64000884D894A8EF800109F27012406F8047C33
:10D650005D600470DA6007B0BDE8F08F43F8260023
:10D66000824D30E6824A47F8380013780133137050
:10D6700042E68B5D032B00F2BA8001A252F823F040
:10D68000F9D20000F9D20000D9D60000D3D60000AC
:10D690006F49724B80220D2008701A70A2077FF527
:10D6A0002FAF26E740F20232904240F0ED81AA8887
:10D6B00002F07F02042A69D86D88002D66D1644982
:10D6C000CDF804E0920011440A7842F002020A7098
:10D6D000C1E101238B550FE600238B550CE6B0F515
:10D6E000086F53D16349644A097811707146ED8817
:10D6F0008D4280F0E88252480478402DAE4644F0D6
:10D70000020C28BF4FF0400E02EB0E0309EBCC01D8
:10D71000029301234A604FEA0E48CEEB05010193C4
:10D720000025C82242EA080384F0010249F83C308F
:10D7300035700270DFF814C1424BDFF8048149BB39
:10D74000BEF1400F7FF42DAF42F0020C09EBCC0389
:10D75000029ADFF8F8E05A608DBB0D0445F08805A9
:10D760009DF804304EF83C500A4433700470134660
:10D7700040297FF416AF0021404A3B60118010E73A
:10D78000AA8802F07F02042A40F28B81304A0F23DC
:10D79000137006E74029D7D942F002020CEBC20011
:10D7A000029E4660BDB19DF8045035481D70334659
:10D7B000403988F8004040334CF83200DCE79DF8EF
:10D7C000043033700D04029B047045F0C8050B440F
:10D7D0004EF83C50CCE79DF804501D70029B1D484C
:10D7E00088F80040403940334CF83200C4E719F063
:10D7F000080F0CBF022303238B557DE521494A689E
:10D80000002AC3D06C88B5F804E003E00C314A6804
:10D81000002ABBD00B88A342F8D14B887345F5D1C1
:10D82000240A032C0CBF1178098960E7124A0221EF
:10D83000147054705BE700BF94200740010004009F
:10D8400024A0FF1FB89FFF1FB99FFF1F0080FF1F6D
:10D85000C020074088004000882007408020074003
:10D8600098200740689FFF1FBC9FFF1F549FFF1F0A
:10D8700025A0FF1F30A0FF1F28A0FF1F649FFF1FD0
:10D88000C8004000D03301008C200740B248116A24
:10D89000AC7804700C0600F19881D9F82820AF49C3
:10D8A000100600F1DB81D9F83020AC49120600F1F6
:10D8B000D081D9F83820A949130600F1C581D9F8DB
:10D8C0004020A649150600F1BA81D9F84820A3499D
:10D8D000140600F1AF81D9F85020A049100600F1DC
:10D8E000A481D9F858209D49120600F19981D9F8F0
:10D8F00060209A49130600F18E81D9F86820974973
:10D90000150600F18381D9F870209449140600F1BE
:10D910007881D9F878209149100600F16D81D9F805
:10D9200080208E49120600F16181D9F888208B4948
:10D93000130600F15581D9F890208849150600F1A9
:10D940004981D9F898208549140600F1FF80844860
:10D95000844A854901908548854D864C049700236B
:10D960000596029580460F4616461D46039430687C
:10D9700028B1446800F04AFA2046002CF9D100236F
:10D980003360029B38681A46002342F8253028B1DC
:10D99000446800F03BFA2046002CF9D100223A609E
:10D9A000019A98F800301146002241F8042B039A9E
:10D9B0000191023B4FF0000122F81510032B07D80C
:10D9C000DFE803F05D025D024FF0010388F80030EC
:10D9D0000135042D06F1040607F1040708F10108DA
:10D9E000C5D1654C654D2278654B049F059E00218D
:10D9F000100729701A7000F19280624962780A70EB
:10DA00000021C9F83010C9F838101107DFF84C812F
:10DA10006ED4A2785C49DFF844810A7000211207B5
:10DA2000C9F85010C9F858104BD4E27857494B4CFC
:10DA30000A7013074FF00001C9F87010C9F8781088
:10DA400000F1AE8033780193002283F00105C9F81C
:10DA50009020C9F898200021029188468E460A46F7
:10DA60004B48047844F0020C09EBCC030393019B70
:10DA7000002B039B5A600CBF8822C82252E64FF04D
:10DA8000000388F80030A3E7B0F5A06F7FF47EAE06
:10DA9000012300250193DEE740F621229042F7D0D2
:10DAA00074E66D88002D7FF471AE3A49CDF804E03C
:10DAB000920011440A7822F002020A70CBE7022198
:10DAC00015E600F083F9002800F0EB800830324AB8
:10DAD000C8F86400C8F8602000F078F9002800F069
:10DAE000DA8008302D4AC9F86C00C9F868209CE734
:10DAF00000F06CF9002800F0E0800830264AC8F8F1
:10DB00004400C8F8402000F061F9002800F0CF8000
:10DB10000830224AC9F84C00C9F8482079E700F0DB
:10DB200055F9002800F0A58008301B4AC9F82400E8
:10DB3000C9F8202000F04AF9002800F0948008304D
:10DB4000164AC9F82C00C9F8282056E7D1F89C00DD
:10DB5000083800F05BF9FAE630A0FF1F0080FF1FD5
:10DB60000CA0FF1FA89FFF1FFC9FFF1F34A0FF1FDB
:10DB7000549FFF1FECA1FF1FCC33010025A0FF1F06
:10DB8000C4200740C8200740CC200740D0200740D1
:10DB900024A0FF1FC020074088004000C8004000AC
:10DBA00000F014F9002870D008304F4AC4F88400FF
:10DBB000C4F8802000F00AF9002860D008304B4AF1
:10DBC000C9F88C00C9F888203CE7506A083800F092
:10DBD0001DF962E6D1F89400083800F017F9B0E6B4
:10DBE000D1F88C00083800F011F9A4E6D1F88400CF
:10DBF000083800F00BF998E6C86F083800F006F90D
:10DC00008DE6486F083800F001F982E6C86E0838E2
:10DC100000F0FCF877E6486E083800F0F7F86CE69C
:10DC2000C86D083800F0F2F861E6486D083800F079
:10DC3000EDF856E6C86C083800F0E8F84BE6486C9A
:10DC4000083800F0E3F840E6C86B083800F0DEF86A
:10DC500035E6486B083800F0D9F82AE6C86A083873
:10DC600000F0D4F81FE62A78C9F8280001322A709B
:10DC7000C3E62A78C9F8200001322A705AE72A78C8
:10DC8000C9F8880001322A70DCE62A78C4F88000DE
:10DC900001322A708EE72A78C9F8680001322A70AA
:10DCA000C3E62A78C8F8600001322A7014E72A789F
:10DCB000C9F8480001322A70ABE62A78C8F840005B
:10DCC00001322A701FE740298E4628BF4FF0400ED0
:10DCD00002EB0E0302930123CEEB01014FEA0E4843
:10DCE00000250193BCE600BF88004000C80040004A
:10DCF000F8B500F08FFD294B29482A4C2A4F2B4DAF
:10DD0000DFF8BCC0DFF8BCE0294E00221A605A6080
:10DD10009A60DA601A615A619A61DA611A625A622B
:10DD20009A62DA621A635A639A63DA631A645A640B
:10DD30009A64DA641A655A659A65DA651A665A66EB
:10DD40009A66DA661A675A679A67DA67C3F88020B4
:10DD50000168C3F8842041F480210160C3F30721E6
:10DD60002170C3F30740134938701B0E2B70FF233B
:10DD70008CF80030104D8EF8003010480B700123E5
:10DD8000337084F8642070264FF40074102207F872
:10DD90002C3C2E70046081F8F820F8BD0080FF1F35
:10DDA000348004409C200740B0200740B420074046
:10DDB000942007401020074049E400E008E100E01B
:10DDC0008020074088200740704700BF72B60D488A
:10DDD0000268B2FA82F30F2B10DC4FF00041D940F9
:10DDE00022EA0102026062B6074803EBC303DB00CC
:10DDF000C2180021C15010465160704762B6002021
:10DE0000704700BF1092FF1FBC83FF1F0D4B0E4ACF
:10DE1000C31AA2FB03231B090F2B0CD80B4A127841
:10DE200052B972B60A484FF00041026821FA03F372
:10DE30001A43026062B67047064A1278002AF0D090
:10DE4000FFF768B9BC83FF1F398EE33825A0FF1F99
:10DE50001092FF1F30A0FF1F38B50E4B0E4C1B68F1
:10DE6000218805468BB1B1F5917F05D20B4A4B1C39
:10DE700055549BB2238038BD0022084898470021A2
:10DE8000064A55540123238038BDB1F5917FEDD367
:10DE900038BD00BF5CA0FF1FF6A1FF1FFCA1FF1F44
:10DEA0002DE9F843214E224F3168012380463B7013
:10DEB000B1B1204D4B8801EB8302013300240F2BBD
:10DEC000C2F808802C7004D84B8000233B70BDE85A
:10DED000F88340230B800320FFF780F93460F4E7D8
:10DEE000DFF8549099F80030002BF0D0114D45F632
:10DEF000215408E0013C12D02B7883B900F00AFBD2
:10DF000099F800307BB10320FFF7EEF80528F1D82F
:10DF1000FFF75CFF014630600028EBD0CAE7012321
:10DF20002B70BDE8F883BDE8F88300BF78A0FF1F21
:10DF30004CA0FF1F7CA0FF1F30A0FF1F1201F8B5EF
:10DF4000D5B2A1B3012943D04378044600781B061B
:10DF500043EA004040F4704045F004068F1E304311
:10DF6000FFF79EFF022F04F1020314D9053414F8C1
:10DF7000023C14F8032C14F8010C1B0443EA02239E
:10DF8000334343EA0060033FFFF78AFF022F234633
:10DF900004F10304EBD8022F23D0012F0DD045F458
:10DFA000774040F00500BDE8F840FFF779BF14481E
:10DFB0002843BDE8F840FFF773BF187845F47705AC
:10DFC00045F0060545EA0020BDE8F840FFF768BFC8
:10DFD00003780C4845EA03452843BDE8F840FFF7BD
:10DFE0005FBF1A78587845F0774545F0070545EA50
:10DFF000022545EA0040BDE8F840FFF751BF00BFE9
:10E0000006F0F70007F000F738B5084B1C7824B984
:10E01000074D296809B14B8803B938BD9B000B80B7
:10E020000320FFF7DBF82C6038BD00BF4CA0FF1FBA
:10E0300078A0FF1F2DE9F041AD4E33680746002B55
:10E0400000F092801D885A88910803EB8101043208
:10E05000AA428C6842D25A8004F00F064FEA142874
:10E06000A449A6F1080208F00F00C4F30313062A1E
:10E0700000F101050B701AD9B31E012B5FFA88F06D
:10E080004ED9052E48D0042E00F0A481731F022B18
:10E090007FD90F2E0ED1F72842D8F02802D0964B08
:10E0A0001B883BB1FFF7D8FE0020BDE8F08127B107
:10E0B000BD4202D00020BDE8F081082EC4F3033336
:10E0C00000F08780092E11D00A2E40F094800A2B90
:10E0D000F0D18A4B8A4A1B68A02181E01846FFF7DD
:10E0E00095FE0420FEF7E2FF3060B5E7092BE1D191
:10E0F000270E00F07B81834B814A1B689021C4F37B
:10E1000007461170EDB2FCB2002B00F09D80224654
:10E1100031462846984797E0F02843D9F72841D060
:10E12000F1380E28C6D801A353F820F0E3E200002E
:10E13000C7E20000B5E20000B5E00000B5E0000075
:10E14000A7E20000B5E0000087E30000B5E00000B2
:10E1500051E300006BE300008FE20000B5E0000037
:10E1600077E200005BE20000674B1B78002BA1D038
:10E170000420FEF79BFF0346306000289AD00588F4
:10E18000002D7FF460AFFFF741FE35602846BDE803
:10E19000F081FFF761FEC4F30740FFF75DFE072E35
:10E1A00002D1200EFFF758FE534B584A19885848A1
:10E1B0001468584D524A017000270E0AF0201F8043
:10E1C0002E7010700CB301225348A0470120BDE807
:10E1D000F081082B7FF46EAF504B494A1B688021B9
:10E1E000C4F307461170EDB2240E6BB328462246E5
:10E1F0003146984728E00B2E11D10B2B7FF45AAFF4
:10E20000474B3F4A1B68B021EAE7464B1B68002B8F
:10E2100000F0FB80404898470120BDE8F0810C2EBB
:10E2200040F000810C2B7FF445AF3F4B344A1B6814
:10E23000C0211170EDB2C4F30746002B00F0C88076
:10E2400028463146240E98473849314A314B0D70E3
:10E2500016701C700120BDE8F081354B1B68002B47
:10E2600000F0D6809847C4F30746254BEDB2240E44
:10E2700083F80080E8E72F4B1B68002BF2D12E4B70
:10E280001B68A3B1FE209847C4F30746EDE72B4B6C
:10E290001B68002BE6D1284B1B6843B1FC20984734
:10E2A000C4F30746E1E7264B1B68002BDAD1C4F321
:10E2B0000746DAE7234B1B68C4F30746002BD4D08C
:10E2C00030469847D1E7204B1A68002AEFD0260C39
:10E2D000630C06F07F0003F47E531843F6B29047B8
:10E2E000C3E71A4B1B68C4F30746002BE8D1BCE711
:10E2F00084A0FF1FFAA1FF1FF6A1FF1F60A0FF1F50
:10E30000F4A1FF1F94A0FF1F30A0FF1F5CA0FF1F00
:10E31000F8A1FF1FF9A1FF1FFCA1FF1F8CA0FF1F89
:10E3200090A0FF1F74A0FF1F50A0FF1FFBA1FF1FA5
:10E330003CA0FF1F40A0FF1F44A0FF1F80A0FF1FA5
:10E3400070A0FF1F88A0FF1F58A0FF1F6CA0FF1F19
:10E350003F4B1B68002B85D13E4B1B68002BA6D082
:10E36000FA209847C4F307467FE73B4B1B68002B16
:10E370007FF478AF374B1B68002B98D0FB20984771
:10E38000C4F3074671E7354B1B68002B7FF46AAF77
:10E39000304B1B68002B8AD0F8209847C4F30746FF
:10E3A00063E70E2B7FF486AE2D4A2E4B1268E021D8
:10E3B0001970002A47D0260C610C06F07F0301F487
:10E3C0007E511943EDB2A1F5005128469047F6B2AF
:10E3D000240E39E7FFF740FDC4F30740FFF73CFD8B
:10E3E000200EFFF739FD0020BDE8F0811E4B1D4ACD
:10E3F0001B6880211170EDB2C4F3074683B131462A
:10E4000028463A4698473C461EE70120BDE8F08181
:10E41000104B1B68002B3FF44AAFFF20984746E79C
:10E420001C4611E70D2EBCD10D2B7FF443AE0F4BD4
:10E430000C4A1B68D0211170EDB2C4F30746002BC3
:10E440007FF4FEAEC4E7C4F30746EDB2240EFBE64C
:10E4500068A0FF1F44A0FF1F48A0FF1F38A0FF1F98
:10E4600054A0FF1FF4A1FF1F8CA0FF1F64A0FF1F7B
:10E4700038B5164D2868E0B101884488A14213DD03
:10E4800003191B7A83B104F10803C2180C1B002383
:10E4900002E012F8011F21B10133A342F9D1204655
:10E4A00038BD1C46204638BDFFF7B0FC0020286070
:10E4B00038BD074B1B780BB9002038BD0220FEF792
:10E4C000F5FD28600028D7D1F6E700BFA0A0FF1F08
:10E4D00030A0FF1F0D4B1B78BBB910B50C4C216849
:10E4E00003F0FF024B883F2B07DC07330B4401F19D
:10E4F000470003F8012F8342FBD140230B8001200A
:10E50000FEF76CFE0023236010BD704798A0FF1F2C
:10E510009CA0FF1F38B5224C237803B138BD0123DE
:10E520002370FFF7A5FF70BB00F048F840BB00F078
:10E53000DBF810BBFEF7F8FCE0B900232370EFF323
:10E540000583002BEAD1EFF3108172B6154B1868E2
:10E55000E0B1154C2278CAB945691D6001232370CA
:10E56000C5B1AA6101B962B60025457783689847AD
:10E570002570D3E700F020F8DFE700F01BF8D9E7BB
:10E5800000F016F8D3E7FFF71FFCCDE70029C5D14F
:10E5900062B638BD054B1D600029E5D1E3E700BF39
:10E5A000A5A0FF1FBC9EFF1FC09EFF1FB89EFF1FA0
:10E5B000704700BF704700BF704700BF054A064B59
:10E5C00010781B78C0B2DBB2984238BF4030C01A16
:10E5D000704700BFACA0FF1FADA0FF1FF0B4384BC9
:10E5E0001A7912F0300F2CD072B6997D01F0FF022B
:10E5F00000293DD062B6334F334938780D78334E19
:10E600001C46C0B2EDB2431C402BE17928BF002369
:10E61000AB4202F1FF32C9B21CBFF154184612F0EE
:10E62000FF02F0D12A4B1B68C2B23A704BB1A8422C
:10E6300036BFC5F14005401B40192728C4BF012241
:10E640001A701F49CA78D2B2150616D452060DD5D3
:10E650001B4B1B795B0609D51E4B1F491B6800220B
:10E660000A7003B11A70164B3C22DA70F0BC704786
:10E670004022D9795A7462B6E3E70B791C06E5D5D6
:10E68000164B174E1C783378E4B2DBB29C420ED0A6
:10E69000144D01E0A3420AD00133402B28BF0023D0
:10E6A0000879E85CC0B2C871087D0728F2D9DBB2EE
:10E6B000034933700B79180644BF7C23CB70C5E740
:10E6C00000A00640ACA0FF1FADA0FF1FF0A0FF1FE1
:10E6D000A8A0FF1F34A1FF1F30A1FF1F38A1FF1FFB
:10E6E00031A1FF1FB0A0FF1F054A064B10781B7811
:10E6F000C0B2DBB2984238BF4030C01A704700BF8A
:10E70000ACA1FF1F41A1FF1FF0B4384B1A7912F0E2
:10E71000300F2CD072B6997D01F0FF0200293DD058
:10E7200062B6334F334938780D78334E1C46C0B249
:10E73000EDB2431C402BE17928BF0023AB4202F12C
:10E74000FF32C9B21CBFF154184612F0FF02F0D1DB
:10E750002A4B1B68C2B23A704BB1A84236BFC5F112
:10E760004005401B40192728C4BF01221A701F49C9
:10E77000CA78D2B2150616D452060DD51B4B1B799A
:10E780005B0609D51E4B1F491B6800220A7003B1A6
:10E790001A70164B3C22DA70F0BC70474022D979CF
:10E7A0005A7462B6E3E70B791C06E5D5164B174E93
:10E7B0001C783378E4B2DBB29C420ED0144D01E0F9
:10E7C000A3420AD00133282B28BF00230879E85C34
:10E7D000C0B2C871087D0728F2D9DBB20349337093
:10E7E0000B79180644BF7C23CB70C5E700B0064008
:10E7F000ACA1FF1F41A1FF1F6CA1FF1F3CA1FF1F88
:10E80000B0A1FF1F40A1FF1FB4A1FF1FADA1FF1FBB
:10E8100044A1FF1F70B584B072B6194B194D1A4848
:10E82000702241260F2480211A702E701A4604701F
:10E83000197013781B06FCD5144B186862B6144B7C
:10E84000144C984298BF00EB800001A998BF40008B
:10E850000A22FDF7CFFE01A92046002311F8012B63
:10E8600001333AB10A2B20F8022FF7D11623237077
:10E8700004B070BD5B00DBB2237004B070BD00BF9C
:10E88000000002400700024006000240080002406B
:10E890007F969800DC92FF1F2DE9F043DFF8EC80B3
:10E8A0008BB006460F4600F073F898F9003001333C
:10E8B00004460D4637D03046394600F0DFF90028CF
:10E8C00031D02BA3D3E900233046394600F026FE91
:10E8D000814668BB28A3D3E900233046394600F0BF
:10E8E000FFFD00B398F90030254ACDF820900424AC
:10E8F00000200021022BCDE90467CDE902670094D6
:10E900000192CDE906012CD0684600F0BDF940B374
:10E91000089B1BB101F0AAF9089B0360DDE9060121
:10E920000BB0BDE8F083204629460BB0BDE8F0836C
:10E93000134A98F90030019203210022CDE90467BF
:10E94000CDE90267009108922BB90E4B4FF060425F
:10E95000CDE90623D8E70C490020022BCDE90601BA
:10E96000D2D101F083F922230360D1E7AFF3008015
:10E97000EF39FAFE422E864051302DD5104987C01E
:10E980003C340100FFFFEF470000F07FF292FF1FD1
:10E990002DE9F04FB04F21F00042BA4283B00C464F
:10E9A0004FEAD17605460DD9AC4FBA4225D9C1F30D
:10E9B0001303034340F0EF800EB10020014603B083
:10E9C000BDE8F08FA64B9A4200F2CC80A54B9A424C
:10E9D00000F2DE808AA3D3E9002300F05DF9002273
:10E9E000A14B00F09BFD002800F005812846214640
:10E9F00000229D4B00F050F9E1E783A3D3E9002307
:10EA000000F08CFD002840F0CB802846214680A3F2
:10EA1000D3E9002300F064FD0028CED1934B2846B3
:10EA200003EBC60821467CA3D3E9002300F0E6FAF5
:10EA3000D8E9002300F030F900F07AFD804600F0BC
:10EA400077FA77A3D3E9002306460F4600F0D6FAFB
:10EA500002460B462846214600F01CF972A3D3E972
:10EA60000023CDE900013046394600F0C7FA82465E
:10EA70008B4652465B46DDE9000100F00BF9054686
:10EA80000C462A4623462846214600F0B7FA68A3DA
:10EA9000D3E9002306460F4600F0B0FA66A3D3E997
:10EAA000002300F0F7F832463B4600F0A7FA64A3D3
:10EAB000D3E9002300F0F0F832463B4600F09EFA1E
:10EAC00061A3D3E9002300F0E5F832463B4600F0AD
:10EAD00095FA5FA3D3E9002300F0DEF832463B4607
:10EAE00000F08CFA02460B462846214600F0D2F888
:10EAF00006460F462846214632463B46B8F1000FEF
:10EB000056D000F07BFA324604460D463B460020C4
:10EB10004FF0804100F0BEF802460B4620462946E1
:10EB200000F096FB02460B465046594600F0B2F8FC
:10EB3000DDE9002300F0AEF80B4602464A4900200A
:10EB400000F0A8F86FF47F7398454FDA08F57A78EB
:10EB500001EB085100224FF0B87300F04FFA03B0F8
:10EB6000BDE8F08F424B9A423FF658AF414BF4005C
:10EB70002344D3E9002300F08DF83F4BC6F1010890
:10EB80001C44CDE90001D4E900ABC6EB080870E7EE
:10EB90004FF0000875E702460B4600F07DF80EE7DF
:10EBA00017A3D3E900231046194600F027FA06E719
:10EBB00000F024FA0022804689464FF08043304618
:10EBC000394600F067F802460B464046494600F0D9
:10EBD0003FFB2A46234600F05DF802460B46002024
:10EBE000214900F057F803B0BDE8F08F01EB085160
:10EBF00003B0BDE8F08F804643E700BFAFF300806D
:10EC00009C7500883CE4377EEF39FAFE422E864040
:10EC100051302DD5104987C0FE822B654715F73F2F
:10EC20000000E0FE422EE63F763C7935EF39EA3DC2
:10EC3000D0A4BE726937663EF16BD2C541BDBB3E02
:10EC40002CDE25AF6A56113F93BDBE166CC1663FE0
:10EC50003E5555555555C53F412E8640FFFFEF7F28
:10EC6000422ED63FFFFF2F3E0000F03F4034010010
:10EC7000B1A2F03F603401005034010041F0004186
:10EC800001F58010C00F70470020704781F00041EF
:10EC900002E000BF83F0004330B54FEA41044FEA81
:10ECA000430594EA050F08BF90EA020F1FBF54EA1C
:10ECB000000C55EA020C7FEA645C7FEA655C00F0B8
:10ECC000E2804FEA5454D4EB5555B8BF6D420CDD89
:10ECD0002C4480EA020281EA030382EA000083EA0C
:10ECE000010180EA020281EA0303362D88BF30BDAC
:10ECF00011F0004F4FEA01314FF4801C4CEA113102
:10ED000002D0404261EB410113F0004F4FEA033360
:10ED10004CEA133302D0524263EB430394EA050FEB
:10ED200000F0A780A4F10104D5F1200E0DDB02FA5A
:10ED30000EFC22FA05F2801841F1000103FA0EF2EE
:10ED4000801843FA05F359410EE0A5F120050EF1B4
:10ED5000200E012A03FA0EFC28BF4CF0020C43FAE5
:10ED600005F3C01851EBE37101F0004507D54FF0F2
:10ED7000000EDCF1000C7EEB00006EEB0101B1F542
:10ED8000801F1BD3B1F5001F0CD349085FEA300088
:10ED90004FEA3C0C04F101044FEA445212F5800F93
:10EDA00080F09A80BCF1004F08BF5FEA500C50F130
:10EDB000000041EB045141EA050130BD5FEA4C0C13
:10EDC000404141EB010111F4801FA4F10104E9D19C
:10EDD00091F0000F04BF01460020B1FA81F308BF93
:10EDE0002033A3F10B03B3F120020CDA0C3208DD5F
:10EDF00002F1140CC2F10C0201FA0CF021FA02F13A
:10EE00000CE002F11402D8BFC2F1200C01FA02F1A9
:10EE100020FA0CFCDCBF41EA0C019040E41AA2BFCE
:10EE200001EB0451294330BD6FEA04041F3C1CDA96
:10EE30000C340EDC04F11404C4F1200220FA04F0B6
:10EE400001FA02F340EA030021FA04F345EA030160
:10EE500030BDC4F10C04C4F1200220FA02F001FA22
:10EE600004F340EA0300294630BD21FA04F02946A4
:10EE700030BD94F0000F83F4801306BF81F480113D
:10EE80000134013D4EE77FEA645C18BF7FEA655CB0
:10EE900029D094EA050F08BF90EA020F05D054EA82
:10EEA000000C04BF1946104630BD91EA030F1EBF87
:10EEB0000021002030BD5FEA545C05D1400049418B
:10EEC00028BF41F0004130BD14F580043CBF01F57E
:10EED000801130BD01F0004545F0FE4141F4700164
:10EEE0004FF0000030BD7FEA645C1ABF194610463F
:10EEF0007FEA655C1CBF0B46024650EA013406BF40
:10EF000052EA033591EA030F41F4002130BD00BFFE
:10EF100090F0000F04BF0021704730B54FF48064BB
:10EF200004F132044FF000054FF0000150E700BF3C
:10EF300090F0000F04BF0021704730B54FF480649B
:10EF400004F1320410F0004548BF40424FF0000188
:10EF50003EE700BF42004FEAE2014FEA31014FEACB
:10EF600002701FBF12F07F4393F07F4F81F060511A
:10EF7000704792F0000F14BF93F07F4F704730B589
:10EF80004FF4607401F0004521F0004120E700BF1C
:10EF900050EA010208BF704730B54FF000050AE0A3
:10EFA00050EA010208BF704730B511F0004502D5A4
:10EFB000404261EB41014FF4806404F132045FEAA6
:10EFC000915C3FF4DCAE4FF003025FEADC0C18BF4B
:10EFD00003325FEADC0C18BF033202EBDC02C2F141
:10EFE000200300FA03FC20FA02F001FA03FE40EAD3
:10EFF0000E0021FA02F11444C1E600BF70B54FF0D3
:10F00000FF0C4CF4E06C1CEA11541DBF1CEA1355B4
:10F0100094EA0C0F95EA0C0F00F0DEF82C4481EA1C
:10F02000030621EA4C5123EA4C5350EA013518BF3C
:10F0300052EA033541F4801143F4801338D0A0FB29
:10F0400002CE4FF00005E1FB02E506F00042E0FBD6
:10F0500003E54FF00006E1FB03569CF0000F18BFDC
:10F060004EF0010EA4F1FF04B6F5007F64F5407484
:10F0700004D25FEA4E0E6D4146EB060642EAC62117
:10F0800041EA55514FEAC52040EA5E504FEACE2E84
:10F09000B4F1FD0C88BFBCF5E06F1ED8BEF1004F87
:10F0A00008BF5FEA500E50F1000041EB045170BD03
:10F0B00006F0004646EA010140EA020081EA030147
:10F0C000B4EB5C04C2BFD4EB0C0541EA045170BD43
:10F0D00041F480114FF0000E013C00F3AB8014F1BD
:10F0E000360FDEBF002001F0004170BDC4F1000406
:10F0F000203C35DA0C341BDC04F11404C4F1200587
:10F1000000FA05F320FA04F001FA05F240EA0200E1
:10F1100001F0004221F0004110EBD37021FA04F617
:10F1200042EB06015EEA430E08BF20EAD37070BDD1
:10F13000C4F10C04C4F1200500FA04F320FA05F030
:10F1400001FA04F240EA020001F0004110EBD37032
:10F1500041F100015EEA430E08BF20EAD37070BDA2
:10F16000C4F1200500FA05F24EEA020E20FA04F37B
:10F1700001FA05F243EA020321FA04F001F000412A
:10F1800021FA04F220EA020000EBD3705EEA430E9B
:10F1900008BF20EAD37070BD94F0000F0FD101F0CA
:10F1A0000046400041EB010111F4801F08BF013C03
:10F1B000F7D041EA060195F0000F18BF704703F041
:10F1C0000046520043EB030313F4801F08BF013DC8
:10F1D000F7D043EA0603704794EA0C0F0CEA135584
:10F1E00018BF95EA0C0F0CD050EA410618BF52EA3E
:10F1F0004306D1D181EA030101F000414FF0000044
:10F2000070BD50EA410606BF1046194652EA430651
:10F2100019D094EA0C0F02D150EA013613D195EAC5
:10F220000C0F05D152EA03361CBF104619460AD10D
:10F2300081EA030101F0004141F0FE4141F4700117
:10F240004FF0000070BD41F0FE4141F4780170BD07
:10F2500070B54FF0FF0C4CF4E06C1CEA11541DBF6C
:10F260001CEA135594EA0C0F95EA0C0F00F0A7F86E
:10F27000A4EB050481EA030E52EA03354FEA01319B
:10F2800000F088804FEA03334FF0805545EA1313AE
:10F2900043EA12634FEA022245EA111545EA106576
:10F2A0004FEA00260EF000419D4208BF964244F10D
:10F2B000FD0404F5407402D25B084FEA3202B61A2C
:10F2C00065EB03055B084FEA32024FF480104FF400
:10F2D000002CB6EB020E75EB030E22BFB61A754674
:10F2E00040EA0C005B084FEA3202B6EB020E75EB07
:10F2F000030E22BFB61A754640EA5C005B084FEA6F
:10F300003202B6EB020E75EB030E22BFB61A75463B
:10F3100040EA9C005B084FEA3202B6EB020E75EB46
:10F32000030E22BFB61A754640EADC0055EA060E07
:10F3300018D04FEA051545EA16754FEA06164FEA4A
:10F34000C30343EA52734FEAC2025FEA1C1CC0D1F6
:10F3500011F4801F0BD141EA00014FF000004FF083
:10F36000004CB6E711F4801F04BF01430020B4F144
:10F37000FD0C88BFBCF5E06F3FF6AFAEB5EB030CFC
:10F3800004BFB6EB020C5FEA500C50F1000041EBF9
:10F39000045170BD0EF0004E4EEA113114EB5C04C6
:10F3A000C2BFD4EB0C0541EA045170BD41F4801199
:10F3B0004FF0000E013C90E645EA060E8DE60CEAA1
:10F3C000135594EA0C0F08BF95EA0C0F3FF43BAFBE
:10F3D00094EA0C0F0AD150EA01347FF434AF95EA75
:10F3E0000C0F7FF425AF104619462CE795EA0C0F59
:10F3F00006D152EA03353FF4FDAE1046194622E726
:10F4000050EA410618BF52EA43067FF4C5AE50EAFF
:10F4100041047FF40DAF52EA43057FF4EBAE12E7EF
:10F420004FF0FF3C06E000BF4FF0010C02E000BFD0
:10F430004FF0010C4DF804CD4FEA410C7FEA6C5CB3
:10F440004FEA430C18BF7FEA6C5C1BD001B050EA56
:10F45000410C0CBF52EA430C91EA030F02BF90EA41
:10F46000020F0020704710F1000F91EA030F58BF00
:10F47000994208BF90422CBFD8176FEAE37040F062
:10F48000010070474FEA410C7FEA6C5C02D150EA00
:10F49000013C07D14FEA430C7FEA6C5CD6D152EABB
:10F4A000033CD3D05DF8040B704700BF8446104680
:10F4B00062468C461946634600E000BF01B5FFF77F
:10F4C000B7FF002848BF10F1000F01BD4DF808ED4F
:10F4D000FFF7F4FF0CBF012000205DF808FB00BF20
:10F4E0004DF808EDFFF7EAFF34BF012000205DF87A
:10F4F00008FB00BF4DF808EDFFF7E0FF94BF0120C7
:10F5000000205DF808FB00BF4DF808EDFFF7CEFFC7
:10F5100094BF012000205DF808FB00BF4DF808ED06
:10F52000FFF7C4FF34BF012000205DF808FB00BFD7
:10F530004FEA410212F5001215D211D56FF478731B
:10F54000B3EB625212D94FEAC12343F0004343EABE
:10F55000505311F0004F23FA02F018BF4042704799
:10F560004FF00000704750EA013005D111F0004023
:10F5700008BF6FF0004070474FF00000704700BFB9
:10F580004FEA4102B2F1E04324BFB3F5001CDCF1C5
:10F59000FE5C0DD901F0004C4FEAC0024CEA5070FD
:10F5A000B2F1004F40EB830008BF20F0010070472C
:10F5B00011F0804F21D113F13872BCBF01F000402F
:10F5C000704741F480114FEA5252C2F11802C2F161
:10F5D000200C10FA0CF320FA02F018BF40F00100E2
:10F5E0004FEAC1234FEAD32303FA0CFC40EA0C0094
:10F5F00023FA02F34FEA4303CCE77FEA625307D1D1
:10F6000050EA01331EBF4FF0FE4040F44000704707
:10F6100001F0004040F0FE4040F40000704700BFA1
:10F6200080F0004002E000BF81F0004142001FBFB7
:10F630005FEA410392EA030F7FEA226C7FEA236CC0
:10F640006AD04FEA1262D2EB1363C1BFD2184140B5
:10F6500048404140B8BF5B42192B88BF704710F04B
:10F66000004F40F4000020F07F4018BF404211F0EE
:10F67000004F41F4000121F07F4118BF494292EA56
:10F68000030F3FD0A2F1010241FA03FC10EB0C0082
:10F69000C3F1200301FA03F100F0004302D549420F
:10F6A00060EB4000B0F5000F13D3B0F1807F06D3BC
:10F6B00040084FEA310102F10102FE2A51D2B1F1B4
:10F6C000004F40EBC25008BF20F0010040EA0300A9
:10F6D0007047490040EB000010F4000FA2F1010256
:10F6E000EDD1B0FA80FCACF1080CB2EB0C0200FAE0
:10F6F0000CF0AABF00EBC25052421843BCBFD0402E
:10F700001843704792F0000F81F4000106BF80F4A7
:10F7100000000132013BB5E74FEA41037FEA226C6A
:10F7200018BF7FEA236C21D092EA030F04D092F035
:10F73000000F08BF0846704790EA010F1CBF002069
:10F74000704712F07F4F04D1400028BF40F00040C6
:10F75000704712F100723CBF00F50000704700F0E6
:10F76000004343F0FE4040F4000070477FEA22620D
:10F7700016BF08467FEA23630146420206BF5FEADE
:10F78000412390EA010F40F4800070474FF00003DE
:10F7900004E000BF10F0004348BF40425FEA000CA5
:10F7A00008BF704743F0964301464FF000001CE04D
:10F7B00050EA010208BF70474FF000030AE000BFA3
:10F7C00050EA010208BF704711F0004302D54042E1
:10F7D00061EB41015FEA010C02BF84460146002053
:10F7E00043F0B64308BFA3F18053A3F50003BCFA6E
:10F7F0008CF2083AA3EBC25310DB01FA02FC63441B
:10F8000000FA02FCC2F12002BCF1004F20FA02F221
:10F8100043EB020008BF20F00100704702F1200214
:10F8200001FA02FCC2F1200250EA4C0021FA02F275
:10F8300043EB020008BF20EADC7070474FF0FF0C7A
:10F840001CEAD0521EBF1CEAD15392EA0C0F93EA75
:10F850000C0F6FD01A4480EA010C400218BF5FEA17
:10F8600041211ED04FF0006343EA501043EA51118A
:10F87000A0FB01310CF00040B1F5000F3EBF490084
:10F8800041EAD3715B0040EA010062F17F02FD2A88
:10F890001DD8B3F1004F40EBC25008BF20F001006B
:10F8A000704790F0000F0CF0004C08BF49024CEA82
:10F8B000502040EA51207F3AC2BFD2F1FF0340EA14
:10F8C000C250704740F400004FF00003013A5DDC85
:10F8D00012F1190FDCBF00F000407047C2F10002C6
:10F8E000410021FA02F1C2F1200200FA02FC5FEAB3
:10F8F000310040F1000053EA4C0308BF20EADC70FD
:10F90000704792F0000F00F0004C02BF400010F46E
:10F91000000F013AF9D040EA0C0093F0000F01F01B
:10F92000004C02BF490011F4000F013BF9D041EA3D
:10F930000C018FE70CEAD15392EA0C0F18BF93EA3F
:10F940000C0F0AD030F0004C18BF31F0004CD8D169
:10F9500080EA010000F00040704790F0000F17BFF0
:10F9600090F0004F084691F0000F91F0004F14D036
:10F9700092EA0C0F01D142020FD193EA0C0F03D18E
:10F980004B0218BF084608D180EA010000F0004091
:10F9900040F0FE4040F40000704740F0FE4040F46C
:10F9A000400070474FF0FF0C1CEAD0521EBF1CEA0B
:10F9B000D15392EA0C0F93EA0C0F69D0A2EB030229
:10F9C00080EA010C49024FEA402037D04FF08053C3
:10F9D00043EA111143EA10130CF000408B4238BF88
:10F9E0005B0042F17D024FF4000C8B4224BF5B1A96
:10F9F00040EA0C00B3EB510F24BFA3EB510340EAE4
:10FA00005C00B3EB910F24BFA3EB910340EA9C0091
:10FA1000B3EBD10F24BFA3EBD10340EADC001B0101
:10FA200018BF5FEA1C1CE0D1FD2A3FF650AF8B42A5
:10FA300040EBC25008BF20F0010070470CF0004CB2
:10FA40004CEA50207F32C2BFD2F1FF0340EAC250DD
:10FA5000704740F400004FF00003013A37E792F09E
:10FA6000000F00F0004C02BF400010F4000F013AFC
:10FA7000F9D040EA0C0093F0000F01F0004C02BFF7
:10FA8000490011F4000F013BF9D041EA0C0195E760
:10FA90000CEAD15392EA0C0F08D142027FF47DAFF9
:10FAA00093EA0C0F7FF470AF084676E793EA0C0FE9
:10FAB00004D14B023FF44CAF08466EE730F0004CE7
:10FAC00018BF31F0004CCAD130F000427FF45CAF77
:10FAD00031F000437FF43CAF5FE700BF4FF0FF3CE5
:10FAE00006E000BF4FF0010C02E000BF4FF0010C38
:10FAF0004DF804CD4FEA40024FEA41037FEA226C01
:10FB000018BF7FEA236C11D001B052EA530C18BF22
:10FB100090EA010F58BFB2EB030088BFC81738BF87
:10FB20006FEAE17018BF40F0010070477FEA226C75
:10FB300002D15FEA402C05D17FEA236CE4D15FEA71
:10FB4000412CE1D05DF8040B704700BF84460846A5
:10FB50006146FFE70FB5FFF7C9FF002848BF10F166
:10FB6000000F0FBD4DF808EDFFF7F4FF0CBF0120AB
:10FB700000205DF808FB00BF4DF808EDFFF7EAFF35
:10FB800034BF012000205DF808FB00BF4DF808EDF0
:10FB9000FFF7E0FF94BF012000205DF808FB00BFE5
:10FBA0004DF808EDFFF7D2FF94BF012000205DF86B
:10FBB00008FB00BF4DF808EDFFF7C8FF34BF012078
:10FBC00000205DF808FB00BF4FEA4002B2F1FE4F93
:10FBD0000FD34FF09E03B3EB12620DD94FEA00230F
:10FBE00043F0004310F0004F23FA02F018BF4042E8
:10FBF00070474FF00000704712F1610F01D14202CF
:10FC000005D110F0004008BF6FF0004070474FF082
:10FC10000000704742000ED2B2F1FE4F0BD34FF0FE
:10FC20009E03B3EB126209D44FEA002343F0004372
:10FC300023FA02F070474FF00000704712F1610F95
:10FC400001D1420202D14FF0FF3070474FF0000067
:10FC5000704700BF0B460146184600F001B800BFD0
:10FC600013460A460146022000F0BCBE014B18684C
:10FC7000704700BF2097FF1F70B50F4E0F4D761BCA
:10FC8000B61018BF002405D0013455F8043B98473E
:10FC9000A642F9D10A4E0B4D761B03F0EBFBB610D2
:10FCA00018BF002406D0013455F8043B9847A642FB
:10FCB000F9D170BD70BD00BF8034010080340100F7
:10FCC0009434010080340100024B0146186800F0B2
:10FCD0000BB800BF2097FF1F024B0146186800F0C9
:10FCE00045BF00BF2097FF1F2DE9F04F01F10B0525
:10FCF000162D83B0064640F29F8035F0070500F1CF
:10FD0000BF80A94200F2BC8000F058FBB5F5FC7F33
:10FD1000C0F09C826B0A00F0BA80042B00F2838151
:10FD2000A80900F1390E4FEA4E033830C44F07EBF3
:10FD30008303A3F108015C68A14207D1ACE0002A6B
:10FD400080F2AC80E468A14200F0A680636823F0F2
:10FD500003035A1B0F2AF2DDB9493C6901F1080E71
:10FD6000744500F0B381636823F003035A1B0F2A24
:10FD700000F39981002AC1F814E0C1F810E080F284
:10FD80009E80B3F5007F80F06781DB0803F1010CF2
:10FD900001229B1002FA03F34A6851F83C80C4F830
:10FDA000088001EBCC091A43A9F10803E3604A601B
:10FDB00041F83C40C8F80C40831001249C40944218
:10FDC00000F28A80144206D120F00300640014423D
:10FDD00000F10400FAD007EBC009CC468046DCF8FD
:10FDE0000C108C4507D173E1002A80F28181C9682B
:10FDF0008C4500F06D814B6823F003035A1B0F2ADA
:10FE0000F2DD0C46D1F80CC054F8088F4B1945F0C0
:10FE100001054D6042F00101C8F80CC03046CCF835
:10FE200008807B613B61C3F80CE0C3F808E05960CF
:10FE30009A5000F0C5FA1FE0102921D800F0BEFA50
:10FE40001025062302207E4F07EB8303A3F108024F
:10FE50005C68944200F045816368E168A56823F01E
:10FE60000303234430465A68E96042F001028D6082
:10FE70005A6000F0A5FA0834204603B0BDE8F08FC0
:10FE800000240C232046336003B0BDE8F08F8023AC
:10FE90004FF0400E3F2049E770465DE72344E1689C
:10FEA0005A68A56842F00102E96030468D605A60E8
:10FEB00000F086FA0834204603B0BDE8F08F2344F2
:10FEC00030465A6842F001025A6000F079FA08346C
:10FED000204603B0BDE8F08FBC68636823F00308D8
:10FEE000A84504D3C5EB08030F2B00F38C80554BBA
:10FEF000DFF860911A68D9F8003001332A4404EB26
:10FF0000080A00F0608102F580520F3222F47F620D
:10FF100022F00F0211463046019200F04BFCB0F186
:10FF2000FF3F8346019A00F05881824500F2FC8031
:10FF3000454B1968DA451144196000F05381D9F82E
:10FF40000000DFF810E101301BBFCAEB0B0A51447F
:10FF5000CEF800B019601BF0070100F01781C1F165
:10FF60000800C1F58051834408315A44C2F30B02A2
:10FF7000C2EB010949463046019300F01BFC431CCB
:10FF8000019B00F03F81CBEB00024A4442F00102AA
:10FF90001968C7F808B04944BC42CBF8042019607E
:10FFA000DFF8A49016D0B8F10F0F40F2FD80626820
:10FFB000A8F10C0323F00703E01802F001024FF050
:10FFC000050E1A430F2B6260C0F804E0C0F808E089
:10FFD00000F21C811D4BBC681A68914288BF1960F1
:10FFE0001B4B1A689142626888BF196022F00302B5
:10FFF0009542A2EB050301D80F2B04DC304600F03C
:020000021000EC
:10000000DFF9002438E7621943F0010345F00105E8
:1000100065603046BA60536000F0D2F9083420467B
:1000200003B0BDE8F08F142B71D9542B00F2A480DB
:10003000280B00F16F0E4FEA4E036E3076E600BFDC
:100040002497FF1FC0A1FF1FC4A1FF1FBCA1FF1F5A
:10005000B8A1FF1F309BFF1F5A0A042A5ED9142A39
:1000600000F2B38002F15C0149005B3207EB810CC6
:1000700057F82110DFF8DC81ACF1080C8C4500F05A
:1000800088804A6822F00302934202D289688C4534
:10009000F7D1D1F80CC07A68C4F80CC0A160CCF8D4
:1000A0000840CC6088E6631942F0010745F001057D
:1000B000656030464B610B61C3F80CE0C3F808E0A3
:1000C0005F609A50083400F07BF9D5E64A6873E621
:1000D00008F1010818F0030F0CF1080C7FF47FAE53
:1000E00030E0DC68A34208BF02303FF435AEB3E62F
:1000F0000B440C465A68C96854F8085F42F0010284
:100100005A603046E9608D6000F05AF9B4E603F1B8
:100110005C0E03F15B004FEA4E0307E69A0902F119
:10012000390149003832A1E7BC424A4B3FF400AFE5
:100130009C68626822F003025AE759F80839994529
:1001400040F0828010F0030F00F1FF30F5D17B68A2
:1001500023EA04037B6064009C423FF6BDAE002CA2
:100160003FF4BAAE1C4240467FF435AE64001C42F8
:1001700000F10400FAD02EE6B3F5AA7F18D8E80BF8
:1001800000F1780E4FEA4E037730CFE54FF48051FF
:10019000EBE60121D8F80430921001FA02F21A437A
:1001A000C8F80420614677E70123CBF8043025E73F
:1001B00040F25452934220D8A80C00F17D0E4FEA31
:1001C0004E037C30B2E51032A4E6542A26D81A0B2E
:1001D00002F16F0149006E3248E7BC68626822F0A4
:1001E000030205E7CAF30B0000287FF4A8AE4244DF
:1001F000BB6842F001025A60ECE6FE234FF07F0E2E
:100200007E2093E501224FF00009C1E604F10801C8
:10021000304600F0ABFCD9F80010DBE6B2F5AA7F5F
:1002200005D8DA0B02F17801490077321EE740F277
:1002300054518A4205D89A0C02F17D0149007C3262
:1002400014E7FE217E2211E77B6884E7E808431C5F
:100250005B00F8E52497FF1F8842F0B50DD98B1895
:1002600098420AD28118002A51D09A1A13F8014DE7
:1002700001F8014D9342F9D1F0BD0F2A48D941EA66
:1002800000039B0746D100F1100401F1100315464D
:1002900053F8106C44F8106C53F80C6C44F80C6C68
:1002A00053F8086C44F8086C103D53F8046C44F89B
:1002B000046C0F2D03F1100304F11004E8D8A2F12F
:1002C000100323F00F0302F00F0E1033BEF1030FE3
:1002D0001944034421D91E1F0D467446043C55F8A9
:1002E000047B46F8047F032CF8D8AEF1040424F014
:1002F000030404342344214402F0030262B1013BAD
:100300000A4411F8014B03F8014F8A42F9D1F0BDBC
:100310000346F3E70346F2E7F0BD7246EEE700BF9F
:1003200070B4840746D0541E002A41D0CDB2034693
:1003300002E0621EE4B3144603F8015B9A07F8D1A9
:10034000032C2ED9CDB245EA05250F2C45EA0545EB
:1003500019D903F110022646103E0F2E42F8105C08
:1003600042F80C5C42F8085C42F8045C02F11002AE
:10037000F2D8A4F1100222F00F0204F00F041032A0
:10038000032C13440DD91E462246043A032A46F88C
:10039000045BFAD8221F22F003020432134404F053
:1003A00003042CB1C9B21C4403F8011BA342FBD1C6
:1003B00070BC704714460346C2E700BF704700BFD9
:1003C000704700BF024B0A460146186800F002B8A9
:1003D0002097FF1F2DE9F04F174683B0002900F04A
:1003E000C1800E46814607F10B05FFF7E7FF56F87F
:1003F00004EC162D2EF00304A6F1080840D81022B4
:100400001546AF4241D8944275DAC94B996808EB5A
:1004100004008842416800F0D98021F001030344C0
:100420005B68DB077DD51EF0010F35D039464846A5
:10043000FFF75AFC0746E0B156F8043C23F00103ED
:100440004344A0F108029A4200F04481221F242A6A
:1004500000F23181132A00F204810346324611680A
:1004600019605168596092689A603146484600F0B8
:100470007DFB4846FFF7A4FF384603B0BDE8F08F88
:1004800025F00705002D2A46BBDA0C230020C9F809
:10049000003003B0BDE8F08F56F8083CC3EB080A03
:1004A000DAF8043023F0030C04EB0C039342BDDBB9
:1004B0005746DAF80C1057F8080F221F242AC1609B
:1004C000886000F21781132A40F212813168CAF85D
:1004D00008107168CAF80C101B2A00F22B8108362C
:1004E0000AF110023168116071685160B168916061
:1004F0003E461C46D046631B0F2B1DD8D8F804304F
:1005000003F0010323434444C8F80430636843F014
:10051000010363604846FFF753FF304603B0BDE870
:10052000F08F21F003012144914221DBC3688268EE
:100530000C46D3609A60DEE7D8F8042008EB05018A
:1005400002F00102154343F001020B44C8F80450C5
:100550004A605A6842F0010208315A60484600F089
:1005600005FBD7E7114603B0BDE8F04FFFF7BCBB72
:100570001EF0010F7FF45AAF56F8083CC3EB080A8F
:10058000DAF8043023F0030C01EB0C0E96458BDBFC
:10059000C36882685746D3609A6057F8081FDAF834
:1005A0000C30CB60221F242A996000F29980132A14
:1005B00062D93368CAF808307368CAF80C301B2A4D
:1005C00000F2A08008360AF1100356E021F0030B78
:1005D000A34405F11000834559DA1EF0010F7FF4A2
:1005E00025AF56F8081CC1EB080ADAF8041021F010
:1005F000030CE34458453FF757AF5746DAF80C1061
:1006000057F8080F221F242AC160886000F2B480C6
:10061000132A40F2A5803168CAF808107168CAF838
:100620000C101B2A00F2AF8008360AF11002316864
:10063000116071685160B16891600AEB0501C5EB0A
:100640000B0242F0010299604A60DAF8043003F0CC
:1006500001031D434846CAF80450FFF7B1FE38466F
:100660005CE733680360736843601B2A27D800F196
:10067000080306F10802F2E63B4632681A60726827
:100680005A60B2689A603E467446D04633E708EB3B
:100690000501C5EB0B0B4BF0010299604A6056F85F
:1006A000043C03F001031D43484646F8045CFFF791
:1006B00087FE304632E73146FFF7CEFDD5E6B36818
:1006C0008360F368C360242A28D000F1100306F188
:1006D0001002C4E650F8043C23F003031C440AE76C
:1006E000314638467446D046FFF7B6FD3E4602E72F
:1006F0003A46F7E6314638461C46D046FFF7ACFD91
:100700003E46F8E6B368CAF81030F368CAF8143009
:10071000242A1BD010360AF11803AEE733690361AF
:100720007369436106F1180200F1180397E600BFF0
:100730002497FF1FB168CAF81010F168CAF81410A6
:10074000242A0FD010360AF11802CBE63369CAF812
:1007500018307369CAF81C3018360AF120038CE788
:100760003A4664E73269CAF818207269CAF81C2050
:1007700018360AF12002B5E6314638460193FFF7F4
:100780006BFD019B59E7B168CAF81010F168CAF80F
:100790001410242A03D010360AF1180247E73269F0
:1007A000CAF818207269CAF81C2018360AF120020B
:1007B0003DE700BF38B5074C0023054608462360D7
:1007C000FBF7E2FE431C00D038BD2368002BFBD0B2
:1007D0002B6038BD20A3FF1FFFFFFFFFFFFFFFFFC0
:1007E000FFFFFFFFFFFFFFFFFFFFFFFFFFFFFFFF19
:1007F000FFFFFFFFFFFFFFFFFFFFFFFFFFFFFFFF09
:1008000090F800F06DE9024520F007016FF0000C50
:1008100010F0070491F820F040F049804FF00004F8
:100820006FF00700D1E9002391F840F000F10800D3
:1008300082FA4CF2A4FA8CF283FA4CF3A2FA8CF30B
:100840004BBBD1E9022382FA4CF200F10800A4FA72
:100850008CF283FA4CF3A2FA8CF3E3B9D1E90423C6
:1008600082FA4CF200F10800A4FA8CF283FA4CF3FD
:10087000A2FA8CF37BB9D1E9062301F1200182FAB7
:100880004CF200F10800A4FA8CF283FA4CF3A2FABD
:100890008CF3002BC6D0002A04BF04301A4612BACB
:1008A000B2FA82F2FDE8024500EBD2007047D1E9CE
:1008B000002304F00305C4F100004FEAC50514F05D
:1008C000040F91F840F00CFA05F562EA05021CBF2E
:1008D00063EA050362464FF00004A9E7002A41D00D
:1008E00040EA010313F00303F0B425D1032A23D90E
:1008F00004680D68AC421FD1043A35D0A4F101352B
:1009000025EA040414F0803F31D1071D0D1D0DE0D0
:1009100057F8043B0E68A3F10134B34224EA030400
:100920000AD1043A20D014F0803F23D1032A29466B
:10093000384605F10405EBD803780C789C4202F1A7
:10094000FF320CD182B114B916E06AB17BB110F854
:10095000013F11F8014FA34202F1FF32F5D0181BFD
:10096000F0BC7047104670471046F0BC7047184600
:10097000F0BC70470020F3E72046F1E740EA0103AE
:100980009B0770B42BD1032A29D90C460346214674
:1009900054F8046BA6F1013525EA060515F0803FF1
:1009A00006D1043A032A43F8046B2146EFD8A2B1DA
:1009B0000C781C70013A013301313CB16AB111F875
:1009C000014B03F8014B013A002CF7D12AB11A442C
:1009D000002103F8011B9A42FBD170BC704703460B
:1009E000E5E700BF2DE9F047254C2568D5F84841DB
:1009F0000646884692469946C4B360681F2817DCAD
:100A0000431C76B104EB80050122C5F888A0D4F818
:100A1000881182401143022EC4F88811C5F808914C
:100A20001ED00230636044F820800020BDE8F087CB
:100A3000144B03B34FF4C870FFF746F90446D0B126
:100A4000D5F84831002780E88800C5F84841384685
:100A50000123C4F88871C4F88C71002EE1D0D1E76D
:100A6000D4F88C110A43C4F88C21DAE705F5A67492
:100A7000C5F84841C1E74FF0FF30BDE8F08700BF3F
:100A800070340100C9FC0000024B13B1024800F0B1
:100A900005B8704700000000A90A010000230146C4
:100AA0001A461846FFF79EBF38B5074D074C2C1B5A
:100AB000A41005D0013C55F8043D9847002CF9D10D
:100AC000BDE8384002F0E6BC000000000000000075
:100AD000F8B5234F0C460646FFF770FCBB685D680F
:100AE00025F00305291B01F6EF7121F47F6121F048
:100AF0000F01A1F58054B4F5805F07DB002130467B
:100B0000FFF758FEBB682B44984204D03046FFF7ED
:100B100057FC0020F8BD61423046FFF74BFE013024
:100B20000DD0104BBA6819682D1B45F001053046F1
:100B3000091B55601960FFF743FC0120F8BD002137
:100B40003046FFF737FEBA68831A0F2BDEDD064CFE
:100B50000449246843F00103001B53600860D5E793
:100B60002497FF1FC4A1FF1F309BFF1F002945D002
:100B70002DE9F0410D468046FFF720FC55F8047C36
:100B80006A4927F00103A5F10804E2188E6850684D
:100B9000B24220F0030062D0FE0750600BD455F83B
:100BA000087CE41B01F1080EA56875453B446FD035
:100BB000E768EF60BD6015186D68ED0742D543F03A
:100BC00001026260E350B3F5007F18D2DB085A1CC3
:100BD0004D6851F83270A76001209B1000FA03F3B2
:100BE00001EBC2001D430838E0604D6041F832401F
:100BF000FC604046BDE8F041FFF7E2BB70475A0A8F
:100C0000042A53D89A0902F139077F0002F1380506
:100C100001EB870051F827204449083890424DD015
:100C2000516821F003018B4202D292689042F7D1C1
:100C3000D068E060A2608460D4604046BDE8F041C6
:100C4000FFF7BEBB95683A4FBD4203443FD0D06822
:100C5000E86043F0010285606260E350B3E7FF079C
:100C6000034407D455F8082CA41A1344A068E2687A
:100C7000C26090602F4A126843F0010093426060A6
:100C80008C60B6D32C4B40461968FFF721FFB0E7C4
:100C900011184968C90744D49168D268CA600344EE
:100CA00043F0010091606060E350A2E7142A17D876
:100CB00002F15C077F0002F15B05A9E7AA104B680F
:100CC000012505FA02F213434B600246B1E743F0F7
:100CD00001024C610C61E560A5606260E35088E749
:100CE000542A06D81A0B02F16F077F0002F16E0535
:100CF0008EE7B2F5AA7F06D8DA0B02F178077F00FB
:100D000002F1770584E740F25450824206D89A0CEB
:100D100002F17D077F0002F17C0579E7FE277E2541
:100D200076E743F001026260E35062E72497FF1F19
:100D30002C97FF1F2C9BFF1FC0A1FF1F00007805F1
:100D40003408540B800C3C0F5C12E015FA19141E89
:100D50006022AC265C2B0C30BC34023AFF3FFFFF14
:100D6000FDFFFFFFFBFFFFFFF8FFFFFFFDFFFFFFA2
:100D7000FBFFFFFFF8FFFFFFFDFFFFFFFAFFFFFF95
:100D8000F7FFFFFFFDFFFFFFFBFFFFFFF7FFFFFF89
:100D9000FCFFFFFFFBFFFFFFF7FFFFFFFDFFFFFF74
:100DA000FAFFFFFFF7FFFFFFFDFFFFFFFBFFFFFF66
:100DB000F8FFFFFFFDFFFFFFFBFFFFFFF8FFFFFF57
:100DC000FDFFFFFFFAFFFFFFF7FFFFFFFCFFFFFF45
:100DD000FBFFFFFFF7FFFFFFFDFFFFFFFBFFFFFF35
:100DE000F7FFFFFFFDFFFFFFFAFFFFFFF7FFFFFF2A
:100DF000FDFFFFFFFBFFFFFFF7FFFFFFFDFFFFFF13
:100E0000FBFFFFFFF7FFFFFFFDFFFFFFFAFFFFFF05
:100E1000F7FFFFFFFDFFFFFFFAFFFFFFF8FFFFFFF8
:100E2000FDFFFFFFFAFFFFFFF7FFFFFFFDFFFFFFE3
:100E3000FAFFFFFFF7FFFFFFFDFFFFFFFAFFFFFFD6
:100E4000F8FFFFFFFDFFFFFFFAFFFFFFF8FFFFFFC7
:100E5000FDFFFFFFFAFFFFFFF7FFFFFFFCFFFFFFB4
:100E6000FBFFFFFFF7FFFFFFFDFFFFFFFAFFFFFFA5
:100E7000F7FFFFFFFDFFFFFFFAFFFFFFF7FFFFFF99
:100E8000FEFFFFFFFBFFFFFFF8FFFFFFFEFFFFFF7F
:100E9000FBFFFFFFF8FFFFFFFDFFFFFFFAFFFFFF74
:100EA000F7FFFFFFFCFFFFFFFAFFFFFFF7FFFFFF6A
:100EB000FCFFFFFFFAFFFFFFF7FFFFFFFDFFFFFF54
:100EC000FAFFFFFFF7FFFFFFFDFFFFFFF9FFFFFF47
:100ED000F7FFFFFFFDFFFFFFF9FFFFFFF7FFFFFF3A
:100EE000FDFFFFFFFAFFFFFFF7FFFFFFFDFFFFFF23
:100EF000FAFFFFFFF7FFFFFFFDFFFFFFFAFFFFFF16
:100F0000F6FFFFFFFDFFFFFFFAFFFFFFF7FFFFFF09
:100F1000FEFFFFFFFBFFFFFFF7FFFFFFFEFFFFFFEF
:100F2000FBFFFFFFF7FFFFFFFDFFFFFFFAFFFFFFE4
:100F3000F7FFFFFFFDFFFFFFFBFFFFFFF8FFFFFFD6
:100F4000FDFFFFFFFBFFFFFFF8FFFFFFFDFFFFFFC0
:100F5000FAFFFFFFF7FFFFFFFCFFFFFFF9FFFFFFB7
:100F6000F7FFFFFFFCFFFFFFF9FFFFFFF7FFFFFFAA
:100F7000FDFFFFFFFAFFFFFFF7FFFFFFFDFFFFFF92
:100F8000FAFFFFFFF7FFFFFFFDFFFFFFF9FFFFFF86
:100F9000F6FFFFFFFDFFFFFFFAFFFFFFF7FFFFFF79
:100FA000581501003415010010150100EC14010062
:100FB000A41101006010010084100100A8100100BC
:100FC000CC1001000C130100301301003C0D010096
:100FD000C811010000000000070000000C00000024
:100FE0001000000013000000180000001C000000AA
:100FF00000000000070000000C00000013000000CB
:10100000180000001F000000240000000000000085
:101010000C00000018000000240000003000000058
:101020003C0000004800000000000000FBFFFFFF44
:10103000F4FFFFFFEFFFFFFFE8FFFFFFE3FFFFFF0E
:10104000DCFFFFFF00000000F4FFFFFFE8FFFFFFF1
:10105000DCFFFFFFD0FFFFFFC4FFFFFFB8FFFFFF74
:101060000000580246056608540BD80E5C12E015C5
:10107000FA19141E6022AC265C2B0C30BC34023AE8
:10108000FF3FFFFF0000900120031405D0075A0A1C
:10109000AC0DCC10B4146A18E81C342180252A2B1E
:1010A00070301437FF3FFFFF0000C800F4018403D5
:1010B000140508072E091C0CD80EF811AE15961948
:1010C000401F1C25F22B5834FF3FFFFF0000640037
:1010D000C8009001BC021A04DC059E07F609800CCA
:1010E000A00F2413A2174C1D5424442FFF3FFFFFD1
:1010F000FBFFFFFFF8FFFFFFF4FFFFFFFAFFFFFF1B
:10110000F7FFFFFFF4FFFFFFFDFFFFFFF9FFFFFF0A
:10111000F4FFFFFFFAFFFFFFF7FFFFFFF4FFFFFF02
:10112000FCFFFFFFF7FFFFFFF4FFFFFFFBFFFFFFE9
:10113000F8FFFFFFF4FFFFFFFDFFFFFFFAFFFFFFD8
:10114000F4FFFFFFFDFFFFFFF9FFFFFFF4FFFFFFCD
:10115000FDFFFFFFF8FFFFFFF4FFFFFFFCFFFFFFB6
:10116000F7FFFFFFF4FFFFFFFBFFFFFFF8FFFFFFAD
:10117000F4FFFFFFFCFFFFFFF7FFFFFFF4FFFFFFA0
:1011800040067805B004E80384032003BC0258023B
:10119000F40190012C01FA00C800960064003200AE
:1011A0001900FFFF0000FF03FF07FF0BFF0FFF13F6
:1011B000FF17FF1BFF1FFF23FF27FF2BFF2FFF330F
:1011C000FF37FF3BFF3FFFFF0000D007800CD80E2A
:1011D0000010C012EC130C17FA19141E6022AC2672
:1011E0005C2B0C30BC34023AFF3FFFFFFBFFFFFFDC
:1011F000F8FFFFFFF4FFFFFFFAFFFFFFF7FFFFFF1E
:10120000F4FFFFFFFDFFFFFFF9FFFFFFF4FFFFFF0C
:10121000FAFFFFFFF7FFFFFFF4FFFFFFFCFFFFFFF9
:10122000F7FFFFFFF4FFFFFFFBFFFFFFF8FFFFFFEC
:10123000F4FFFFFFFDFFFFFFFAFFFFFFF4FFFFFFDB
:10124000FBFFFFFFF8FFFFFFF4FFFFFFFDFFFFFFC6
:10125000F8FFFFFFF4FFFFFFFCFFFFFFF7FFFFFFBB
:10126000F4FFFFFFFBFFFFFFF8FFFFFFF4FFFFFFAF
:10127000FCFFFFFFF7FFFFFFF4FFFFFFFBFFFFFF98
:10128000F8FFFFFFF6FFFFFFFAFFFFFFF8FFFFFF8A
:10129000F6FFFFFFFDFFFFFFFBFFFFFFF9FFFFFF73
:1012A000FDFFFFFFF9FFFFFFF7FFFFFFFEFFFFFF5F
:1012B000FCFFFFFFF7FFFFFFFBFFFFFFF8FFFFFF54
:1012C000F6FFFFFFFCFFFFFFFAFFFFFFF6FFFFFF48
:1012D000FDFFFFFFFBFFFFFFF9FFFFFFFCFFFFFF2D
:1012E000FAFFFFFFF6FFFFFFFEFFFFFFFCFFFFFF20
:1012F000F7FFFFFFFBFFFFFFF8FFFFFFF6FFFFFF1A
:10130000FEFFFFFFFCFFFFFFF7FFFFFF000058029B
:1013100046056608540BD80E5C127017FC21F82A9B
:1013200070305834DC37663A8C3C803EFF3FFFFF1C
:101330000000580246056608540BA00FD417282356
:10134000F82A442F643284354038663A8C3C803E1B
:10135000FF3FFFFF00000000070000000C0000003E
:1013600010000000130000001A0000001F00000021
:1013700000000000070000000C000000100000004A
:1013800013000000180000001C0000002C011301D5
:10139000FA00E100C800AF0096007D0064004B0039
:1013A0003200190000000000CDCC4C3DCDCCCC3D2E
:1013B0009A99193ECDCC4C3E0000803E9A99993EB8
:1013C0003333B33ECDCCCC3E6666E63EFBFFFFFF3B
:1013D000F7FFFFFFF6FFFFFFFBFFFFFFF7FFFFFF3A
:1013E000F6FFFFFFFBFFFFFFF7FFFFFFF6FFFFFF2B
:1013F000FDFFFFFFFCFFFFFFF8FFFFFFFDFFFFFF0B
:10140000FCFFFFFFF8FFFFFFFDFFFFFFFCFFFFFFFB
:10141000F8FFFFFFFBFFFFFFF7FFFFFFF6FFFFFFF8
:10142000FBFFFFFFF7FFFFFFF6FFFFFFFBFFFFFFE5
:10143000FAFFFFFFF8FFFFFFFCFFFFFFF9FFFFFFD1
:10144000F8FFFFFFFDFFFFFFFCFFFFFFF8FFFFFFBF
:10145000FCFFFFFFFAFFFFFFF7FFFFFFFBFFFFFFB0
:10146000F7FFFFFFF4FFFFFFFBFFFFFFF7FFFFFFAB
:10147000F4FFFFFFFBFFFFFFF7FFFFFFF4FFFFFF9E
:10148000FDFFFFFFF8FFFFFFF4FFFFFFFDFFFFFF82
:10149000F8FFFFFFF4FFFFFFFDFFFFFFF8FFFFFF77
:1014A000F4FFFFFFFBFFFFFFF7FFFFFFF4FFFFFF6E
:1014B000FBFFFFFFF7FFFFFFF4FFFFFFFBFFFFFF57
:1014C000F8FFFFFFF4FFFFFFFCFFFFFFF9FFFFFF47
:1014D000F4FFFFFFFDFFFFFFF8FFFFFFF4FFFFFF3B
:1014E000FCFFFFFFF7FFFFFFF4FFFFFF00007805A1
:1014F000220B0410B4143219B01DFC214826FE2919
:10150000822D383126344637663A223DFF3FFFFFB1
:101510000000D007100E88133219AA1E2823742742
:101520005C2B442F643284354038663A8C3C803ED4
:10153000FF3FFFFF0000540BEC13FA1908201C2595
:101540003629EC2C0C302C33E8357238663AF63BF1
:10155000863D163FFF3FFFFF0000CC10581BFC21CB
:10156000AC26C62A7C2E3831F4334C36A438983A4F
:101570005A3C543D803E7A3FFF3FFFFF0000000091
:10158000070000000C000000100000001300000025
:10159000180000001A000000070000000C00000006
:1015A0001000000013000000180000001A000000E6
:1015B0001F000000FBFFFFFFF7FFFFFFF4FFFFFF2F
:1015C000FBFFFFFFF7FFFFFFF4FFFFFFFDFFFFFF44
:1015D000F7FFFFFFF4FFFFFFFDFFFFFFF8FFFFFF37
:1015E000F4FFFFFFFAFFFFFFF7FFFFFFF4FFFFFF2E
:1015F000FBFFFFFFF7FFFFFFF4FFFFFFFBFFFFFF16
:10160000F7FFFFFFF4FFFFFFFBFFFFFFF7FFFFFF09
:10161000F4FFFFFFFDFFFFFFF8FFFFFFF4FFFFFFF9
:10162000FDFFFFFFF8FFFFFFF4FFFFFFFDFFFFFFE0
:10163000F8FFFFFFF4FFFFFFFAFFFFFFF8FFFFFFD8
:10164000F4FFFFFFB4160100109CFF1F0000FF0F06
:10165000BC9DFF1F0000FF0F9D5100008016010080
:10166000B49DFF1F32005E0100000000000000007A
:101670003D51000054485200534E53004D41580014
:10168000544F5543482053454E53450045585452F6
:101690004120434F4E54524F4C4C455200000000E5
:1016A00050495443482042454E4400004249544565
:1016B0000000000042524541544800FF8C160100D2
:1016C0000C9DFF1FF401A00F089DFF1FF401A00F48
:1016D00049510000AC160100789DFF1FBC025C124E
:1016E000909DFF1FBC025C1281510000A0160100FA
:1016F0005A9DFF1FF401A00FA29BFF1FF401A00F32
:101700006551000028200100302001001C2001004C
:101710002020010024200100901E0100E01F010094
:10172000FC1F01000020010004200100082001002E
:101730000C2001001020010014200100E81F01000E
:1017400018200100901E01008C1E0100F01F0100F6
:10175000F41F0100F81F0100901E0100E01F0100AE
:10176000E41F0100E81F0100EC1F0100CC1F010075
:10177000D01F0100D41F0100D81F0100DC1F010091
:1017800058270100C41F0100C81F010038200100B4
:101790003C200100402001004420010048200100BD
:1017A0004C2001005020010054200100582001006D
:1017B0005C2001006020010064200100682001001D
:1017C000010000006C200100070000000000000084
:1017D0000000000000000000000000000000000009
:1017E00000000000000000000000000000000000F9
:1017F00000000000000000000000000000000000E9
:1018000000000000000000000000000000000000D8
:1018100000000000000000000000000000000000C8
:1018200000000000000000000000000000000000B8
:1018300000000000000000000000000000000000A8
:101840000000000000000000000000000000000098
:101850000000000000000000000000000000000088
:101860000000000000000000000000000000000078
:101870000000000000000000000000000000000068
:101880000000000000000000000000000000000058
:101890000000000000000000000000000000000048
:1018A0000000000000000000000000000000000038
:1018B0000000000000000000000000000000000028
:1018C0000000000000000000000000000000000018
:1018D0000000000000000000000000000000000008
:1018E00000000000000000000000000000000000F8
:1018F0000001FFFFFFE360000773600000000000CD
:101900000001FFFFFFE360000EE360000000000045
:1019100000018000000360001DC3600000000000A3
:101920000001BFFFFFE360003B8360000000000098
:101930000001BFFFFFE360007703600000000000CC
:101940000001B00000036000EE0360000000000032
:101950000001B00000036001DC0360000000000033
:101960000001B00000036003B80360000000002025
:101970000001B00000036007700360000000006019
:101980000001BFFFFFE3600EE003600000000060A5
:101990000001BFFFFFE3601DC003600000030060A3
:1019A000000180000003603B80036000000300E052
:1019B0000001BFFFFFE3607700036000000300C089
:1019C0000001BFFFFFE360EE00036000000380C082
:1019D0000001B000000361DC00036000000780C06C
:1019E0000001B000000363B8000360000007C0C03E
:1019F0000001B00000036770000360000006C0C073
:101A00000001B00000036EE000036000000660C14A
:101A10000101B00000037DC000036000000630C378
:101A20000301BFFFFFE37B8000036000000C30C3B5
:101A30000701BFFFFFE3770000036000000C1CC339
:101A40000601800000030E0000036000000C0CC2C1
:101A50000E01FFFFFFE3FC0000036000000C0EC658
:101A60001E01FFFFFFE3F80000036000000C07C643
:101A70001E0000000000000000000000000C03C673
:101A8000760000000000000000000000000C01C70C
:101A9000E60000000000000000000000000C00C78D
:101AA000C60000000000000000000000000C000361
:101AB000060000000000000000000000000C000014
:101AC000000000000000000000000000000C00000A
:101AD0000000000000000000000000000000000006
:101AE00000000000000000000000000000000000F6
:101AF00000000000000000000000000000000000E6
:101B000000000000000000000000000000000000D5
:101B100000000000000000000000000000000000C5
:101B200000000000000000000000000000000000B5
:101B300000000000000000000000000000000000A5
:101B40000000000000000000000000000000000095
:101B50000000000000000000000000000000000085
:101B60000000000000000000000000000000000075
:101B70000000000000000000000000000000000065
:101B80000000000000000000000000000000000055
:101B90000000000000000000000000000000000045
:101BA0000000000000000000000000000000000035
:101BB0000000000000000000000000000000000025
:101BC0000000000000000000000000000000000015
:101BD000F822010004230100169DFF1F00000A00E7
:101BE0000100000041600000A95C0000000000004E
:101BF00000000000F023010084230100A49BFF1FCC
:101C00000000300000000000456F0000ED5B0000A8
